:020000040800F2
:1000000000000120FD3C0008C9250008CB250008A0
:10001000CD250008CF250008D125000800000000EC
:10002000000000000000000000000000D3250008D0
:10003000D525000800000000D7250008D9250008B4
:100040004D3D00084D3D0008DD2500084D3D0008F0
:100050004D3D00084D3D0008E9250008EF2500084A
:100060004D3D00084D3D00080D2600084D3D00089F
:10007000F5250008F7250008F9250008FB250008EC
:10008000FD250008012600084D3D00084D3D0008F3
:10009000000000004D3D00080F2600084D3D0008FF
:1000A0004D3D00084D3D00084D3D00084D3D000808
:1000B0004D3D00084D3D00084D3D00084D3D0008F8
:1000C0004D3D00084D3D00084D3D00084D3D0008E8
:1000D0004D3D0008192600084D3D00084D3D000823
:1000E0004D3D000811260008252600084D3D00085A
:1000F0004D3D000800000000000000004D3D0008DC
:100100004D3D00084D3D0008312600084D3D0008DA
:100110004D3D00084D3D00084D3D00084D3D000897
:100120004D3D00084D3D00084D3D00084D3D000887
:080130004D3D00084D3D0008A3
:1001380010B5054C237833B9044B13B10448AFF319
:1001480000800123237010BD4C0100200000000036
:100158003809010808B5034B1BB103490348AFF33D
:10016800008008BD00000000500100203809010887
:1001780014214160704714207047406A704700009E
:10018800790100087F01000883010008990100082F
:1001980010B5044604F1100000F05CFCC4F8F80047
:1001A8000148C4F87C0110BD88010008F8B5E6B024
:1001B80004460D4616461F460A4906A800F0CAFE20
:1001C80070996F9A05910492009733466E996D9ACB
:1001D800039102922A466C990191214600F060F839
:1001E80067B0F0BD94010008F8B5E6B004460D46C6
:1001F80016461F46094906A800F0ACFE6F996E9A8C
:100208000491039200976D996C9A0291019233467A
:100218002A46214600F087F867B0F0BD940100082F
:1002280038B500281CBF01680029184A23D1184B8B
:100238001C684FF6F0710C404CF24025AC421FBFD1
:100248001B6819404CF27024A14212D1114D296843
:1002580079B911490B68C3F30B03B3F58A6F1FBF54
:100268000968C1F30B0140F28343994204BF01219D
:10027800117028B905E0094B994204BF012111709A
:100288004068BDE8324001F099BE00BF6801002017
:1002980000ED00E0002004E00010005C000037489A
:1002A8002DE9F04104460D46216816464A681F4666
:1002B80090478046B8F5403F2ED122680A99936846
:1002C800204698478046B8F5403F25D12368089ACC
:1002D8000799D3F80CC02046E0478046B8F5403F60
:1002E8001AD12368069A39461F692046B8478046BE
:1002F800B8F5403F10D1236829465D69324620464B
:10030800A8478046B8F5403F06D123680B9A09995B
:100318009D692046A847804621680A68204690477C
:100328004046BDE8F0812DE9F04104460D462168BC
:1003380016464A681F4690478046B8F5403F2ED17A
:1003480022680A999368204698478046B8F5403F46
:1003580025D12368089A0799D3F80CC02046E047AE
:100368008046B8F5403F1AD12368069A39461F6976
:100378002046B8478046B8F5403F10D12368294643
:100388005D6932462046A8478046B8F5403F06D109
:1003980023680999DD6900222046A847804621681C
:1003A8000A68204690474046BDE8F0814FF4403047
:1003B80070470000F0B50C4685B0114600281A4673
:1003C8001CBF0568002D0B4B11D082B104B971B95F
:1003D8000D9860B10F9E0E9F0A9B0290049603979A
:1003E8000B980C9E009001962046A8470346184695
:1003F80005B0F0BD020003002DE9F04F0646D0B06D
:100408000868F56DD6F860E0726EB76EF36E00BAE4
:1004180000906C46486800BA60600DF14008886832
:1004280000BAA060C86800BAE060086900BA206134
:10043800486900BA6061886900BAA061C86900BAF1
:10044800E061086A00BA2062486A00BA6062886A95
:1004580000BAA062C86A00BAE062086B00BA2063FA
:10046800486B00BA6063886B00BAA063C86B00BAB7
:10047800E063402058F80C1C58F820CC58F838ACE9
:100488008CEA010158F840CC8AEA01018CEA01099A
:100498004FEAF979401E48F8049BEBD187EA02003D
:1004A80000EA0E00784010EBF5610098DFF824C4EC
:1004B80041186144C81882EABE032B404FEAF06134
:1004C80053405918636859186144CF194FEAB50366
:1004D80083EABE01014081EABE0111EBF765A1681C
:1004E8004D196544A91883EAB0023A404FEAF1650C
:1004F8005A405519E26855194FEAB70282EAB0071F
:1005080065440F4005EBBE0E97EAB00717EBFE6592
:1005180027697D194FEAB10782EA0701654401EAB4
:100528000E01EB18514011EBF36561694D194FEA63
:10053800BE0187EA010E65440EEA030E15EBB00012
:100548008EEA070E0EEBF065D4F818E075446544A2
:10055800AA1881EAB30505404FEAF26E4D40AE4451
:10056800E569AE44E64477444FEAB00080EAB30E4A
:100578000EEA020E8EEAB30E0EEBF765D4F820E011
:1005880075446544691880EAB2053D404FEAF16E4A
:100598004540AE44656AAE44E6440EEBB3034FEA09
:1005A800B70787EAB20E0EEA010E8EEAB20E0EEB1C
:1005B800F365D4F828E075446544281887EAB1053E
:1005C8001D404FEAF06E7D40AE44E56AAE44E64415
:1005D8000EEBB2024FEAB30383EAB10E0EEA000E45
:1005E8008EEAB10E0EEBF265D4F830E0754465443E
:1005F800EF1983EAB00515404FEAF76E5D40AE4447
:10060800656BAE44E6440EEBB1014FEAB20282EAF2
:10061800B00E0EEA070E8EEAB00E0EEBF165D4F8B6
:1006280038E075446544EB1882EAB7050D404FEA97
:10063800F36E5540AE44E56BAE44E6440EEBB000B5
:100648004FEAB10181EAB70E0EEA030E8EEAB70E41
:100658000EEBF065D4F840E07544654481EAB30ECA
:10066800AA180EEA000E4FEAF2658EEA010E7544EA
:10067800DDF844E04FEAB000754480EAB30E654403
:100688000EEA020E15EBB7078EEAB30E0EEBF7650E
:10069800DDF848E04FEAB202754480EA020E65448C
:1006A8000EEA070E69188EEA000E0EEBF165DDF80A
:1006B8004CE07544654405EBB3034FEAB70E1427C5
:1006C8000DF1500CDFF810528EEA010B82EA0B0B89
:1006D8000BEBF36A5CF804BBDA44AA44504483EA9F
:1006E800B10B4FEAF06A8EEA0B0BDA445CF804BBF4
:1006F800DA44AA44524480EAB30B4FEAF26A8BEA1E
:10070800B10BDA445CF804BBDA444FEAB000AA44FF
:1007180080EA020BD6448BEAB30B0BEBFE6A5CF85B
:1007280004BBDA444FEAB202AA4482EA0E0B0AEB8F
:10073800B10180EA0B0B0BEBF16A5CF804BBDA44FD
:100748007F1DAA44282F0AEBB3034FEABE0EBBD382
:100758003C2F61D3502F4DD204EB870CC7F15407BF
:100768005E4CA7FB04A504465D4FA8088EEA010A63
:1007780082EA0A0A5CF804BB0AEBF3655D447D195A
:100788002C1983EAB10A4FEAF4658EEA0A0A55443D
:100798005CF804AB5CF804BB55447D19AA1884EADC
:1007A800B30A4FEAF2658AEAB10A55445D444FEA52
:1007B800B4047D1984EA020AAE448AEAB30A0AEB51
:1007C800FE655CF804AB55444FEAB2027D1982EA33
:1007D8000E0A15EBB10184EA0A0A5CF804BB0AEBBD
:1007E800F1655D447D1915EBB303401E4FEABE0E5B
:1007F800BCD12046F46D1B19F365336EC9183166F8
:10080800716E71447166B36ED218B266F16E40189B
:10081800F06650B0BDE8F08F4EEA010B0EEA010A0F
:100828000BEA020B4BEA0A0A0AEBF36554F827A015
:10083800DFF8B0C0554443EAB10B654403EAB10A96
:100848000BEA0E0B28184BEA0A0A7F1C0AEBF06524
:1008580054F827A0554440EAB30B654400EAB30AAC
:100868000BEAB10BAA184BEA0A0A7F1C0AEBF265DD
:1008780054F827A055444FEAB00040EA020B6544FB
:1008880000EA020A0BEAB30BAE444BEA0A0A7F1CE1
:100898000AEBFE6554F827A055444FEAB20242EA33
:1008A8000E0B654402EA0E0A0BEA000B15EBB101C8
:1008B8004BEA0A0A7F1C0AEBF16554F827A0554455
:1008C8007F1C65443C2F05EBB3034FEABE0EA3D350
:1008D80040E700BF9979825AA1EBD96ECDCCCCCC38
:1008E800D6C162CADCBC1B8F00B581B00168074A5B
:1008F800914200D110B9064801B000BD7C210FF02B
:100908007FFF4FF4003001B000BD00BFFC090008B4
:10091800030002002DE9F0410B4A92E8F85188B033
:10092800694681E8F8510268084B9A4200D118B923
:10093800074808B0BDE8F0811422083000F04FFBEA
:1009480008B0BDE8F08100BFDC090008FC09000818
:1009580003000200152904D20268044B9A4200D110
:1009680008B903487047083000F048BBFC09000884
:100978000300020010B481B013460268074CA2427B
:1009880000D118B901B010BC0548704701B000F19A
:10099800240210BC083000F035BB00BFFC09000879
:1009A8000300020010B481B013460268074CA2424B
:1009B80000D118B901B010BC054870470A4601B00B
:1009C80000F1240110BC083000F070BBFC090008DD
:1009D800030002000123456789ABCDEFFEDCBA981E
:1009E80076543210F0E1D2C300000000000000008D
:1009F80000000000F10800081D0900085D09000852
:100A08007D090008AD09000801040008790F0008F5
:100A1800C50F0008810F0008F0B5A3B004460B48C5
:100A280002900D4616461F46094B0822402104A88D
:100A380000F0D1FA28980190009733462A462146BB
:100A480002A800F01BF823B0F0BD00BFFC090008A5
:100A5800100A000810B5040008BF002408D0054893
:100A6800054B20600822402104F1080000F0B3FA89
:100A7800204610BDFC090008100A00082DE9F041C5
:100A880004460E46216817464A681D469047804628
:100A9800B8F5003F19D1226806999368204698470F
:100AA8008046B8F5003F10D123683146DE683A46E3
:100AB8002046B0478046B8F5003F06D12368079A1C
:100AC80029461D692046A847804621680A682046AD
:100AD80090474046BDE8F08110B500F033FA4FF476
:100AE800403400280EBF034C4FF4C0710FF088FE4D
:100AF800204610BD0200030010B5044600F022FA9B
:100B080008B9054810BD0021A160D0F87C21116802
:100B180088474FF4403010BD0200030070B504460A
:100B28000D4600F00FFA064E40B1D0F87C0141683E
:100B38008847A84224BF65604FF44036304670BDF0
:100B4800020003002DE9FF4715000C4600D02CB128
:100B5800064600F0F7F95FEA000801D16448C3E0EF
:100B6800D8F8F80001684A689047B0F5003F17D1F7
:100B7800D8F87C118A68404690478146B9F1810FC0
:100B880080F09E80A94508F1FC0A17D2D8F8F80031
:100B98000368D3F80CC02A462146E047B0F5003F69
:100BA80040F08E80D8F8F8000368D3F810C06A4681
:100BB8005146E047B0F5003F76D10AE0002004E056
:100BC800215C0AF800100098401C00900098A84288
:100BD800F6D34FF0000C4749474A484B01AC009800
:100BE800844558D2D3E9007001ADC5E9007010788A
:100BF80000281ABF042086464FF0000E085854F803
:100C08000E5028443E4D05600127D0F800E087606B
:100C1800019D4F681AF80C007D408EEA050585F0A5
:100C2800040E65680F687D4085F0FC05754485F005
:100C3800A30568400AF80C000CF1010CCFE7D3E9D2
:100C4800004501A8C0E9004510782E4D002814BFC2
:100C58004FF0040E4FF0000E01A8744651F80EE054
:100C68000459A6440127CEF80050DEF80040CEF81B
:100C780008704D68019F40687D406C400D68684071
:100C880084F0040480F0FC00041984F057040AF886
:100C98000C400CF1010CCC45D1D3D8F8F800016810
:100CA8004A689047B0F5003F0AD1D8F8F8000368C1
:100CB800D3F80C804A465146C047B0F5003F01D0F2
:100CC800114811E0002006E05AF8201081F06A313E
:100CD8004AF82010401CB0EB990FF5D3B06840F0EB
:100CE8000100B0604FF4403004B0BDE8F08700BFA9
:100CF80002000300D009010868010020240F000841
:100D0800ADBE4ED70DBE75A10100030038B50C4627
:100D1800017A1546CA0702D500F014F908B908483F
:100D280032BDD0F8F80003682146DC682A46A0479F
:100D3800B0F5003F01D0034832BD4FF4403032BD1A
:100D480002000300010003002DE9F84191B00546B7
:100D58000E461746402101A80FF052FD297AC80710
:100D680004D5284600F0EEF8040002D1DFF8A4808C
:100D78004BE0D4F8F800DFF8A0800368D3F810C07F
:100D88006A4601A9E047B0F5003F3ED1D4F8F80023
:100D980001684A689047B0F5003F36D1D4F87C1115
:100DA8008A6820469047D4F8F830024618461B68EF
:100DB800D3F80CC004F1FC01E047B0F5003F24D1A2
:100DC800D4F87C0141688847D4F8F83002461846C0
:100DD8001B68D3F80CC001A9E047B0F5003F14D157
:100DE800D4F8F8000268696893689847B0F5003F3E
:100DF8000BD1D4F8F80003681C693A463146A0477D
:100E0800B0F5003F08BF4FF44038404612B0BDE887
:100E1800F08100BF02000300010003002DE9F84142
:100E2800A5B0074688461646402115A80FF0E8FCED
:100E380000220492402105A80FF0E2FC387AC1078D
:100E48005ED5384600F07EF8050059D0D5F8F80090
:100E58002D4C0368D3F810C06A4605A9E047B0F5E1
:100E6800003F3CD1D5F8F80001684A689047B0F5D2
:100E7800003F34D1D5F87C118A6828469047D5F8C8
:100E8800F830024618461B68D3F80CC005F1FC017F
:100E9800E047B0F5003F22D1D5F87C01416888478A
:100EA800D5F8F830024618461B68D3F80CC005A9D7
:100EB800E047B0F5003F12D1D5F8F800026879682C
:100EC80093689847B0F5003F09D1D5F8F800036852
:100ED8001D6904AA15A9A847B0F5003F01D020460E
:100EE8000FE00A4B0A490B4A0396029101924046C9
:100EF8001C68049B009415AA796800F0E5F900E0E5
:100F0800054826B0BDE8F08101000300D8090108B2
:100F1800936E030026C703000200030004B001011A
:100F280000170145E10A0008010B0008250B00081D
:100F3800B50300084D0B0008150D0008510D0008F9
:100F4800250E00080168024A914218BF0020704728
:100F58002C0F000810B5040008BF002404D0034873
:100F68002060204609688847204610BD2C0F0008DD
:100F780020225C300FF042BCF0B58468A308002240
:100F880004F0030407E000F15C0555F8226035BA67
:100F980041F82250521C9A42F5D300220BE000F18E
:100FA8005C0502EB830755F82360D500C5F11805E9
:100FB800EE40CE55521CA242F1D3F0BD30B5C46804
:100FC80003690022E31AD5188C5C0544521C082AD0
:100FD8002C77F8D330BD0360C1600261704738B523
:100FE800044615460022626023685A68904700202C
:100FF8006061A061A5604FF4003032BD81604FF49C
:10100800003070472DE9F84304462079D4F80C8065
:10101800450748BF244845D466691D46A8F1010024
:1010280000EAD60306EBC506B6EBC50F666102D229
:10103800A669761CA6611746A66906EB5576A661D1
:101048000E46E918884225D2A8EB03094A463146DC
:10105800F8180FF0D3FB2268136839460FE04246B0
:1010680038460FF0CBFB23681A683946204690476C
:1010780007E0311811F00300F1D122681368204607
:101088009847484600EB0809A9F10101A942F0D3A5
:10109800002300E000202A1A3118F8180FF0AEFBE0
:1010A8004FF40030BDE8F283040002002DE9FC4F44
:1010B800024685B0D0681369DFF86CC1DFF86C812F
:1010C800A0EB030A506840F004005060002703A812
:1010D80002900DF10C0ED8E9003403A8544DC0E974
:1010E80000342878534D00280CBF00230423994668
:1010F8005CF803305EF80940234401261D601C6833
:101108009E60DCF80430039DDCF80090DEF8046093
:101118005D406540484C654089EA0606474C664094
:101128007519474C6540D8E9006B03AC0028C4E941
:10113800006B0EBF002404200424029E5CF800000B
:10114800345920183F4C04600126046886600398CF
:10115800029E43406340384C7068634089EA00004F
:10116800364C6040034438484340280018BF0120EB
:101178005B1E9B41042F2CBFC0B2D80F02F1140391
:1011880053F8200007F00303C3F10303DB00D84042
:101198000DF807007F1C082F9DD315460C466A6979
:1011A800AB69E868D20842EA4372401E00EA0207C7
:1011B800002302409B420AD8524508D28020E055BD
:1011C8007F1C574516D2AAEB0701E01910E08020D2
:1011D800E05500E0E355E8687F1C8742FAD32A68A7
:1011E800136828469847BAF1000F03D051462046A5
:1011F8000FF006FB2A68069E059F936869462846F5
:1012080098472A68D2F8009021462846C8472B6894
:10121800DA683946284690470EB1A86830604FF41E
:10122800003007B0BDE8F08FD0090108541200085B
:10123800680100205FC5109304850012FC68017ADC
:10124800C0F524FF24AF33D426AF698B04B0010165
:1012580000170145F8B501240094002300240DE08F
:10126800009D065D0F5D7E40F643761CF60F86F006
:10127800010635400095641C009DEB189442EFD39D
:101288001846F2BDF8B5002301240094002A11E0A5
:10129800009C85188F1815F8016C17F8015C6E40D2
:1012A800F643761CF60F86F0010634400094009C45
:1012B800E318521EECD11846F2BD00005D1200087A
:1012C8008D120008010000002DE9F84F1D46DDF8D9
:1012D80028900B9F0D9C4FF0FF3300930E469246CB
:1012E800D9F800B0804632465146D847834664B3A1
:1012F800D9F8043032465146404698476FEA0B0207
:10130800521C42EA0B0200996FEAD2735B1C194027
:10131800C2430091521C024300996FEAD2735B1CCE
:101328001940009186F05531484087EA000181F064
:101338005531216080F05531C943491C0843009A52
:101348006FEAD070401C82430092D9F80800012847
:1013580009D17540E943491C0D4300986FEAD572DD
:10136800521C90430AE0F11C85EA9102D243521CB8
:10137800154300986FEAD5735B1C984386F0AA362C
:10138800009086EA0B0686F0AA33F243DB430C98FA
:10139800C2F3C0725B1C42EAD3720099D243521C5A
:1013A80091430091774000998843009987F0AA37C4
:1013B8000F403843BDE8F28F034613F8012B002A8B
:1013C800FBD1181A0138704781F0004102E000BFD4
:1013D80083F0004330B54FEA41044FEA430594EAED
:1013E800050F08BF90EA020F1FBF54EA000C55EA28
:1013F800020C7FEA645C7FEA655C00F0E2804FEAF9
:101408005454D4EB5555B8BF6D420CDD2C4480EADA
:10141800020281EA030382EA000083EA010180EA0A
:10142800020281EA0303362D88BF30BD11F0004F58
:101438004FEA01314FF4801C4CEA113102D040428E
:1014480061EB410113F0004F4FEA03334CEA1333C9
:1014580002D0524263EB430394EA050F00F0A780E1
:10146800A4F10104D5F1200E0DDB02FA0EFC22FADC
:1014780005F2801841F1000103FA0EF2801843FAD0
:1014880005F359410EE0A5F120050EF1200E012AC1
:1014980003FA0EFC28BF4CF0020C43FA05F3C018FF
:1014A80051EBE37101F0004507D54FF0000EDCF178
:1014B800000C7EEB00006EEB0101B1F5801F1BD321
:1014C800B1F5001F0CD349085FEA30004FEA3C0C25
:1014D80004F101044FEA445212F5800F80F09A801B
:1014E800BCF1004F08BF5FEA500C50F1000041EB1F
:1014F800045141EA050130BD5FEA4C0C404141EB23
:101508000101013C28BFB1F5801FE9D291F0000F1D
:1015180004BF01460020B1FA81F308BF2033A3F1CC
:101528000B03B3F120020CDA0C3208DD02F1140CC3
:10153800C2F10C0201FA0CF021FA02F10CE002F1FE
:101548001402D8BFC2F1200C01FA02F120FA0CFCF7
:10155800DCBF41EA0C019040E41AA2BF01EB045140
:10156800294330BD6FEA04041F3C1CDA0C340EDC3E
:1015780004F11404C4F1200220FA04F001FA02F381
:1015880040EA030021FA04F345EA030130BDC4F13F
:101598000C04C4F1200220FA02F001FA04F340EA34
:1015A8000300294630BD21FA04F0294630BD94F0E5
:1015B800000F83F4801306BF81F480110134013DCC
:1015C8004EE77FEA645C18BF7FEA655C29D094EA3D
:1015D800050F08BF90EA020F05D054EA000C04BFBB
:1015E8001946104630BD91EA030F1EBF00210020A6
:1015F80030BD5FEA545C05D14000494128BF41F045
:10160800004130BD14F580043CBF01F5801130BDA8
:1016180001F0004545F0FE4141F470014FF0000033
:1016280030BD7FEA645C1ABF194610467FEA655CE4
:101638001CBF0B46024650EA013406BF52EA033586
:1016480091EA030F41F4002130BD00BF90F0000F74
:1016580004BF0021704730B54FF4806404F13204B0
:101668004FF000054FF0000150E700BF90F0000F69
:1016780004BF0021704730B54FF4806404F1320490
:1016880010F0004548BF40424FF000013EE700BF60
:1016980042004FEAE2014FEA31014FEA02701FBFF0
:1016A80012F07F4393F07F4F81F06051704732F022
:1016B8007F4208BF704793F07F4F04BF41F4002179
:1016C800704730B54FF4607401F0004521F00041D7
:1016D8001CE700BF50EA010208BF704730B54FF061
:1016E80000050AE050EA010208BF704730B511F062
:1016F800004502D5404261EB41014FF4806404F19A
:1017080032045FEA915C3FF4D8AE4FF003025FEA1F
:10171800DC0C18BF03325FEADC0C18BF033202EBA3
:10172800DC02C2F1200300FA03FC20FA02F001FAFD
:1017380003FE40EA0E0021FA02F11444BDE600BFA0
:101748004FF0FF3C06E000BF4FF0010C02E000BF85
:101758004FF0010C4DF804CD4FEA410C7FEA6C5C68
:101768004FEA430C18BF7FEA6C5C1BD001B050EA0B
:10177800410C0CBF52EA430C91EA030F02BF90EAF6
:10178800020F0020704710F1000F91EA030F58BFB5
:10179800994208BF90422CBFD8176FEAE37040F017
:1017A800010070474FEA410C7FEA6C5C02D150EAB5
:1017B800013C07D14FEA430C7FEA6C5CD6D152EA70
:1017C800033CD3D05DF8040B704700BF8446104635
:1017D80062468C461946634600E000BF01B5FFF734
:1017E800B7FF002848BF10F1000F01BD4DF808ED04
:1017F800FFF7F4FF0CBF012000205DF808FB00BFD5
:101808004DF808EDFFF7EAFF34BF012000205DF82E
:1018180008FB00BF4DF808EDFFF7E0FF94BF01207B
:1018280000205DF808FB00BF4DF808EDFFF7CEFF7C
:1018380094BF012000205DF808FB00BF4DF808EDBB
:10184800FFF7C4FF34BF012000205DF808FB00BF8C
:101858004FEA410212F5001215D211D56FF47873D0
:10186800B3EB625212D94FEAC12343F0004343EA73
:10187800505311F0004F23FA02F018BF404270474E
:101888004FF00000704750EA013005D111F00040D8
:1018980008BF6FF0004070474FF00000704700BF6E
:1018A80080F0004002E000BF81F0004142001FBF0D
:1018B8005FEA410392EA030F7FEA226C7FEA236C16
:1018C8006AD04FEA1262D2EB1363C1BFD21841400B
:1018D80048404140B8BF5B42192B88BF704710F0A1
:1018E800004F40F4000020F07F4018BF404211F044
:1018F800004F41F4000121F07F4118BF494292EAAC
:10190800030F3FD0A2F1010241FA03FC10EB0C00D7
:10191800C3F1200301FA03F100F0004302D5494264
:1019280060EB4000B0F5000F13D3B0F1807F06D311
:1019380040084FEA310102F10102FE2A51D2B1F109
:10194800004F40EBC25008BF20F0010040EA0300FE
:101958007047490040EB0000013A28BFB0F5000F7E
:10196800EDD2B0FA80FCACF1080CB2EB0C0200FA34
:101978000CF0AABF00EBC25052421843BCBFD04083
:101988001843704792F0000F81F4000106BF80F4FD
:1019980000000132013BB5E74FEA41037FEA226CC0
:1019A80018BF7FEA236C21D092EA030F04D092F08B
:1019B800000F08BF0846704790EA010F1CBF0020BF
:1019C800704712F07F4F04D1400028BF40F000401C
:1019D800704712F100723CBF00F50000704700F03C
:1019E800004343F0FE4040F4000070477FEA226263
:1019F80016BF08467FEA23630146420206BF5FEA34
:101A0800412390EA010F40F4800070474FF0000333
:101A180004E000BF10F0004348BF40425FEA000CFA
:101A280008BF704743F0964301464FF000001CE0A2
:101A380050EA010208BF70474FF000030AE000BFF8
:101A480050EA010208BF704711F0004302D5404236
:101A580061EB41015FEA010C02BF844601460020A8
:101A680043F0B64308BFA3F18053A3F50003BCFAC3
:101A78008CF2083AA3EBC25310DB01FA02FC634470
:101A880000FA02FCC2F12002BCF1004F20FA02F277
:101A980043EB020008BF20F00100704702F120026A
:101AA80001FA02FCC2F1200250EA4C0021FA02F2CB
:101AB80043EB020008BF20EADC7070474FEA40029F
:101AC800B2F1FE4F0FD34FF09E03B3EB12620DD964
:101AD8004FEA002343F0004310F0004F23FA02F0CE
:101AE80018BF404270474FF00000704712F1610F75
:101AF80001D1420205D110F0004008BF6FF000404C
:101B080070474FF00000704753B94AB9002908BF21
:101B180000281CBF4FF0FF314FF0FF3000F06AB9CA
:101B2800ADF1080C6DE904CE00F006F8DDF804E02C
:101B3800DDE9022304B070472DE9F047089D0C4603
:101B4800002B4ED194468C458646B2FA82F262D971
:101B58004AB1C2F12003914020FA03F30CFA02FCC7
:101B6800194300FA02FE4FEA1C471FFA8CF6B1FB34
:101B7800F7F44FEA1E4307FB141143EA014304FB41
:101B880006F199420AD91CEB030304F1FF3080F0F7
:101B98001281994240F20F81023C6344591A1FFA9C
:101BA8008EF3B1FBF7F007FB101143EA014300FB8A
:101BB80006F69E420AD91CEB030300F1FF3180F0C0
:101BC800FC809E4240F2F980634402389B1B40EA45
:101BD800044000211DB1D3400022C5E90032BDE810
:101BE800F0878B4205D90DB1C5E9000100210846EF
:101BF800F5E7B3FA83F1002946D1A34202D3904214
:101C0800C0F0F080861A64EB03030120002DE6D0B3
:101C1800C5E90063E3E7002A40F09080A1EB0C04DB
:101C28004FEA1C481FFA8CF70121B4FBF8F64FEA7B
:101C38001E4308FB164443EA044307FB06F0984298
:101C480008D91CEB030306F1FF3402D2984200F2D4
:101C5800CD8026461C1A1FFA8EF3B4FBF8F008FB59
:101C6800104443EA044300FB07F79F4208D91CEBE2
:101C7800030300F1FF3402D29F4200F2B0802046F5
:101C8800DB1B40EA0640A5E7C1F120068B4022FA9B
:101C980006F71F4320FA06FC04FA01F343EA0C0393
:101CA800F44000FA01F8380C4FEA1349B4FBF0FE8F
:101CB8001FFA87FC00FB1E4449EA04440EFB0CF99A
:101CC800A14502FA01F20AD93C190EF1FF3A80F057
:101CD8008480A14540F28180AEF1020E3C44A4EB21
:101CE80009041FFA83F9B4FBF0F300FB134449EA33
:101CF800044403FB0CFCA44507D93C1903F1FF304D
:101D080067D2A44565D9023B3C4443EA0E40A0FB98
:101D18000293A4EB0C049C42CE469C4651D34ED071
:101D280055B1B8EB0E0364EB0C0404FA06F6CB408D
:101D38001E43CC40C5E90064002150E7C2F12003EE
:101D480020FA03F10CFA02FC24FA03F394400C4342
:101D58004FEA1C4800FA02FE1FFA8CF7B3FBF8F0B2
:101D680008FB1031230C43EA014300FB07F19942B9
:101D780008D91CEB030300F1FF362CD299422AD96B
:101D8800023863445B1AA4B2B3FBF8F108FB1133C1
:101D980044EA034401FB07F3A34208D91CEB0404FB
:101DA80001F1FF3613D2A34211D902396444E41A6F
:101DB80041EA004139E70446F0E6084606E7C84527
:101DC800AED2B9EB020E63EB070C0138A8E7314637
:101DD800EDE7034699E73046D4E7D6467FE7634404
:101DE80002384DE70646234608460FE7023E63449D
:101DF80030E700BF704700BF1348144A08B54FF0DA
:101E08000043C0E900230422426101220023C26189
:101E18004FF480510722C0E90233C0E90933C0E911
:101E28000C1203610383837680F8203080F82C300D
:101E3800826380F83C30C36401F0C0FF18B1BDE88C
:101E4800084000F00DBB08BD6C01002000240140D3
:101E58000268084B9A4282B00AD14FF0B0431A6E1A
:101E680042F400721A661B6E03F400730193019B1F
:101E780002B07047002401400268054B9A4201BF36
:101E88004FF0B042136E23F400731366704700BF1F
:101E98000024014030B585B000240546CDE9014451
:101EA8000394FFF7A9FF144802F01CFB08B100F0E7
:101EB800D7FA1148039401A9CDE9015402F0DCF8DE
:101EC80008B100F0CDFA0C4802F036FA08B100F07B
:101ED800C7FA4FF0FF31084802F070F8064802F0E0
:101EE800E3FA054802F0C4F80446034802F086FA0B
:101EF800204605B030BD00BF6C010020014B024AEE
:101F08001A6070476C0100200024014008B5094898
:101F1800FFF7C0FF68B1084BB3F8AA304FF6FF725D
:101F2800934216BF40F6E442044B5343B3FBF0F32D
:101F380098B208BD002000B40075FF1FD8084C00F7
:101F480013B50023ADF80630FFF7E0FF0446194843
:101F5800FFF7A0FF184BB3F8C820B3F8A8108A42BF
:101F680004FB00F018D040F6E443B0FBF3F3642020
:101F78005B1A4343521A93FBF2F31E331BB2ADF8BC
:101F88000630BDF806305BB21B02ADF80630BDF86E
:101F9800060000B202B010BD4FF47A7240F6FF732B
:101FA800B0FBF3F35343A3F53923A3F50C6340F6D1
:101FB800C412E0E7001000B00075FF1F4FF0B043F7
:101FC80082B09A6A22F480529A629A6C42F48052E1
:101FD8009A649B6C03F480530193019B002002B028
:101FE80070474FF0B04307B59A6C42F004029A6408
:101FF8009A6C02F004020192019A9A6C42F0010272
:102008009A649B6C002203F001030093114611208F
:10201800009B02F005FB112003B05DF804EB02F011
:1020280031BB000008B502F071FD10B16FF004007B
:1020380008BD064B9A6942F040429A614CF2FA3266
:102048001A6102F075FD0028F2D0EFE70040005851
:10205800F0B585B000230D4600930646A8B3FFF7F8
:10206800E1FF044670BB02F051FD88BB1A481B4AC9
:1020780002230193D0F8E01506F1784302EA8121A2
:10208800B3FBF1F701FB1733DB0A0293D0F8E00545
:1020980005F178410139314402EA8022B1FBF2F0BE
:1020A80002FB1011C3EBD1230133694601A8039346
:1020B80002F0BEFD20B1022814BF6FF00104012414
:1020C80002F036FD204605B0F0BD6FF00504F9E7D3
:1020D8006FF00404F6E700BF0070FF1F00FCFF0369
:1020E800014B186000207047D00100202DE9F04F07
:1020F800B0F1006F89B006460F469046C0F0C08028
:10210800DFF89091644DD9F8E03505EA832303F1AF
:102118000063013B984200F2B380002900F0B380CD
:1021280040EA02035B0740F0AE80FFF77BFF0446FE
:1021380090BB02F0EBFC002840F0A880D9F8E0152D
:10214800009705EA812106F17842B2FBF1F301FB21
:10215800132208F17843013B3344B3FBF1F001FB50
:102168001033DB0A01334FEAD22AA3EBD222012A29
:10217800039388BFC6F30A050AF58037C6F108033A
:102188008CBFC5F500654546FF02B3460693039B21
:102198009A4505D302F0CCFC204609B0BDE8F08F83
:1021A800A6F10803069A1A4495421CD8009B049588
:1021B8000193CDF814B04FF00009059B09EB03011A
:1021C800049B99453DD3009BAB442B44A8EB0505E4
:1021D800B5F5006F009328BF4FF400650AF1010AB6
:1021E80007F50067D3E753F8081F5A68B2F1FF3FB5
:1021F80008BFB1F1FF3FD5D0284B186810B96FF070
:102208000504C7E727B14FF4006239460DF08EFE8A
:10221800DFF888900099D9F80030CBF30A00184409
:10222800AAB20DF083FE4FF400613846FFF710FFA5
:1022380000BBD9F8003001934FF40063059704936D
:10224800B9E7019B07914B4402930120D3E900238E
:1022580002F0A8FC88B90799019BD1E9000259F856
:102268000310029B5B689A4208BF884205D109F1B6
:102278000809A2E76FF001048CE76FF0030489E70F
:102288004FF0FF3488E76FF0050485E76FF004042A
:1022980082E700BF0070FF1F00FCFF03D001002091
:1022A800B1F1006F70B510D30B4BD3F8E0650B4B51
:1022B80003EA862303F10063013B994205D838B14C
:1022C80092B20DF033FE002070BD4FF0FF30FBE7F7
:1022D8006FF00500F8E700BF0070FF1F00FCFF0368
:1022E800B0F1006F10B40DD3084BD3F8E045084B9C
:1022F80003EA842303F10063013B984202D810BC2F
:10230800FFF7A6BE4FF0FF3010BC70470070FF1FEC
:1023180000FCFF034FF0B04382B0DA6C0243DA648A
:10232800DB6C03400193019B02B0704710B586B087
:102338001422002101A80EF035FA0120FFF7EAFF68
:102348000220FFF7E7FF0420FFF7E4FF10211648FB
:10235800002202F0E1FD012402224FF4041301A936
:102368004FF09040CDE90123039402F0AFFC4FF405
:10237800441301A94FF09040CDE90234019402F0D2
:10238800A5FC00221146062002F04AF9062002F0B8
:1023980079F900221146072002F042F9072002F0DD
:1023A80071F906B010BD00BF0004004800B59BB02D
:1023B8004822002108A80EF0F5F91822002102A8E9
:1023C8000EF0F0F902F0BAFD4FF0B0420120D2F859
:1023D800903023F01803C2F89030D2F8003423F478
:1023E800C06343F40073C2F80034D2F8003403F435
:1023F800C0630193019B2423089381230B9300233B
:10240800CDE91003B02208A8CDE9122302F00EFF8F
:1024180008B172B6FEE74F23CDE90230CDE90400DA
:10242800CDE90600022102A803F09AF908B172B6B4
:10243800FEE71BB05DF804FB08B501F085FCFFF76B
:10244800B5FFFFF773FF05480022102102F064FD75
:1024580000F032FD00F037FDFCE700BF0004004843
:1024680072B6FEE700B58DB02C22002101A80EF04F
:1024780099F91748174B03601F2383604FF0804278
:102488000023C0E90433C0E9072383614FF4807354
:10249800436203F00BFC08B1FFF7E2FF0C4803F0BE
:1024A80031FD08B1FFF7DCFF4FF00053002207931E
:1024B800074808924FF4807301A9029206920B9381
:1024C80003F054FC08B1FFF7CBFF0DB05DF804FB37
:1024D800D40100200028004010B5044690B03822EE
:1024E800002102A80EF05EF92268194B9A422CD1FD
:1024F8004FF48033029302A84FF480730F9303F0D4
:1025080053FA08B1FFF7ACFF4FF0B0430220D3F8FD
:10251800902042F40042C3F890209A6D42F4806201
:102528009A659B6D002203F4806311460193019B19
:1025380002F076F8022002F0A5F800222A201146BF
:1025480002F06EF82A2002F09DF810B010BD00BF0E
:10255800002800407047000008B500224FF6FF71C0
:102568004FF0904002F0D8FC074800224FF6FF7168
:1025780002F0D2FC01F0FEFB044B0120C3F88800F6
:10258800BDE8084002F032BD0004004800040058CD
:1025980001F0F7BB08B501F0F4FB00F0D7FBFFF73B
:1025A800C5FEBDE80840FFF71CBD08B501F0E2FB19
:1025B800BDE808400121002002F0C8BC7047704700
:1025C800FEE7FEE7FEE7FEE7FEE770477047704765
:1025D80070470000014803F0BBBC00BFD4010020D5
:1025E800012002F09FBC022002F09CBC704770479B
:1025F8007047704770470000014802F019BA00BFE1
:1026080050020020704770474FF4806002F08ABC87
:10261800014804F05FB800BFB0020020014803F091
:10262800CBBA00BFD4010020014803F0BABE00BFF6
:10263800380200202DE9F04389B080460020109E22
:102648000790894615461F46FDF7EAFDF0B9104C7C
:10265800CDE90090CDE9020407AB0E480593142399
:1026680004933A46434629460068FDF7A3FE2346ED
:10267800324604F1140153F8044B42F8044B8B42E0
:10268800F9D1079B337509B0BDE8F0830120FAE75B
:1026980022020020CC0901081FB50E4C00233C2261
:1026A80002A8CDE902336275237500F0B7F8042358
:1026B80003AA009412210848FFF7BCFF0749142217
:1026C80020460EF05FF8B0FA80F35B09637504B03A
:1026D80010BD00BF0C020020F409010861050020AC
:1026E800054808B50823036003F078FC18B1BDE875
:1026F8000840FFF7B5BE08BD380200204FF0B043D0
:1027080007B55A6E42F001025A665B6E002203F06A
:102718000103019311463220019B01F081FF322011
:1027280003B05DF804EB01F0ADBF00000CB407B5D1
:10273800054A05AB102101930DF002FF03B05DF8C7
:1027480004EB02B0704700BF060A010830B585B037
:10275800044602A80D460DF01FFDBDF90C30064ACF
:1027680000931021029B2046FFF7E0FF2046FEF76A
:1027780023FE288005B030BD060A01084FF0B0429C
:1027880010B5936823F4004393600DF08DFD0D4B55
:1027980001241C700DF05AFA0B480DF071FA0B4B1E
:1027A8004FF400421A6100200DF070FAFFF7A6FB03
:1027B80000F0B4F80DF064FB21462046BDE8104057
:1027C8000DF07EBB44020020552700080040005849
:1027D8000DF08CBB08B5FFF799FB40F6B83398426B
:1027E8000CD8B0F5E16F0BD3FE23A0F5E160584398
:1027F8004FF49663B0FBF3F0C0B208BDFE20FCE7CF
:102808000020FAE77FB5684600F06CF80198FFF7FA
:1028180055F900B207B05DF804FB0000194A38B555
:10282800D2F88035591C044619D101F0B1FA054691
:1028380001F0BAFA054401F0B1FA2B0EE3712B0C42
:10284800A3712B0A6371030EE370C0F30742C0F350
:1028580007232571C0B2A2706370207038BD190AB1
:10286800C3718171190C1B0E41710371D2F8843543
:10287800C370D2F88405C0F30722C0F30743000EE3
:10288800E9E700BF0070FF1F38B5094BD3F8803562
:1028980003600133054609D101F07AFA044601F0D4
:1028A8007DFA444001F080FA44402C6038BD00BFF6
:1028B8000070FF1F012102200DF0ECBA0021022058
:1028C8000DF0E8BA00207047024B187808B100F004
:1028D8005DB870474402002082B00190019802B0B0
:1028E80000F0F0B810B50446FFF72AFB074BA360C9
:1028F80040F30F20FFF78EF8054B064A2360064B7E
:102908006060C4E90323002010BD00BF00004842F6
:1029180000007A440D093E00AB0305000020704713
:10292800014B1868704700BF480200200320704719
:1029380008B501464FF47A7200238002890DFFF72B
:10294800E3F808BD4FF47A73A0FB0303800A40EA5A
:1029580083507047034B98689A689042FBD1C043F4
:10296800704700BF0028004008B5FFF7F3FF014B90
:10297800186008BD4802002008B5FFF7EBFF024BBE
:102988001B68C01A08BD00BF48020020024B187817
:1029980008B1FFF7DFBF70474C02002010B5074BA6
:1029A800074C0122DA654FF48071204603F0CAF81B
:1029B8004FF0FF332363002010BD00BF0028004004
:1029C800D401002002460021014803F0D2BA00BF1A
:1029D800D401002002460121014803F0CABA00BF11
:1029E800D401002010B58CB02C220021044601A887
:1029F8000DF0D8FEFFF7D2FF0C4B0D481B681C44A6
:102A08000023089306934FF00053E44307930122F1
:102A18004FF4807301A902940B9303F0A7F908B14E
:102A2800FFF71EFD00200CB010BD00BF48020020BB
:102A3800D401002038B50546FFF78CFF0221044673
:102A4800074803F09DFAC4F309024FF47A71A2FB18
:102A58000121920AA30A2A8043EA805038BD00BFA8
:102A6800D40100200148002103F08ABAD4010020D3
:102A78000148012103F084BAD4010020F8B50F4DB4
:102A88002E78CEB90E4C4FF0FF372763FFF7EAFCDC
:102A9800FFF784FF4FF48071204603F053F8204677
:102AA800276303F011FA32462046022103F061FA47
:102AB800FFF75AFF01232B700020F8BD4C020020BD
:102AC800D4010020014610B54FF47A720023800229
:102AD800890DFFF719F80146FFF73CFF0446FFF799
:102AE80039FF031B8B4200D310BD00BFF7E70DF081
:102AF800E3BC000010B5064C0221204603F040FA62
:102B08000221421C2046BDE8104003F032BA00BF43
:102B1800D40100201648174A08B54FF4E133C0E93C
:102B2800002300230C22C0E90233C0E90523C0E9D1
:102B38000733C0E90933036104F0B1FB08B1FFF7BB
:102B48008FFC0B48002104F022FD08B1FFF788FC38
:102B58000748002104F03BFD08B1FFF781FC044859
:102B680004F0F5FC18B1BDE80840FFF779BC08BDD2
:102B7800B00200200044004070B596B0064614220A
:102B8800002103A80DF00EFE3822002108A80DF040
:102B980009FE32682C4B9A4253D10223089308A8A5
:102BA8002A4B0A9302F000FF08B1FFF759FC4FF0D7
:102BB800B04300259A6D42F400329A659A6D02F48A
:102BC80000320292029ADA6C42F00102DA64DB6C9B
:102BD80003F0010301930422019B0223CDE903239F
:102BE8000324072303A94FF09040CDE90554079328
:102BF80002F06CF8082303A94FF09040CDE90334A4
:102C08000595134C02F062F8124925621423C4E9B1
:102C180000131023C4E9023520468023C4E9043593
:102C2800C4E9065501F08EFD08B1FFF719FC25200F
:102C3800F46700220221A66201F0F2FC252001F0CF
:102C480021FD16B070BD00BF0044004004000C0018
:102C5800500200208000024002680C4B9A4210B5D6
:102C6800044612D14FF0B0420C21936D23F4003387
:102C780093654FF0904002F0D5F8E06F01F0D4FD75
:102C8800BDE81040252001F00BBD10BD00440040F8
:102C980008B50A460146024803F080FC002008BD3A
:102CA800B002002013B5114B114C18604FF40013FB
:102CB800009302AB13E90600204604F0ECFB2368FE
:102CC800DA69D103FCD4DA695202FCD59A6808485B
:102CD80042F480029A6004F024FC06490448012268
:102CE80004F092FB002002B010BD00BF4403002096
:102CF800B00200204C03002008B5074B1860FFF70E
:102D080070F9FFF707FF054AD2F8803043F00063F7
:102D1800C2F88030002008BD480300200008005891
:102D280008B54FF0B04308489A6B42F400329A63F2
:102D38009A6B22F400329A63FFF78EFF0F2001F09E
:102D4800AFFC002008BD00BFB002002008B507484E
:102D580004F0A5FA08B1FFF783FB054801F0F2FC7F
:102D680018B1BDE80840FFF77BBB08BDB0020020E2
:102D7800500200200268044B9A4203D1034B002002
:102D88001B681847704700BF0044004048030020F4
:102D980002680B4B9A4210B504460FD1094B1B68C9
:102DA8002BB1D0F8902012B9074801219847204646
:102DB8000549BDE81040012204F026BB10BD00BF44
:102DC80000440040440300204C03002010B50A4C86
:102DD80023780BB9E37C6BB1FFF75EFC0038074B37
:102DE80018BF0120400018701B78022B02BF002377
:102DF8002370E37410BD00BF610500205403002058
:102E080038B5114C2378EBB9E37CDBB90F4D2B684F
:102E1800012B07D92B68042B04D80D4A0421012063
:102E280000F0D6F92B68042B0CD9FFF735FC0038D5
:102E3800084B18BF0120400018701B78022B04BFF4
:102E48000023237038BD00BF610500205003002017
:102E5800600A01085403002070477047022808B52B
:102E68000ED801221021074802F056F83220FFF749
:102E780033FDBDE8084003480022102102F04CB899
:102E880008BD00BF000400487047000010B50121CC
:102E980004464FF0904002F039F8054AB0FA80F342
:102EA8005B0913701378A370024B01221A7010BDCE
:102EB8004D0300205F05002008B5FFF75FFCBDE863
:102EC800084000F011BB4FF0FF300DF073B87047A9
:102ED80070470000014BD870704700BF0C000020FD
:102EE800014B1874704700BF0C000020002101201E
:102EF8000DF028B810B5044640B190F906302BB94A
:102F080007480DF039FA074BE2791A70064B01228F
:102F18001A70BDE81040002102200DF013B800BF60
:102F2800700300205E0500205D05002010B542F208
:102F38001073084C002818BF0346074823600DF09B
:102F48001BFA216804480DF09FFABDE810400248BA
:102F58000DF060BA08000020C404002010B5094C28
:102F6800206023680BB9084B236008480DF004FA69
:102F7800216806480DF088FABDE8104003480DF0B6
:102F880049BA00BFB4000020A08601005803002001
:102F98000A460149FFF784B900F0030838B50C4820
:102FA8000DF0EAF904F074FF60B90A4C0A480125EB
:102FB800257004F001FE2078294604F055FB0448EA
:102FC8000DF028FABDE8384004480DF023BA00BFD8
:102FD800C4040020700000200C000020AC04002075
:102FE80004F0F4BF30B585B0FFF7F4FB044604F0F5
:102FF80035FC0546002841D101A8FFF747FF2B4AB9
:103008002B490423137053680878187053685D704F
:1030180053681821997053680121D970516823B2F7
:1030280003EB430303EB4313FE24B3FBF4F30B71ED
:10303800204B197821B31D70536860F07F00187019
:103048000523137005231C491C4C0978012988BFE6
:1030580000235370637A33B104F0ECFB012802D1EA
:1030680020460DF089F9164B1048D978002204F053
:103078000BFCA8B9134B1870134B187005B030BD72
:10308800114B1B781BB90F4B1B78002BDAD05368F8
:103098000121597153689DF8061099710723D2E7E9
:1030A8000630EBD104F0C0FBE8E700BF00000020C9
:1030B800B80300205D0500205403002070030020A1
:1030C8000C0000205F050020DC04002020B10378FC
:1030D80013B102480DF09EB9704700BFA00300204D
:1030E80008B5104B0122002102201A700CF02AFFAB
:1030F8000D480DF08FF90D4B1B788BB10C4B1A78DE
:1031080072B9DB7C63B90B4B1A68042A9EBF1A6834
:1031180001321A600021BDE8084010200CF012BFEF
:1031280008BD00BF5D050020580300205E05002093
:103138006105002050030020044B1B78022B03D1AB
:10314800002108200CF0FEBE704700BF7000002070
:1031580008B504F0A6FE80B904F06CFB01280CD178
:10316800BFF34F8F0549064BCA6802F4E062134368
:10317800CB60BFF34F8F00BFFDE708BD00ED00E057
:103188000400FA0538B504460D4607484FF40061B7
:10319800FFF7A6F830B92A4621460348BDE838406B
:1031A800FEF7A4BF38BD00BF00F0030870477047A2
:1031B800704770477047012802D0022804D0704732
:1031C800002102200CF0BEBE00210820FAE7000012
:1031D80070B505460C46164604F040FB034620B37E
:1031E80070BD4A68F05CD0540133DAB2A242F8D319
:1031F8000F4B0D701B78012B88BF00244C700D4CB1
:10320800637A33B104F016FB012802D120460DF091
:10321800B3F8094B0948D978002204F035FB063089
:10322800DED1BDE8704004F0FFBA0449DDE700BF15
:1032380054030020700300200C0000200000002030
:10324800044B1B7823B9044A05210120FFF7C0BFAE
:10325800704700BF54030020650A010810B5002418
:1032680090B03C22214601A800940DF09BFA2C4B0B
:103278002022DA7219788DF8001059788DF801102B
:1032880099788DF80210D9788DF8031019798DF88E
:10329800041059798DF8051099798DF80610D979A7
:1032A8008DF80710197A8DF80810597A8DF80910D9
:1032B800997A8DF80A108DF80B2021460DF10B0232
:1032C80058180131007B02F8010F1C29F8D193F836
:1032D80028208DF8282093F829208DF8292093F8A4
:1032E8002A208DF82A2093F82B208DF82B200DF119
:1032F8002B0100229818013290F82C0001F8010FD8
:10330800142AF7D107484FF40061FEF7E9FF20B906
:10331800044840226946FEF7E9FE10B010BD00BF20
:103328007100002000F80308014940220CF0FEBD9E
:1033380000F8030870B52A4D28796B794D2BC0B277
:1033480033D1C0EB001080000A2838BF0A204FF4A0
:103358007A735843234BAC791860EB794D2BE4B260
:103368002BD1C4EB0414A40095F82C301E4E63BB7B
:1033780095F83F304BBB42F21070FFF7D7FD30682D
:10338800FFF7ECFD2B7A194A1949DBB213706B7AF7
:10339800184ADBB213700023EA1892F82C20D2B234
:1033A800CA540133142BF7D170BD6B79482B0ABF6F
:1033B8004FF461636B795843C6E7EB79482B0ABF32
:1033C8004FF46163EB795C43CEE7FFF7AFFD012C67
:1033D80038BF01244FF47A735C433460CFE700BFF1
:1033E8007100002008000020B400002060050020C3
:1033F800610500205403002010B590B000213C2244
:1034080001A800910DF0CEF94022344968460CF02D
:103418008DFD9DF800203AB99DF80100182803D1C8
:103428009DF8021001290ED0FFF718FF2C4814222E
:1034380000210CF085FD4FF47A70FFF74DFAFFF785
:1034480079FF10B010BD274B1A70587099709DF80D
:103458000310D9709DF8041019719DF80510597161
:103468009DF8061099719DF80710D9719DF80810FC
:1034780019729DF8091059729DF80A1099729DF8F1
:103488000B1001F03F01D972D87AD1B288421BD80B
:103498009DF8282083F828209DF8292083F82920E2
:1034A8009DF82A2083F82A209DF82B2083F82B20CA
:1034B8000DF12B0100229818013211F8014F80F804
:1034C8002C40142AF7D1BAE701F1400068441944A6
:1034D80010F8340C08730132D6E700BF00F803086F
:1034E80061050020710000201FB5002403A92046B3
:1034F800039404F0BBFC03A9012004F0B7FC2F4B94
:103508002F48009422464FF4FA710CF0D7FE2D4B49
:103518002D48009422464FF4FA710CF0CFFE2B4B45
:103528002B48009401224FF4FA710CF0C7FE204694
:10353800FEF7D6FD08B1FEF793FF264B0094002254
:103548004FF4FA6124480CF0B9FE244A0021012006
:103558000CF0B4FD224A002102200CF0AFFD214AF4
:10356800002104200CF0AAFD1F4A002108200CF0BD
:10357800A5FD00F043FB1D491D4804F02DFC1D4826
:1035880004F01AFB12480CF045FF1B4B0021187879
:1035980004F06AF8FFF730FF184A002110200CF0F9
:1035A8008DFD174B17481968174B009400220CF033
:1035B80085FE14480CF02EFF04B010BDB931000888
:1035C800A0030020BB31000888030020B5310008A3
:1035D8007003002041310008AC040020C5790008C0
:1035E800ED2F0008E92F0008A52F000800000301AF
:1035F800240000200C00002070000020092E000884
:10360800B400002058030020E930000830B5A1B00C
:1036180000217C2201A800910DF0C4F853238DF8F5
:10362800003001244FF48C73ADF802308DF804405B
:10363800FFF7D0F8FE23B0FBF3F058231D468DF8B2
:10364800063000EB40000D4B00EB40108DF80500F4
:103658002922802118460DF0A5F80346BDF804106C
:1036680023F8031CC21F009843F8070C07212046C3
:103678009571FFF7ADFD21B030BD00BFE404002017
:1036880070B50378592B90B0044640F0D2810529D3
:1036980059D84378443B162B55D8DFE813F01E0160
:1036A80054000E01540016015400540054005400F4
:1036B80075005400F9005400540054008901540066
:1036C8005400910054005400540017008578482D88
:1036D80011D1AD4A14210120FFF77AFD41F288305B
:1036E800FFF7FAF840F6B830FFF7F6F810B0BDE883
:1036F8007040FFF72DBD532D0ED130228021A348F5
:103708000DF050F8FFF782FF41F28830FFF7E4F838
:103718009E4A1521012067E0432D16D100246846F2
:103728008DF8004004F0C0F9984A4C231370182310
:1037380093709DF80030547001204133D07013719C
:103748000521FFF745FD10B070BD442DFBD1904B0E
:103758002B22802118460DF025F8441F002300F87D
:10376800055C637001251823A370E5702571FFF7C8
:1037780031F8FE23B0FBF3F000EB400000EB401003
:10378800607122460621C5E78378303BDBB2092BFE
:10379800D9D88049804A0B700B78DBB253727B4AC8
:1037A800592313704D2353700B78012030330321B4
:1037B8009370FFF70DFD10B0BDE87040FFF74EBDE8
:1037C8008578482D15D1714A5623137000235370FC
:1037D80018239370537105230321012093711E232D
:1037E8001171D070D371082110B0BDE87040FFF797
:1037F800EFBC432DA7D100213C2201A800910CF079
:10380800D1FF6846FFF790FD644B232280211846BC
:103818000CF0C8FF9DF8002000F80C2C9DF8012042
:1038280000F80B2C9DF8022000F80A2C9DF80320C4
:1038380000F8092C9DF8042000F8082C9DF80520B4
:1038480000F8072C9DF8062000F8062C9DF80720A4
:1038580000F8052C9DF8082000F80D5C00F8042CF1
:103868009DF80B509DF8092000F8032C9DF80A20BC
:1038780000F8022C03A92A46A0F10D0400F8015C07
:103888000CF0C1FF05F10D012246C9B2012058E72D
:10389800807839280CD83038C0B2FFF7DDFA3B4AB7
:1038A8002378137063785370A3789370032131E7FA
:1038B80010B0BDE87040FFF7C3BC80783928F7D84E
:1038C8003038C0B2FFF7C9FAE9E780783928EFD86D
:1038D8003038C0B2FFF7C2FAE1E78378303BDAB29A
:1038E800092AE5D8C0783038C2B2092AE0D8217947
:1038F800A1F14802D2B20B2ADAD8294D45FA02F2D0
:10390800D207D5D40A224D2902FB030036D13C2325
:1039180058434FF47A735843224B1860224B18606F
:10392800FFF704FB194A2378137063785370A37860
:103938009370E378D3700521237913710120FFF781
:1039480047FC154B00221A7018225A7001229A70EF
:10395800DA70A278303A02EB8201E278303A02EB70
:103968004102D2B21A7122795A71104A1278D2B22F
:103978001A72084A1278D2B25A721CE74829C8D17A
:103988004FF46163C4E700BF6B0A0108DD0400203F
:10399800E20400205403002071000020EA04002003
:1039A800DEF7FFFF08000020B400002060050020BB
:1039B8008678A6F13003092B3FF67AAFC078A0F1DC
:1039C8003003092B3FF674AF2179A1F14802D2B236
:1039D8000B2A3FF66DAF5A4B134113F001057FF4E4
:1039E80067AF584A59231370D070532311710120BF
:1039F800052153709670FFF7EBFB534918230D70A0
:103A08004B7001238B70CB70A378303B03EB8302A0
:103A1800E378303B03EB4203DBB28B712379CB7144
:103A28004A4B1B78DBB20B72494B1B78DBB24B72EB
:103A3800C1E6502B48D102297FF685AE4378303B4A
:103A4800012B3FF680AE8378312B7FF47CAE0B29B7
:103A580004D8FFF7F5FB00213A4A5BE63A4D0234F9
:103A6800002214F8013FA918303B0132DBB20C2ABE
:103A78000B73F6D1FFF708FA324B502218211A704F
:103A88009970002201215A70D97003F8041FA918EF
:103A98000132097B0C2A01F1300103F8011FF6D12C
:103AA80000232B7018236B700123AB70EB70274B2E
:103AB8001B78DBB22B72264B1B78DBB26B72EA7277
:103AC800FFF7CCFB1121C7E7412B7FF43CAE4378CD
:103AD800432B7FF438AE16297FF435AE1D4D421CBA
:103AE800002312F8011FE9540133142BF9D1FFF711
:103AF8006DF9194B5B7D012B1DD113490023EA5C3D
:103B0800C8180133D2B2142B80F82C20F7D1104BEF
:103B180000221A701B78DBB24B72FFF79FFB094A31
:103B2800631E153413F8011F02F8011BA342F9D1D3
:103B3800044A1621EEE5064B02221A70EFE700BF91
:103B4800DEF7FFFFDD040020710000206005002083
:103B580054030020610500200C02002037B50446FC
:103B68000D46002939D022480CF054FC2B78A3B319
:103B78009CB36068237880B3032B0DD0042B2ED020
:103B8800022B2AD16178012927D00B0625D403B04E
:103B9800BDE83040FFF774BD6378012B07D100788A
:103BA800012802D0022800D008B903F037FF00240A
:103BB8000DF107008DF8074003F076FF0D4A4C23FE
:103BC8001370182393709DF8073054700120413307
:103BD8000521D0701371FFF7FBFA03B030BD63788D
:103BE800012BFAD10378044A03F001031370F4E7B8
:103BF80088030020DD040020B8030020034B0022C6
:103C0800C3E902220122C3E9002270477805002097
:103C180000487047780500204FF0B04382B0DA6C56
:103C28000243DA64DB6C03400193019B02B07047E6
:103C38002DE9F04186B000240220154D0594FFF7C8
:103C4800EBFF0420FFF7E8FF124F03944FF4807650
:103C580001230DEB0001CDE90163284603230493FA
:103C68004FF4005801F032F801A93846CDF8048025
:103C780001F02CF822464146384601F04DF9284615
:103C88002246314601F048F9204606B0BDE8F081E9
:103C98000004004800080048032810B50ED8012881
:103CA80010D868B902460B484FF4807101F034F916
:103CB800002209484FF4005101F02EF9002010BDF0
:103CC8000122F0E7002203484FF4807101F024F943
:103CD8000122EEE70004004800080048022070476F
:103CE8000020704701207047002814BF16200F20BD
:103CF800704700000D48854600F025F80C480D492E
:103D08000D4A002302E0D458C4500433C4188C422E
:103D1800F9D30A4A0A4C002301E013600432A24294
:103D2800FBD30CF047FDFEF787FBFEE70000012000
:103D3800000000204C0100204C1501084C01002017
:103D480010230020FEE7704710B5032000F056FC52
:103D580001F05CFA064B18600F20FEF7B3FD04462D
:103D680018B9FEF72CFC204610BD0124FBE700BF64
:103D7800B80000204FF0E022136923F0020313611A
:103D880070474FF0E022136943F002031361704754
:103D9800014BD3F8900570470070FF1F014BD3F813
:103DA800940570470070FF1F014BD3F898057047C2
:103DB8000070FF1F8068C0F380007047F7B50023CC
:103DC80001930446002800F0E980856D25B9FEF7C7
:103DD8003FF8E56584F8545023689A68D00040F1AC
:103DE800A1809A68D10000F1B480A26D42F010025F
:103DF800A265E26D42F00102E26501251846FFF76F
:103E0800D9FFA26D02F01002024340F0C980A26DF2
:103E1800206922F4817242F00202A2659A68D207F0
:103E28005DD4226BA67E94F82CC0003A18BF0122FC
:103E38001703D4E902120A43217E42EA8132617EE5
:103E480042EAC13242EA4632002842EA4C02B4BF92
:103E580020F000414FF400113A430A4394F820102F
:103E6800012903D1002E76D142F48032616A21B152
:103E7800A66A01F4E07131430A43D968E66C21F47B
:103E8800FE3121F4FF711143D96094F83C20616838
:103E9800012A01F0404C4CEA060609D1D4E9102762
:103EA8003A433243A66C324342EA0C0242F001061E
:103EB8001F693E4A3A4032431A6121F00042B2F18A
:103EC800804F0CD0B1F1004F09D0394ED6F80827F1
:103ED80001F4701122F470120A43C6F808275A69CF
:103EE800666BA16B22F0070232435A615A6922F0CD
:103EF800700242EA01125A61002835D19A6A62F0CA
:103F08000F029A625B6903F007039E423CD10023CB
:103F1800E365A36D23F0030343F00103A36528467B
:103F280003B0F0BD9A68234922F0104222F017022C
:103F380042F080529A60204A1268B2FBF1F20132D4
:103F480052000192019A002A3FF44BAF019A013ABC
:103F5800F7E7002552E7A16D41F02001A165E16D69
:103F680041F00101E16581E7B0F5001FCAD19A6A05
:103F7800E269013A92006FF00F0102F01C0201FAA7
:103F880002F2216E0A43BCE7A36D23F0120343F04B
:103F98001003A365E36D43F00103E3650125BEE764
:103FA800A36D43F01003A365F8E700BF02FCFF1FF1
:103FB80000200140400D0300B8000020F8B5456915
:103FC800082D04460E460AD00368DB68D80705D5D5
:103FD800A36D43F02003A3650120F8BD0425FEF777
:103FE80073FC074623681A682A4220D0A26D42F45F
:103FF8000072A265DA6812F4406F14D1A27E92B9F9
:104008001A6812070FD51846FFF7D4FE20BB5A6866
:1040180022F00C025A60A26D22F4807222F0010292
:1040280042F00102A265227EFAB10020D5E7711C98
:10403800D9D0FEF749FCC01BB04201D8002ED1D11F
:1040480023681B682B40CDD1A26D84F8543042F010
:104058000402A2650320C0E7A26D42F02002A26517
:10406800E26D42F00102E265DDE70C221A60DCE74E
:104078000368186C70470000F7B50023019390F8A7
:104088005430012B044600F0C08005680269012302
:1040980080F854302846FFF78DFE002840F0AF80A6
:1040A800D1E90030022822F004027ED0B2F1004F9C
:1040B800C3F3110E35D1AA6A42EA0E02AA628A68CF
:1040C800686902EA032222F07C4222F0FF0220EA19
:1040D80003210A43002B6A611DDA4D4A4D4DD2F87F
:1040E8000817AB4201F0E07043D10D0213D4D2F8A7
:1040F800083723F0E073034343F40003C2F808379A
:10410800454B1A68454BB2FBF3F20C2302FB033311
:104118000193019B53BB0020002384F8543003B063
:10412800F0BD226E00F01F074FF00F0C0CFA07FCD1
:104138006FEA0C0622EA0C0CBEF1000F11D1C3F392
:104148008462BA4042EA0C0222668008E2690130C1
:104158009042B4D8A86AC3F38362BA400640324397
:10416800ACE793FAA3F2B2FA82F2EAE7019B013BC9
:10417800CEE72B4DAB420BD1C901CCD4D2F80837CE
:1041880023F0E073034343F08073C2F80837C2E7B3
:10419800244DAB42BFD14B02BDD4D2F8083723F02F
:1041A800E073034343F48003EFE7B2F1004F01BF2C
:1041B800AA6AC3F311018A43AA62002BABDA154835
:1041C80013498342D1F8082709D1D1F8083702F0FA
:1041D800A07223F0E0731A43C1F808279BE7104840
:1041E800834204D1D1F8083702F44002F1E70D48C0
:1041F800834290D1D1F8083702F0C072E9E7A26D86
:1042080042F02002A265184686E7022087E700BF31
:1042180000200140001000B0B8000020400D03004D
:10422800004000B8002000B4026838B504461046C3
:10423800FFF7C0FD08B9002038BD9368990707D477
:10424800936823F0004323F0170343F010039360AF
:10425800FEF73AFB054623689B685B07EBD5FEF73C
:1042680033FB401B0228F6D923689B685A07F2D50E
:10427800A36D43F01003A365E36D43F00103E36509
:104288000120D9E773B50023026801939368DD071D
:10429800044602D5002002B070BD9168214B194236
:1042A80009D0A36D43F01003A365E36D43F0010348
:1042B800E3650120EFE7936823F0004323F0170339
:1042C80043F001039360184BD3F8083718021CD445
:1042D800637E012BDED0FEF7F7FA144E05462268FE
:1042E8001368DB07D6D49368D9075FBF9368334058
:1042F80043F001039360FEF7E7FA401B0228EED96A
:1043080023681B68DA07EAD4CBE7094B094A1B681C
:10431800B3FBF2F301330193019B002BD8D0019B2F
:10432800013BF8E71700008000200140E8FFFF7F0D
:10433800B8000020400D030038B504460068FFF7B8
:1043480039FD054620BB94F85430012B20D00123B9
:1043580084F854302046FFF795FFB0B9A36D226862
:1043680023F4706323F0010343F48073A3651C23D3
:10437800E065136084F85400936823F0004323F049
:10438800170343F00403936038BD84F85450FBE7E7
:104398000220F9E7026838B5936891680446C807AF
:1043A80001D4002038BD9907FBD4936803F00503B6
:1043B800012B19D1936823F0004323F0170343F02E
:1043C8000203936003231360FEF77EFA0546236811
:1043D8009B68DB07E5D5FEF777FA401B0228F6D97C
:1043E80023689B68DA07F2D5A36D43F01003A36531
:1043F800E36D43F00103E3650120D3E770B504469C
:1044080000284BD0836D43F002038365FFF70CFF50
:10441800054668B92046FFF7BDFF054608B90123E0
:10442800A3652268936823F0104323F01703936071
:1044380023685A6822F4677222F003025A6040F235
:104448009F321A60D968164A0A40DA601A6922F05F
:1044580040421A615A6922F007025A611A6A02F048
:10446800F0221A625A6A02F0F0225A62DA6A02F0FC
:10447800F022DA629A6A0B4A00269E62D2F808375E
:1044880023F0FE73C2F808372046FDF7F5FCE66511
:104498002666A66584F85460284670BD0125FBE7AA
:1044A80000023E830020014010B590F85430012BE3
:1044B800044615D0012380F85430FFF7B5FE58B9EB
:1044C8002046FFF767FF38B9A36D23F4807323F004
:1044D800010343F00103A365002384F8543010BDA1
:1044E8000220FCE7F7B50023019390F85430012B24
:1044F80004467FD0012380F85430FFF74BFF236830
:104508009A6812F00102054607D0A36D43F0100324
:10451800A365002384F854302DE0A16D364F21F4B3
:10452800817141F00201A165DE68D96826F4FF4671
:1045380026F07C0621F40041360421F00301360CF4
:10454800D96008209968394041F00041996099681C
:10455800002913DA0199013101910199B1F52E3F32
:10456800F5D3A36D23F0120343F01003A3650023D2
:1045780084F854300125284603B0F0BDD3F8B410B0
:10458800013801F07F010A44DCD199681A480140DA
:1045980041F001019960D3F8B41021F07F0141EA9C
:1045A800D202C3F8B4209A68024042F002029A602C
:1045B800FEF78AF9074623689A68D20708D4DA68AA
:1045C8003243DA60A36D23F0030343F001039FE74E
:1045D800FEF77AF9C01B0228EDD923689B68D90732
:1045E800E9D5A36D43F01003A365E36D43F0010320
:1045F800E365BFE70225BEE7E8FFFF7F0749CA6812
:1046080022F4E0620302120403F4E063120C134381
:1046180043F0BF6343F40033CB60704700ED00E024
:10462800164B30B5DC68C4F30224C4F10703251D1A
:10463800042B28BF0423062D4FF0FF358CBF033C05
:10464800002405FA03F321EA0303A54022EA050240
:10465800A340002843EA0203ACBF00F16040084AC7
:104668004FEA0313B8BF00F00F00DBB2AABF00F592
:104678006140135480F8003330BD00BF00ED00E006
:1046880014ED00E0002807DB044A4109012300F08B
:104698001F00834042F82130704700BF00E100E06E
:1046A80000280CDB4309064900F01F0020330122D3
:1046B800824041F82320BFF34F8FBFF36F8F7047BD
:1046C80000E100E070B5D0E913456560446D14B1B0
:1046D800D0E916456560D0E9105404F01C060124A1
:1046E800B4406C60046863608368102B0BBFA260E1
:1046F800A160E160E26070BD0268416CD3B210B5A0
:10470800083B1424B3FBF4F30B4CA24288BF0B4ABA
:1047180021F0030199BF01F1804202F502325218DB
:1047280007338264064AC26403F01F03012202FAB7
:1047380003F3036510BD00BF070402401C080240D4
:104748008008024038B500285CD002682E4B9A4297
:104758004FF014014AD82D4B1344B3FBF1F32C4905
:104768009B00C0E91013022380F8253013680569FF
:1047780023F4FF4323F070031360D0E9024323437B
:104788002B43456911682B4385692B43C5692B4326
:10479800056A2B430B431360FFF7AEFFB4F5804F58
:1047A80004BF002343604368816C03F07F020A6002
:1047B800D0E91314013B032B4C601ED8154B164946
:1047C800816513449B000121013A01FA02F200219C
:1047D8004365C2651960114B5A6400230122C36303
:1047E80080F8243080F82520184638BD0C4B134437
:1047F800B3FBF1F30B499B00B3E70023C0E9153382
:10480800C365EAE70120F0E707040240F8FFFDBFAF
:10481800000002403F8200104009024000090240A7
:10482800F8FBFDBF0004024038B5002841D00268FB
:10483800136823F0010313601F4B9A424FF01401D1
:1048480030D81E4B1344B3FBF1F31D499B00C0E95C
:104858001013012403F01C0304FA03F30025156068
:104868004B60FFF749FF836C41681D60D0E9133244
:104878005A604A1E032A06D8124B0B449B009440E8
:104888001D60114B5C640023C363C0E91533C0E9A4
:104898000B33C0E90D33C36580F8253080F8243028
:1048A800184638BD094B1344B3FBF1F308499B0084
:1048B800CDE70120F5E700BF07040240F8FFFDBF80
:1048C800000002403F82001000090240F8FBFDBFD3
:1048D8000004024070B590F82450012D04463BD0E6
:1048E80090F825600125AE4280F824504FF000066C
:1048F8002CD1022580F825500568C6632E6826F05D
:1049080001062E60FFF7DEFE036BBBB12B6843F098
:104918000E032B60A36C1A68D20342BF1A6842F4D4
:1049280080721A60636D1BB11A6842F480721A6053
:104938002B6843F001032B60002070BD2B6823F027
:1049480004032B602B6843F00A03E2E78023C36368
:1049580080F824602846F0E70220EEE7034640B1DD
:1049680090F82520022A06D00422C263002280F88B
:104978002420012070470268806C116821F00E0124
:104988001160016821F480710160116821F0010152
:104998001160D3E9100202F01C0101228A40426032
:1049A800D3E9132151605A6D32B1116821F4807135
:1049B8001160D3E9162151600122002083F82520D7
:1049C80083F82400704708B590F82530022B03D0EF
:1049D8000423C363012008BD03681A6822F00E028D
:1049E8001A601A6822F001021A60826C136823F4B4
:1049F80080731360D0E9101303F01C020123934065
:104A08004B60D0E913325A60436D33B11A6822F40F
:104A180080721A60D0E916325A60012380F8253076
:104A2800002380F82430836B03B198470020D2E735
:104A380070B4426C046C036826681D6802F01C029E
:104A48000421914031420FD015F0040F0CD01A68A0
:104A580092065EBF1A6822F004021A60036B616056
:104A6800002B33D070BC184702219140314217D037
:104A780015F0020F14D01A68940606D41A6822F0AA
:104A88000A021A60012280F82520114A93428CBF3D
:104A9800104B114B5960002380F82430C36ADFE7BC
:104AA80008219140314211D029070FD5196821F00A
:104AB8000E011960012303FA02F26260C36380F8F1
:104AC8002530002380F82430436BC9E770BC704759
:104AD8008000024000040240000002400A4A536974
:104AE80043F4802330B55361EFF3108472B600238A
:104AF800CD58C5500433B3F5807FF9D11369DB0372
:104B0800FCD484F3108830BD00400058064B5A6925
:104B1800002ABFBF054A9A6002F188329A60BABF7C
:104B28005869C00F002070470040005823016745AE
:104B3800044B5A6942F000425A615869C043C00F99
:104B4800704700BF0040005870B50546FDF7BCFE31
:104B5800124E04463369D90313D43369DA0744BFC4
:104B6800012232614CF2FA32134011D10B4E3069F6
:104B780010F480200BD0FDF7A7FE001BA842F6D347
:104B880004E0FDF7A1FE001BA842E3D3032070BD9B
:104B9800024A1361024A01205360F8E700400058B6
:104BA800880500202DE9F041184D98462B78012BF7
:104BB80006460C46174626D001232B704FF47A7010
:104BC80000236B60FFF7C0FFA0B9012E16D1104A71
:104BD800536943F0010353612760BFF36F8FC4F833
:104BE80004804FF47A70FFF7AFFF094A536923EA4C
:104BF8000603536100232B70BDE8F0813946204637
:104C0800FFF76CFFEDE70220F6E700BF88050020FC
:104C180000400058054A536923F47E7343EAC000F4
:104C280040F4803040F00200506170470040005866
:104C38002DE9F041234F3B78012B054688463FD0AC
:104C480001233B704FF47A7000237B60FFF77CFFF1
:104C5800044688B92B68042B13D11B4A536943F4C3
:104C6800803343F0040353614FF47A70FFF76CFF0D
:104C78000446154B1A681B6800233B702046BDE8A4
:104C8800F0814FF0FF33C8F800306E68D5E9013283
:104C98001344B3420AD93046FFF7BCFF4FF47A7089
:104CA800FFF752FF50B1C8F800600446064A53693E
:104CB80023F47E7323F002035361DAE70136E5E754
:104CC8000224DBE788050020004000582DE9F04F5A
:104CD800524C00234FF00F090A6832FA03F501D14C
:104CE800BDE8F08F012505FA03F818EA020200F082
:104CF8008E804E68032706F003054FEA430E07FA35
:104D08000EFC6F1E012F6FEA0C0C32D8876807EA79
:104D18000C0ACF6807FA0EF747EA0A078760476860
:104D280027EA0808C6F300179F4047EA08074760C4
:104D3800C76807EA0C088F6807FA0EF747EA0807FA
:104D4800022DC76017D14FEAD30800EB880803F09B
:104D5800070AD8F820704FEA8A0A09FA0AFB27EAF4
:104D68000B0B0F6907FA0AF747EA0B07C8F8207018
:104D780001E0032DDCD1076805FA0EF507EA0C07F8
:104D88003D4316F4403F056041D023F0030707F187
:104D9800804707F5803703F0030CBD684FEA8C0C99
:104DA8004FF0070E0EFA0CFEB0F1904F25EA0E0EEA
:104DB8002FD01B4DA8422ED005F58065A84214BF00
:104DC8000725022505FA0CF545EA0E05BD6025689C
:104DD800D74316F4801F0CBF3D4015432560656816
:104DE80016F4001F0CBF3D4015436560D4F8805091
:104DF80016F4803F0CBF3D401543C4F88050D4F8EA
:104E08008450B60354BF3D401543C4F88450013361
:104E180062E70025D6E70125D4E700BF000800585F
:104E280000040048374A2DE9F04F00234FF0010AEB
:104E38004FF0070B4FF00F0931FA03F401D1BDE829
:104E4800F08F0AFA03FC1CEA010654D023F003048D
:104E580004F1804404F5803403F00307A568BF001B
:104E68000BFA07F8B0F1904F08EA050E45D0264D29
:104E7800A84244D005F58065A8420CBF0225072545
:104E8800BD40754517D1D2F8805025EA0605C2F80D
:104E98008050D2F8845025EA0605C2F88450156877
:104EA80025EA06051560556825EA06055560A568D2
:104EB80025EA0805A560056803265C0006FA04F4DF
:104EC80023FA06F6254300EB8606056003F007057E
:104ED800376AAD0009FA05F527EA050737628568DC
:104EE80025EA04058560456825EA0C054560C5681E
:104EF80025EA0404C46001339EE70025C0E70125C4
:104F0800BEE700BF000800580004004803691942C2
:104F180014BF0120002070470AB181617047816287
:104F280070470000044AD168014208B502D0D06039
:104F3800FEF741F908BD00BF00080058024A13688F
:104F480043F4807313607047000400580D4B10B58C
:104F58005B690C4628B99A0507D500F027F820B1F7
:104F680010BD9B0501D400F019F8074A1369012CFC
:104F780023F00403136101D130BFF1E740BF20BF24
:104F880020BFEDE70004005800ED00E0024B186870
:104F980000F4C060704700BF00040058024A13685C
:104FA80043F4804313607047000400580C4A1368A8
:104FB80023F4804313600B4B1B6832214B430A498F
:104FC800B3FBF1F35169890500D533B9536913F47B
:104FD800007F14BF032000207047013BF2E700BFA9
:104FE80000040058B800002040420F000B4A136824
:104FF80023F0070343F002031360094B1A690128E1
:1050080042F004021A6105D130BF1A6922F0040285
:105018001A61704740BF20BF20BFF6E70004005860
:1050280000ED00E04FF0B0431868C0F3404070470F
:105038004FF0B0431868C0F3400070474FF0B042DB
:10504800536823F47F4343EA0023536070474FF0CB
:10505800B0431868C0F34060704700007FB54FF058
:10506800B0432C4AD3F80831C0F3031003F00F0300
:1050780052F82040284A52F82330B4FBF3F4FFF7E3
:1050880085FF264B054693E80700B5F5007F04AB7E
:1050980003E9070010D0224B9C4218D303F5B7034D
:1050A80003F67F539C4229D903F5741303F5106363
:1050B8009C4225D802230BE01A4B9C4207D91A4B75
:1050C8009C421BD903F5370303F5D853F0E70023B7
:1050D80004AA02EB830353F80C4C144D2B6823F0FD
:1050E800070323432B60FDF7EFFB06462B6803F00D
:1050F80007039C4206D1002004B070BD0123E7E7F6
:105108000024EAE7FDF7E0FB801B0228EED9032024
:10511800F2E700BF800A0108E00A01085009010807
:10512800C0CF6A00BFEA21013F9334020040005813
:105138004FF0B04310B59A68D96812F00C0205D048
:105148000C2A4AD101F00303012B51D14FF0B04191
:105158002B480B6813F0080306D00B6813F00803FC
:1051680037D1D1F8941007E00C68240756BFD1F85E
:1051780094300968C3F3032350F82330002A0CBF86
:10518800184600204FF0B0418A6802F00C020C2A41
:105198001ED1CA6802F00302022A2ED0032A06D1C1
:1051A8000B68184A13F4801F174B18BF13464FF0AB
:1051B800B042D068D168D268C0F306205843C1F322
:1051C80002130133B0FBF3F0530F0133B0FBF3F0DC
:1051D80010BD0B68C3F30313CEE7042A05D0082AD1
:1051E80006D11B6813F4801305D006480023C9E7CD
:1051F80000231846C6E70448C4E7024BD7E700BFB8
:10520800800A01080024F4000048E80108B5FFF707
:105218008FFF4FF0B043044A9B68C3F3031352F85F
:105228002330B0FBF3F008BDE00A01082DE9F04196
:105238000446002853D04FF0B0439D68DE680368E9
:105248009B0605F00C0506F0030668D5026A1DB139
:105258000C2D46D1012E44D1002A40D04FF0B04346
:10526800A16A1A68170756BFD3F894301B681B0940
:1052780003F0F00399421FD90846FFF7EFFE002814
:105288002DD14FF0B042136843F008031360136840
:10529800A16A23F0F0030B431360606AFFF7CEFEA8
:1052A800FFF7B4FFAB4B1860AB4B1868FDF70AFB70
:1052B800002834D0BDE8F0814FF0B042136843F0C5
:1052C80008031360136823F0F0030B431360606A4C
:1052D800FFF7B4FE0846FFF7C1FE0028E0D0012022
:1052E800E8E74FF0B043002A54D01A6842F00102B0
:1052F8001A60FDF7E9FA0746FFF79AFE002842D040
:105308004FF0B042136843F0080313601368A16AB2
:1053180023F0F0030B431360606AFFF78FFE2368E6
:10532800D80748D42368990700F18C8023681E07A2
:1053380040F1FA80A3694FF0B046002B00F0E180FD
:10534800D6F89430E16903F01002914200F0C4806D
:1053580003F00302022AC2D0D80740F1B380D6F87E
:10536800943023F00103C6F89430FDF7ADFA0746F0
:10537800D6F89430990740F1A580FDF7A5FAC31B2C
:10538800112BF5D904E0FDF79FFAC01B0228B3D909
:1053980003208FE71A6822F001021A60FDF794FAD9
:1053A8000746FFF745FE0028B9D0FDF78DFAC01B68
:1053B8000228F6D9ECE7082D03D00C2D05D1032ED1
:1053C80003D16368002BADD189E74FF0B043A168E2
:1053D8001A6822F480120A431A606268B2F5803FA4
:1053E80010D11A6842F480321A60FDF76DFA074648
:1053F800FFF718FE002895D1FDF766FAC01B642850
:10540800F6D9C5E7B2F5041F04D11A6842F40012B0
:105418001A60E6E7196821F480311960196821F4E7
:1054280000111960002AE0D1FDF74EFA0746FFF790
:10543800F9FD00283FF476AFFDF746FAC01B642853
:10544800F5D9A5E7042D236903D00C2D0ED1022E22
:105458000CD1002B3FF443AF4FF0B0426169536861
:1054680023F0FE4343EA016353605FE74FF0B04621
:10547800BBB1336843F480733360FDF725FA074600
:1054880033685A0505D4FDF71FFAC31B022BF7D959
:105498007EE77368626923F0FE4343EA0263736040
:1054A80044E7336823F480733360FDF70DFA074649
:1054B80033685B057FF53AAFFDF706FAC31B022B8D
:1054C800F6D965E74FF0B042E169D2F8943023F09D
:1054D80010030B43C2F894304FF0B047D7F894301C
:1054E80043F00103C7F89430FDF7EEF90646D7F804
:1054F80094309A0718D4FDF7E7F9831B112BF6D9D6
:1055080046E7D6F8943023F00103C6F89430FDF747
:10551800DBF90746D6F894309B0705D5FDF7D4F993
:10552800C31B112BF6D933E72368580754D50B4F03
:105538003B68D90514D4FFF701FDFDF7C5F9064608
:105548003B68DA050CD4FDF7BFF9831B022BF7D9AA
:105558001EE700BFB8000020BC000020000400586F
:10556800E3684FF0B046002B58D023F08003052B9A
:1055780002BFD6F8903043F00403C6F890304FF0DD
:10558800B046FDF7A1F9D6F8903043F0010307467D
:10559800C6F8903041F28838D6F890309B0705D489
:1055A800FDF792F9C31B4345F6D9F1E6E36823F00A
:1055B8000403812B1BD1FDF787F9D6F8903043F00F
:1055C8008003C6F8903007464FF0B04641F288385D
:1055D800D6F89030180504D5E36A002B4AD100208C
:1055E80068E6FDF771F9C01B4045F1D9D0E6FDF733
:1055F8006BF9D6F8903023F08003C6F89030074650
:105608004FF0B04641F28838D6F890301905E3D506
:10561800FDF75AF9C01B4045F6D9B9E6FDF754F92C
:10562800D6F8903023F080030746C6F8903041F250
:105638008838D6F890301A0516D4FDF745F9D6F80B
:10564800903023F00103C6F8903007464FF0B04879
:1056580041F28836D8F890309B07BDD5FDF734F96C
:10566800C31BB342F6D993E6FDF72EF9C01B40459C
:10567800DFD98DE60C2D4ED0022B4FF0B0431A68BF
:1056880022F080721A6033D1FDF71EF90546FFF744
:10569800DEFC38BBD4E90C314FF0B0420B43D06884
:1056A8002D4901400B43E16B0B43216C0B43616CAB
:1056B8000B43A16B43EA0123D360136843F0807363
:1056C8001360D36843F08053D360FDF7FDF80446B8
:1056D800FFF7BDFC002882D1FDF7F6F8001B0A2869
:1056E800F6D955E6FDF7F0F8401B0A28CFD94FE662
:1056F800FDF7EAF80446FFF7AAFC30B94FF0B042CC
:10570800164BD1680B40D36069E7FDF7DDF8001B45
:105718000A28F0D93CE6012B3FF4E1AD4FF0B04345
:10572800D868236B00F003029A427FF4D8AD626B0D
:1057380000F0700393427FF4D2ADA26B00F4FE43F5
:10574800B3EB022F7FF4CBAD636C00F06040C01A5E
:1057580018BF0120AEE500BF8C80C111FCFFFEEE32
:105768002DE9F0410D46044610B90120BDE8F0814D
:10577800684E336803F007038B4216D323689A07F1
:1057880027D54FF0B047A268BB6823F0F003134356
:10579800BB60FDF799F80646BB68DB0319D4FDF733
:1057A80093F8831B022BF7D911E0336823F0070322
:1057B8000B433360FDF788F80746336803F00703A7
:1057C800AB42DBD0FDF780F8C01B0228F5D90320D7
:1057D800CCE72368580617D54FF0B0476269D7F869
:1057E800083123F00F0343EA1213C7F80831FDF715
:1057F8006BF80646D7F80831D90305D4FDF764F8E5
:10580800831B022BF6D9E2E723685A0713D54FF01A
:10581800B047E268BB6823F4E0631343BB60FDF75D
:1058280053F80646BB689B0305D4FDF74DF8831B68
:10583800022BF7D9CBE72368180714D54FF0B047E8
:105848002269BB6823F4605343EAC203BB60FDF7D7
:105858003BF80646BB68590305D4FDF735F8831BAA
:10586800022BF7D9B3E72368DA070FD4294C23684A
:1058780003F00703AB4239D8FFF7C8FC264B186082
:10588800264BBDE8F0411868FDF71CB86268022A8B
:105898001DD1FFF7C7FB00283FF467AF4FF0B046B4
:1058A80041F28838B36823F003031343B360FDF76C
:1058B8000BF80746B368626803F00C03B3EB820F7A
:1058C800D4D0FDF701F8C01B4045F3D97FE7032A80
:1058D80002D1FFF7BCFBDEE712B9FFF7A9FBDAE755
:1058E8004FF0B0431B685B05D8D43EE7236823F02C
:1058F80007032B432360FCF7E7FF0646236803F002
:105908000703AB42B8D0FCF7DFFF801B0228F5D9AC
:105918005DE700BF00400058B8000020BC00002030
:1059280008B5FFF773FC4FF0B043044A9B68C3F314
:10593800022352F82330D84008BD00BFC00A01082E
:1059480008B5FFF763FC4FF0B043044A9B68C3F304
:10595800C22352F82330D84008BD00BFC00A01084E
:105968004FF0B043D3F89000C0F3400070474FF0B9
:10597800B0410209D1F8883002F47F22000123EAFD
:10598800020300F47F200343C1F8883070474FF0CA
:10599800B041020CD1F88830120423EA020343EA2A
:1059A8000040C1F8880070470368DA0370B5044600
:1059B80039D5FFF7C3FAFCF787FF614E0546336810
:1059C800DB0532D54FF0B043616BD3F8902002F479
:1059D800407291421DD0D3F89010D3F8902042F431
:1059E8008032C3F89020D3F8902021F4407022F43C
:1059F80080328D07C3F89020C3F8900009D5FCF7D2
:105A080063FF41F288360546FFF7AAFF012840F0F8
:105A180090804FF0B042616BD2F8903023F440731D
:105A28000B43C2F89030002605E0FCF74DFF401B01
:105A38000228C4D903262568E8070AD54FF0B041E3
:105A48006268D1F8883023EA124392B21343C1F84E
:105A58008830A9070AD54FF0B041A268D1F888303C
:105A680023EA124392B21343C1F88830AA0609D533
:105A78004FF0B0422169D2F8883023F440630B43D9
:105A8800C2F88830AB0502D5206AFFF780FF6805A9
:105A980002D5606AFFF77BFF290502D5A06AFFF7E8
:105AA80076FF6A0602D56069FFF761FF2B0602D50B
:105AB800A069FFF75CFFE80502D5E069FFF757FF2B
:105AC800E90610D54FF0B042E168D2F8883023F4E7
:105AD80040730B43C2F88830B1F5807F02BFD368AA
:105AE80043F08073D3602A040ED54FF0B042216B87
:105AF800D2F8883023F040430B43C2F8883019B9F4
:105B0800D36843F08073D3606B0410D54FF0B04274
:105B1800E16AD2F8883023F040530B43B1F1005FBB
:105B2800C2F8883003D1D36843F48033D360304659
:105B380070BDFCF7C9FE401BB0427FF665AF79E740
:105B48000004005830B590F82C30012B02464FF075
:105B5800020022D0174B82F82D00CA24012582F8B2
:105B68002C505C6253245C62B1F5807F146B996998
:105B780014D121F488519961596C24F0010421F061
:105B8800004159641463DD650A4BFF215962002006
:105B9800012382F82D3082F82C0030BD21F4085101
:105BA8009961D96C24F0020421F00041D96414638E
:105BB800D865E9E70028004070B50B4E036B756D9A
:105BC8001D40EA07044603D50123F365FCF78FFF60
:105BD800AB0704D50223F365204600F0C9F9012379
:105BE80084F82D3070BD00BF0028004038B50A4C3D
:105BF800E36823F02003E360FCF766FE0546E368EC
:105C08009B0601D5002038BDFCF75EFE401BB0F5B1
:105C18007A7FF4D90320F6E700280040F8B5114D43
:105C2800EC6814F0400406461AD1EB6843F0800390
:105C3800EB60FCF749FE23460746EC6814F0400485
:105C480001D1032B01D11846F8BDFCF73DFEC01B5E
:105C5800B0F57A7F234684BF032386F82D30ECE71E
:105C68000023F0E70028004038B50F4CE36823F024
:105C78008003E360A3699B06054606D4FFF7B6FFD9
:105C880010B1032085F82D0038BDA36923F0200347
:105C9800A361FFF7ABFF10B1032085F82D00A369BE
:105CA80043F02003A361EFE70028004038B504461D
:105CB80000284BD090F82D3003F0FF021BB980F874
:105CC8002C20FCF709FC0223214D84F82D30EB68C9
:105CD800DB0636D4CA236B6253236B622046FFF778
:105CE8009DFF10B1FF236B6238BDAB6923F08E6353
:105CF80023F04003AB6121696368AA690B4313432E
:105D0800A2691343AB61D4E9022343EA02432B613E
:105D1800D4E90931EA680B4322F4F8521343EB60E3
:105D28002046FFF7A1FF0028DCD1D4E90713AA69B0
:105D38000B4322F06042134362691343AB61FF23B4
:105D48006B62012384F82D300020CDE70120CBE7DA
:105D5800002800400023092803D840EA0310C0B2F5
:105D680070470A380133C0B2F5E700002DE9F04763
:105D780090F82C30012B05464FF0020069D0012322
:105D880085F82C304E4B85F82D00DE6806F44076F9
:105D9800B6F5807F78D04C69087891F8019091F831
:105DA80002A091F82470002A55D19B6913F0400392
:105DB80008BFCB70FFF7CEFF80464846FFF7CAFF03
:105DC80002465046FFF7C6FF81463846FFF7C2FF36
:105DD8000B6ACF78234343EA875343EA090343EA2C
:105DE800084343EA022343EA0063354ACA20506263
:105DF800532050628C6A8869B4F5807F946945D1D4
:105E080024F4885494610124D465B6F5807F09BFD1
:105E1800CB6913640343536418BF5064284B4A6822
:105E28001A672A6B42F001022A639A6942F488527F
:105E38009A61244AD2F8803043F40033C2F88030A3
:105E48001F4BFF225A620020012385F82D3085F868
:105E58002C00BDE8F087B4F1803F07D0B4F5000FFF
:105E680004D09B6913F0400308BFCB700B6ACA7853
:105E78001C4344EA0A0444EA004343EA092343EA88
:105E8800825343EA0763B0E70023AEE724F40854DB
:105E980094610224D465B6F5807F09BFCB69936409
:105EA8000343D36418BFD064054B4A685A672A6B0A
:105EB80042F002022A639A6942F40852B8E700BF26
:105EC800002800400008005890F82C20012A0346BA
:105ED8004FF0020012D00A4A83F82D00CA215162FD
:105EE80053215162916941F020019161FF21516272
:105EF8000020012283F82D2083F82C00704700BF72
:105F08000028004090F82C20012A03464FF0020098
:105F180019D00D4A83F82D00CA21516253215162CC
:105F280091690A4841F080019161D0F8801041F4EC
:105F38008021C0F88010FF2151620020012283F8DF
:105F48002D2083F82C0070470028004000080058D6
:105F5800064B5A6D520610B5044603D54022DA6541
:105F6800FCF7C8FD012384F82D3010BD002800403F
:105F78007047890001F1804101F531410A6070479D
:105F8800890001F1804101F531410868704700003E
:105F9800034AD2F8903043F40043C2F89030704777
:105FA80000040058034AD2F8903023F40043C2F8A2
:105FB8009030704700040058074B1A6822F04002DE
:105FC8001A6040F441704FF4B85218605A601A6869
:105FD80042F040021A6070470000015837B5054684
:105FE80000284ED0837903F0FF046BB1032C0BD04B
:105FF800254B4FF400629A612868FFF7DDFF002403
:1060080001232B71AC602FE000236B712846FCF74D
:1060180075FB1E4AD2F8903043F48053C2F8903092
:10602800002CE5D102234FF0B042AB71D2F8943086
:1060380023F40043C2F89430154B1B681C214B43D2
:10604800DB0C64214B430193019B93B90124AC60A1
:10605800FFF79EFF0C4B9A6842F400629A604FF477
:1060680000629A61002CC7D00123AB71204603B0AF
:1060780030BD019B013B0193D2F894305B04E3D41B
:10608800E6E70124F2E700BF0004005800080058C2
:10609800B800002037B5174D2B6802461C20434333
:1060A800DB0C6420434314480193019B93B90120FE
:1060B8009060114C21732B681C214B43DB0C64212D
:1060C8004B430193019B6BB9012090600A4BDB683D
:1060D80003B030BD019B013B019383689C07E4D565
:1060E8000020E6E7019B013B0193A368DB07E9D5A4
:1060F800ECE700BFB80000200000015837B5184D84
:106108002B6802461C204343DB0C6420434315489C
:106118000193019BA3B901209060124CFF232373C4
:106128002B681C256B43DB0C64256B430193019B97
:1061380073B9012090600B4BDB680B7003B030BD66
:10614800019B013B019383689C07E2D50020E4E7AB
:10615800019B013B0193A368DB07E8D5EBE700BF90
:10616800B8000020000001580E4B0F491B68182288
:10617800534382B01B0D6422534301934B69019A28
:10618800C3F3800322B902238360012002B0704761
:10619800019A013A01924A69920701D5002BEDD183
:1061A8000020F3E7B80000200004005807B5037981
:1061B800012B0FD10A4B1B68182253431B0C019368
:1061C800FFF7F0FE019B013B0193019B002BF9D1E6
:1061D800FFF7DEFE03B05DF804EBFFF7C5BF00BFB5
:1061E800B8000020F8B51E468379012B15460446F1
:1061F8000F46DAB22DD14379012B2AD002234271FE
:106208008371FFF7D3FF0D212046FFF7CBFEFFF781
:1062180041FF390A2046FFF73DFFF9B22046FFF754
:1062280039FF2E44B5420ED12046FFF7B1FEFFF7E5
:106238009BFFA06801230038A3714FF0000318BF2B
:1062480001206371F8BD15F8011B2046FFF722FFF6
:10625800E8E70220F6E7F8B51E468379012B1546D4
:1062680004460F46DAB22FD14379012B2CD0427164
:10627800FFF79CFF1D212046FFF794FEFFF70AFF5A
:10628800390A2046FFF706FFF9B22046FFF702FF5A
:1062980000212046FFF7FEFE2E44B5420ED12046CF
:1062A800FFF776FEFFF760FFA06801230038A371AF
:1062B8004FF0000318BF01206371F8BD294620463E
:1062C800FFF71CFF0135E8E70220F6E7F8B51F469F
:1062D8008379012B154604460E46DAB22CD1437950
:1062E800012B29D04271FFF761FF06F0EF03A3F1FC
:1062F800840253425341237131462046FFF752FE30
:10630800FFF7C8FE2F44AF4210D1FFF741FE842E9D
:1063180002D02046FFF728FFA06801230038A371A8
:106328004FF0000318BF01206371F8BD15F8011B79
:106338002046FFF7AFFEE6E70220F6E7F8B51E466F
:106348008379012B154604460F46DAB227D14379E3
:10635800012B24D04271FFF729FF39462046FFF769
:1063680021FEFFF797FE00212046FFF793FE2E44FB
:10637800B5420ED12046FFF70BFEFFF7F5FEA068E9
:1063880001230038A3714FF0000318BF0120637187
:10639800F8BD29462046FFF7B1FE0135E8E702209F
:1063A800F6E737B50023ADF8043001AA022312211D
:1063B8000546FFF7C3FFBDF80440022364BA01AAEB
:1063C800A4B219462846FFF781FFE20702D52846FE
:1063D80009F03EFBA30702D5284609F03FFB6007FA
:1063E80002D5284609F064FB210702D5284609F0A2
:1063F80065FBE20602D5284609F066FBA30602D52E
:10640800284609F04FFB600602D5284609F02CFB08
:10641800210606D514F4807118BF0121284609F019
:1064280029FBA20502D5284609F034FB630402D5EE
:10643800284609F04FFB03B030BDF8B51E468379F6
:10644800012B154604460F46DAB227D14379012BB2
:1064580024D04271FFF7AAFE0E212046FFF7A2FDC5
:10646800FFF718FE39462046FFF714FE2E44B542C2
:106478000ED12046FFF78CFDFFF776FEA0680123BA
:106488000038A3714FF0000318BF01206371F8BDF5
:1064980015F8011B2046FFF7FDFDE8E70220F6E7A7
:1064A800F8B51E468379012B154604460F46DAB225
:1064B8002BD14379012B28D04271FFF777FE1E219B
:1064C8002046FFF76FFDFFF7E5FD39462046FFF749
:1064D800E1FD00212046FFF7DDFD2E44B5420ED137
:1064E8002046FFF755FDFFF73FFEA068012300385F
:1064F800A3714FF0000318BF01206371F8BD29464E
:106508002046FFF7FBFD0135E8E70220F6E70268C1
:1065180052E8003F23F0C00342E800310268002936
:10652800F5D102F1080353E8003F23F4000302F118
:10653800080C4CE800310029F3D12023C0F888303A
:106548007047000010B5026852E8003F23F49073CA
:1065580042E8003102680029F5D10F4C02F1080326
:1065680053E8003F234002F1080C4CE800310029B1
:10657800F4D1C36E012B07D152E8003F23F010037A
:1065880042E800310029F7D12023C0F88C300023DD
:10659800C366436710BD00BFFEFFFFEFF8B50446B2
:1065A8001346D4F88850202D32D1F1B1EAB1E06F0A
:1065B800A4F85620A4F8542000262122C4F890609C
:1065C8002165C4F88820226888B1124FC762124F2B
:1065D8000763124F2832C0E90D76FEF77BF930B118
:1065E8001023C4F89030C4F888500120F8BD2368FF
:1065F80040221A62226802F1080353E8003F43F080
:10660800800302F1080141E800300028F3D1EDE7EA
:106618000220EBE729660008716600087D6600081D
:1066280008B50346806A1B681B6813F0200317D15E
:10663800A0F85630026802F1080353E8003F23F03F
:106648008003083242E8003102680029F2D152E89A
:10665800003F43F0400342E800310029F7D108BD6C
:10666800FCF788FBFBE7704708B5806AFFF7FBFF7C
:1066780008BD7047806A38B50468D0F88830D0F80B
:106688008C50A268120606D5212B04D10023A0F84D
:106698005630FFF73CFFA3685B0606D5222D04D1D0
:1066A8000023A0F85E30FFF74DFFD0F8903043F09C
:1066B8001003C0F89030FFF7DCFF38BD08B5806ADA
:1066C8000023A0F85E30A0F85630FFF7D2FF08BDCF
:1066D800704700000368D9691A682DE9F04140F64F
:1066E8000F0631429D68044610D18E0640F197800E
:1066F80002F0200605F080573E4300F09080436F7B
:10670800002B00F08580BDE8F0411847AB4EAC483F
:106718002E401040304300F08280CF0709D5D005C5
:1067280007D501201862D4F8900040F00100C4F8A1
:1067380090008F0709D5E80707D502201862D4F81A
:10674800900040F00400C4F890004F0709D5E8070E
:1067580007D504201862D4F8900040F00200C4F86D
:1067680090000F070BD502F02000304307D0082017
:106778001862D4F8900040F00800C4F890000E05A4
:106788000AD5500108D54FF400601862D4F890304B
:1067980043F02003C4F89030D4F89030002B37D061
:1067A8008B0609D502F0200205F080552A4303D054
:1067B800636F0BB1204698472668D4F89020B368D9
:1067C80002F0280203F0400353EA0205204621D0D4
:1067D800FFF7B8FEB3685F0617D5226802F1080311
:1067E80053E8003F23F04003083242E80031002913
:1067F800F3D1D4F8800040B1724B8363FEF7E3F81D
:1068080030B1D4F88000836B7DE72046FFF731FF75
:10681800BDE8F081FFF72DFFC4F89050F8E7E06E6F
:10682800012840F08980CE0640F18680D00640F1EC
:10683800838010221A629A6851064BD5D4F88020BA
:1068480011684A6892B2002AE2D0B4F85C0090421B
:10685800DED9A4F85E200A6892062FD453E8002FE8
:1068680022F4807243E800210029F7D103F10802DD
:1068780052E8002F22F0010203F1080040E800214D
:106888000029F3D103F1080252E8002F22F0400258
:1068980003F1080040E800210029F3D12022C4F8C0
:1068A8008C20E16653E8002F22F0100243E8002113
:1068B8000029F7D1D4F88000FEF750F802232367A7
:1068C800B4F85E30B4F85C10C91A89B22046FFF7F4
:1068D800FFFE9DE7B4F85E20B4F85E00B4F85C10E3
:1068E80080B292B2002893D0891A89B200298FD039
:1068F80053E8002F22F4907243E800200028F7D1D3
:10690800314D03F1080252E8002F2A4003F108062E
:1069180046E800200028F4D12022C4F88C206067C3
:10692800E06653E8002F22F0100243E80020002818
:10693800F7D102232367C9E7CF0209D56E0207D52D
:106948004FF4801220461A62BDE8F04100F0A0BD65
:1069580008060BD502F0800005F40005284305D091
:10696800A36F002B3FF454AF2046CCE64F0611D559
:1069780056060FD553E8002F22F0400243E80021C5
:106988000029F7D12023C4F88830A1672046FCF7F6
:10699800F1F93DE70D0206D5500004D52046BDE8C3
:1069A800F04100F077BDCB017FF532AF002ABFF68A
:1069B8002FAF2046BDE8F04100F06BBD010000108C
:1069C80020010004C5660008FEFFFFEFD0F88C2008
:1069D800B0F86010222A08B5036855D15B6A826D49
:1069E8000B401370836D01338365B0F85E30013B53
:1069F8009BB2A0F85E30B0F85E309BB2002B42D15B
:106A0800026852E8003F23F4907342E800310368BB
:106A18000029F5D103F1080252E8002F22F0010203
:106A280003F1080C4CE800210029F3D12022C0F81A
:106A38008C20184A41679342016705D1C26E012A2A
:106A48000ED0FCF7A5F91EE05A681102F6D553E8F6
:106A5800002F22F0806243E800210029F7D1EDE7FA
:106A68000022C26653E8002F22F0100243E80021FA
:106A78000029F7D1DA69B0F85C10D20644BF1022B9
:106A88001A62FFF725FE08BD9A6942F008029A616A
:106A9800F9E700BF00800040D0F88C20B0F8601003
:106AA800222A08B5036852D15A6A1140826D22F829
:106AB800021B8265B0F85E20013A92B2A0F85E200F
:106AC800B0F85E2092B2002A40D153E8002F22F499
:106AD800907243E800210029F7D103F1080252E837
:106AE800002F22F0010203F1080C4CE800210029D4
:106AF800F3D12022C0F88C20174A416793420167DE
:106B080005D1C26E012A0ED0FCF742F91EE05A6880
:106B18001102F6D553E8002F22F0806243E80021E5
:106B28000029F7D1EDE70022C26653E8002F22F0D2
:106B3800100243E800210029F7D1DA69B0F85C10A7
:106B4800D20644BF10221A62FFF7C2FD08BD9A6937
:106B580042F008029A61F9E7008000402DE9F84FF9
:106B68000368B0F86060D3F81CB01F689D68D0F85F
:106B78008C20222A044640F0B980B0F8683043B12E
:106B8800DFF87491DFF874A14FF000081BF0200FB4
:106B980020D1B4F85E309BB2D3B1B4F868209A42E1
:106BA80016D9226802F1080353E8003F23F0805306
:106BB800083242E8003122680029F2D1504B63675D
:106BC80052E8003F43F0200342E800310029F7D1A2
:106BD800BDE8F88F2368A26D5B6A33401370A36D1C
:106BE8000133A365B4F85E30013B9BB2A4F85E3074
:106BF8002368D3F81CB01BF0070F2ED01BF0010F31
:106C080009D0F90507D501221A62D4F8902042F07C
:106C18000102C4F890201BF0020F09D0EA0707D53B
:106C280002221A62D4F8902042F00402C4F890209C
:106C38001BF0040F09D0E80707D504221A62D4F81C
:106C4800903043F00203C4F89030D4F8903023B168
:106C58002046FFF70EFDC4F89080B4F85E309BB272
:106C6800002B93D1226852E8003F23F4807342E856
:106C7800003123680029F5D103F1080252E8002FFA
:106C880002EA090203F1080040E800210029F3D1D3
:106C980020225345C4F88C20616721670AD05A68BE
:106CA800110207D553E8002F22F0806243E8002143
:106CB8000029F7D1E26E012A14D10022E26653E8D6
:106CC800002F22F0100243E800210029F7D1DA69E9
:106CD800B4F85C10D20644BF10221A622046FFF7AF
:106CE800F7FC53E72046FCF753F84FE79A6942F060
:106CF80008029A616CE700BFFEFFFFEF00800040CA
:106D0800D56900082DE9F84F0368B0F86060D3F83A
:106D18001CB01F689D68D0F88C20222A044640F0D9
:106D2800B780B0F8683043B1DFF87091DFF870A130
:106D38004FF000081BF0200F20D1B4F85E309BB252
:106D4800D3B1B4F868209A4216D9226802F1080330
:106D580053E8003F23F08053083242E800312268AC
:106D68000029F2D14F4B636752E8003F43F02003FC
:106D780042E800310029F7D1BDE8F88F2368A26DF9
:106D8800596A314022F8021BA265B4F85E20013A24
:106D980092B2A4F85E20D3F81CB01BF0070F2ED0D7
:106DA8001BF0010F09D0F90507D501221A62D4F8A2
:106DB800902042F00102C4F890201BF0020F09D085
:106DC800EA0707D502221A62D4F8902042F004029A
:106DD800C4F890201BF0040F09D0E80707D5042257
:106DE8001A62D4F8903043F00203C4F89030D4F813
:106DF800903023B12046FFF73CFCC4F89080B4F8EB
:106E08005E309BB2002B95D1226852E8003F23F4F4
:106E1800807342E8003123680029F5D103F10802A4
:106E280052E8002F02EA090203F1080040E80021B5
:106E38000029F3D120225345C4F88C2061672167CB
:106E48000AD05A68110207D553E8002F22F0806251
:106E580043E800210029F7D1E26E012A14D100226B
:106E6800E26653E8002F22F0100243E800210029CF
:106E7800F7D1DA69B4F85C10D20644BF10221A625E
:106E88002046FFF725FC55E72046FBF781FF51E731
:106E98009A6942F008029A616EE700BFFEFFFFEFB1
:106EA80000800040A16A000838B5044603682169DB
:106EB800A2681D68C0690A4361690A4377490243A9
:106EC80029400A431A605A68E16822F440520A438A
:106ED8005A60734AA16993421CBF226A11439A6897
:106EE80022F06E4222F430620A439A60DA6A616ADA
:106EF80022F00F020A43DA626A4A934219D14FF02C
:106F0800B043694AD3F8883003F0030343F44033AD
:106F1800934200F0B480B3F1031F24D0013A9342A6
:106F280040F0B580B0F5004F40F08F80FEF700F9D3
:106F38006EE05E4A93421CD14FF0B0435C49D3F8EF
:106F4800883003F00C0343F440228A4200F0978013
:106F580006D8002B7CD0574B9A42E3D0012026E07C
:106F6800B2F10C1FFAD1B0F5004F53D04FF40040E6
:106F780075E04B4A9342F1D14FF0B043D3F88830D3
:106F880003F44063B3F5006F18D006D85BB1B3F5CE
:106F9800806FE3D1FEF7CCF807E0B3F5406FDDD1A1
:106FA8004FF400400BE0FEF7BBFC40B900204FF067
:106FB8000113A3660023C4E91D3338BD3E48656844
:106FC8003E4B626A05EB450133F81220B0FBF2F341
:106FD8009942C3D8B3EB053FC0D800231946FAF746
:106FE80093FD090241EA10616B080002C0182A46A5
:106FF8004FF0000341F10001FAF786FD304BA0F590
:1070080040729A42AAD82368D860CFE7FEF788FC76
:107018000028CBD06168294B626A33F81220B0FB94
:10702800F2F24B0803EB42034FF6EF72B3FBF1F3B6
:10703800A3F11001914291D823F00F02216892B276
:10704800C3F342031343CB60B0E7FEF771F804E0E3
:10705800B0F5004FDAD0FEF763FC0028A6D06368CD
:10706800616A164A32F81120B0FBF2F000EB5300C7
:10707800B0FBF3F04FF6EF73A0F11002C1E7B0F5E3
:10708800004F0D48EBD1C5E7FEF75AFCC0E7B0F555
:10709800004FF9D0FEF754FCDFE700BFF369FFCFDC
:1070A8000080004000380140020003000044004016
:1070B80008000C0004000C000024F400200B010858
:1070C800FFFC0F00836ADA0710B506D50168C46AA9
:1070D8004A6822F4003222434A609C0706D50168B8
:1070E800046B4A6822F4803222434A60590706D565
:1070F8000168446B4A6822F4802222434A601A07D6
:1071080006D50168846B4A6822F4004222434A602B
:10711800DC0606D50168C46B8A6822F480522243D3
:107128008A60990606D50168046C8A6822F40052C0
:1071380022438A605A060FD50168446C4A6822F4D3
:1071480080122243B4F5801F4A6005D14A68846CD6
:1071580022F4C00222434A601B0606D50268C16CAD
:10716800536823F400230B43536010BD2DE9F84303
:10717800DDF8209005460F46164698462A68D369DA
:1071880037EA03030CBF01230023B34201D00020D8
:1071980029E0B9F1FF3FF2D0FBF796FBA0EB08001E
:1071A80048452C6802D8B9F1000F1ED154E8003FB9
:1071B80023F4D07344E80032002AF7D104F108031D
:1071C80053E8003F23F0010304F1080141E80032CD
:1071D800002AF3D12023C5F88830C5F88C30002365
:1071E80085F884300320BDE8F88323685A07C5D59D
:1071F800E3691B05C2D54FF40063236254E8003FDE
:1072080023F4D07344E80032002AF7D104F10803CC
:1072180053E8003F23F0010304F1080141E800327C
:10722800002AF3D12023C5F88830C5F88C30C5F87A
:107238009030D4E773B504460026C0F89060FBF799
:1072480043FB23681B681A07054619D423681B6883
:107258005B070AD56FF07E43009300222B464FF45C
:1072680080012046FFF782FFB0B900202023C4F830
:10727800883084F88400C4F88C30E06620670CE01D
:107288006FF07E430093324603464FF400112046C8
:10729800FFF76CFF0028D9D0032002B070BD10B5ED
:1072A800044650B3D0F888301BB980F88430FBF717
:1072B80063FC22682423C4F88830136823F0010390
:1072C80013602046FFF7F0FD012816D0A36A13B11A
:1072D8002046FFF7F7FE23685A6822F490425A6066
:1072E8009A6822F02A029A601A6842F0010220463F
:1072F8001A60BDE81040FFF79DBF012010BD0000D7
:1073080030B581658168A0F85C200023B1F5805F05
:10731800A0F85E20436735D10369002B40F2FF13C4
:1073280018BFFF23A0F860300023C0F89030222354
:10733800C0F88C30016801F1080353E8003F43F0BE
:107348000103083141E800340368002CF2D1456E8E
:1073580084680169B5F1005F32D1B0F86850954290
:107368002ED8B4F5805F244A03D1244C002908BFE5
:1073780022464267B1B153E8002F42F4807243E8D5
:107388000021F7E729B90369002B14BF7F23FF23E6
:10739800C8E7B1F1805FC5D10369002B14BF3F2353
:1073A8007F23BFE703F1080252E8002F42F0805222
:1073B80003F1080040E800210029F3D1002030BD86
:1073C800B4F5805F0E4A03D10E4C002908BF22464F
:1073D800426741B153E8002F42F4907243E800211C
:1073E8000029F7D1EAE753E8002F42F0200243E8EA
:1073F80000210029F7D1E1E7656B00080D6D000851
:10740800D5690008A16A0008D0F88C30202B30B468
:1074180015D1B9B1B2B100230468C3660A4B9C42C6
:107428000AD063681B0207D554E8003F43F0806325
:1074380044E80035002DF7D130BCFFF761BF0220CA
:1074480030BC70470120FBE700800040436E30B538
:107458002BB90123A0F86A30A0F8683030BD036862
:10746800094D9A689968094C490FC2F342626B5CEE
:10747800615CDB00B3FBF1F3A0F86A30AB5CA25CA3
:10748800DB00B3FBF2F3E7E7400B0108380B010818
:107498007047704770471FB504AB03E9060090F8C2
:1074A8008430012B04463AD0012380F88430242309
:1074B800C0F8883003681A6822F001021A609A68D6
:1074C80022F440120A439A6071B95A68BDF80C0058
:1074D8009DF80E1022F0100202435A605A6822F0FA
:1074E8007F4242EA01625A601A6842F001021A6059
:1074F800FBF7EAF96FF07E42034600924FF48001F1
:1075080000222046FFF732FE38B92023C4F888301D
:10751800002384F8843004B010BD0320F8E702206B
:10752800F9E790F88430012B0FD0012380F88430DC
:10753800016851E8002F42F0020241E80023002BC5
:10754800F6D180F88430184670470220704710B58D
:1075580090F88430012B044617D02423C0F88830D3
:1075680003681A68196821F00101196042F0005295
:107578004FF0005141661A60FFF768FF2023C0F8FA
:107588008830002084F8840010BD0220FCE770B524
:1075980090F88430012B044617D005682423C0F8DE
:1075A80088302E682B6823F001032B60AB6823F02A
:1075B80060431943A960FFF749FF20232E60C0F8F4
:1075C8008830002084F8840070BD0220FCE770B584
:1075D80090F88430012B044617D005682423C0F89E
:1075E80088302E682B6823F001032B60AB6823F0EA
:1075F80060631943A960FFF729FF20232E60C0F8B4
:107608008830002084F8840070BD0220FCE7000068
:1076180038B5084D052455F8043B2BB9013C14F046
:10762800FF04F8D1204638BDDB6898470028F5D01C
:10763800F9E700BFDC060020034BD870034B1B683A
:107648001B6C03B118477047C4060020C006002011
:10765800034B1874034B1B685B6C03B118477047E6
:10766800C4060020C0060020F0B5314D314B95F915
:107678000420314E91B00C46012795F905108DF87C
:10768800047002288DF809208DF80A1010D18DF8A1
:107698000800D8711C7202F063FD337803B114B18D
:1076A80001A803F0C1F9254B059A1A6011B0F0BD85
:1076B80059714FF480711A71D9801C7233788DF822
:1076C800087053BB1F2306A88DF81C208DF81830AE
:1076D80002F024FF20238DF8183006A82B798DF8A6
:1076E8001C3002F01BFF22238DF8183006A86B7996
:1076F8008DF81C3002F012FF21238DF8183006A8EF
:107708006B798DF81C3002F009FF29238DF81830A9
:1077180006A80B4B079302F001FF02F021FD01239D
:1077280006A88DF818308DF81C3002F0F7FEB4E783
:10773800C4060020F0000020A005002094060020C8
:10774800000400017FB5092301A88DF8043003F077
:107758006BF90038044B059A1A6018BF01204042A3
:1077680007B05DF804FB00BF9406002070B504461E
:107778000B46144962784A700020A2780A72087091
:107788001A884A729A788A72DB780B746368CB60BD
:107798000D4B1B68DA6A2AB1237803F0FB030A2B26
:1077A80000D09047094E002556F8043B1BB15B6A90
:1077B8000BB1204698470135EBB2052B6DB2F3D1DA
:1077C80070BD00BFC0000020C0060020DC060020FD
:1077D80070B5044611480123037063784370A37899
:1077E8008372E368C360E378037623694376237979
:1077F80043720B4B1B689B6A03B19847094E0025DF
:1078080056F8043B1BB19B690BB1204698470135DC
:10781800EBB2052B6DB2F3D170BD00BFD4000020D0
:10782800C0060020DC060020014B1868704700BF26
:107838009406002000B58BB0012368468DF800300F
:1078480002F046FD38B99DF80400003818BF012041
:107858000BB05DF804FB0020FAE7000008B501F062
:1078680037FE40B9FFF7E6FF012806D0054B197A25
:10787800D879FFF7F9FE012008BDBDE80840FFF7F9
:10788800C7BE00BFF00000202DE9F04186B00546D4
:107898000E46174601F01CFE002873D101F030FE99
:1078A800044640B9FFF7C6FF01280AD03D4B197AB4
:1078B800D879FFF7D9FE6FF00204204606B0BDE87C
:1078C800F081DFF8E48088F80860003E18BF0126E0
:1078D8008DF80460354E687833798DF81230694632
:1078E80002F094FC00283FD08DF804400394ADF8D2
:1078F80010406FF0060495E803002D4B83E8030061
:10790800337988F80A30394601A803F091F9294BF0
:10791800059A1A6011283FD801A353F820F000BF38
:10792800937900088D790008A1790008A1790008E9
:10793800A1790008A1790008A1790008BF7800089A
:10794800A1790008A1790008A179000887790008C1
:10795800A1790008A17900088D7900088D790008BF
:107968008D790008A77900082B788DF808306B7896
:10797800ADF810306B6803934FF0FF34BBE76FF03E
:1079880005049AE76FF0010497E70B4B00221A7081
:10799800E31D18BF144690E74FF0FF348DE76FF0F2
:1079A80004048AE7F0000020D4000020C406002068
:1079B800E4000020940600209306002037B501F06B
:1079C800A9FD134D052455F8043B4BB11A693AB18A
:1079D8009B682BB1984718B155F8043C1B69984728
:1079E800013C14F0FF04EED1FFF712FE68B9094D0F
:1079F8002B7853B1084BADF80040D9780194224652
:107A08006846FFF741FF00B92C7003B030BD00BFD6
:107A1800DC06002093060020C406002030B58BB099
:107A2800044601F055FD0546002835D1FFF702FF51
:107A3800012834D168468DF8005002F049FC40BB5B
:107A48009DF80430A34204D0012C22D0022C12D07D
:107A580014B100200BB030BD002BFAD068468DF869
:107A6800044002F05BFDA0B90E4B1B681B6B002B9A
:107A7800EFD09847EDE763B968468DF8044002F007
:107A88004DFD30B9074B1B681B6B002BE1D020461E
:107A9800EFE74FF0FF30DDE76FF00100DAE76FF056
:107AA8000200D7E7C006002010B504468AB018B90E
:107AB8004FF0FF300AB010BD002368468DF8003043
:107AC80002F006FC0028F3D19DF804302370F1E79A
:107AD8007FB500220B4620498DF8072001220A7045
:107AE80042784A700446002A33D102790A721A8809
:107AF8004A729A788A72DB780B740369CB60C37810
:107B0800164D8DF80830037B8DF809308368039390
:107B18002B68DB6A0BB102A898472B689B6B13B1E3
:107B2800227E02B198470E4E052556F8043B1BB13C
:107B3800DB690BB120469847013D15F0FF05F4D1EC
:107B48000DF10700FFF7B0FF637913B1054B012270
:107B58001A7004B070BD00BFC0000020C00600202D
:107B6800DC0600209306002010B504468AB018B938
:107B78004FF0FF300AB010BD202368468DF8003062
:107B880002F0A6FB0028F3D1024A9DF904302370C5
:107B98001371EFE7C406002000B58BB023230190D2
:107BA80068468DF8003002F0B9FC003818BF012093
:107BB80040420BB05DF804FB70B5654C01468EB0D1
:107BC8001822204606F0C0F8624B00221A70FCF713
:107BD8001FF823784068012202FA03F1014004D11A
:107BE8005D4B084608F09CF8FEE75C495C481A467D
:107BF80002F0F8F818B14FF0FF300EB070BD27232F
:107C080004A88DF8103002F089FC564E564D002815
:107C180070D1012333702B68DB690BB100209847C2
:107C2800272304A88DF8103002F052FB059B93F827
:107C38004820227093F8182193F81A316270A370C3
:107C4800464BD3E9020105F06FFF05460028D2D163
:107C5800464E062304A88DF8103002F039FB059B28
:107C6800736104A802F05AFC022304A88DF81030AE
:107C7800059602F02DFB0836032304A88DF8103072
:107C8800059602F025FB0F2606F014F8012304A838
:107C98008DF814308DF8106002F040FC10230DEBC5
:107CA80003008DF810308DF8145002F037FC0423CF
:107CB8008DF8103004A8A3788DF8143002F02EFC4B
:107CC8003A238DF8103004A86369059302F026FC66
:107CD80002A920788DF8086004F09CF8003818BFD5
:107CE8000120E0711420FFF757FFE07903F062F9F3
:107CF800284682E728238DF810302B681B6943B18A
:107D080004A802F0E5FA2B6805981B6940F2C451F3
:107D18009847272304A88DF8103002F0FFFB50B9CC
:107D2800012304A88DF8103002F0D2FA9DF814301F
:107D3800002B7FF46EAF3378002B7FF46CAF0522F5
:107D480004A88DF81020059302F0E8FB78E700BF3F
:107D5800C406002093060020480B0108980600205E
:107D6800B0060020A0050020C00600200007002063
:107D780037B500230D4601930446D0B900F0A8FB9F
:107D88000190019BD3B10F4A42F824300E4A9A62FF
:107D98000E4A1268916B1963916C596392690C4988
:107DA800D9625A6128465B680A49F222984700203E
:107DB80006E001A900F092FB0028E2D04FF0FF3066
:107DC80003B030BDDC06002071760008C006002034
:107DD8004D770008A1050020194B07B51860194B0D
:107DE800194A1A60194A5A60194A9A60194ADA6097
:107DF800194B02681A6042685A6082689A60C268C1
:107E0800DA60164A1A6182695A61154BC26B5A6068
:107E1800144A019119609A601946134ADA600020E1
:107E2800FFF7A6FF48B901A800F056FB003818BFB5
:107E38000120404203B05DF804FB4FF0FF30F9E742
:107E4800C0060020B0060020D9770008D97A0008BB
:107E5800ED7E00087577000898060020CDBD000863
:107E6800F0060020417600085976000849B118B19B
:107E7800012804D000207047034B0B60FAE7034B3E
:107E8800FBE74FF0FF3070470004000101000102DA
:107E980008B503F0ABF8002814BF6FF0010000200C
:107EA80008BD08B502F084F9002814BF6FF001007E
:107EB800002008BD10B504468AB018B94FF0FF304D
:107EC8000AB010BD212368468DF8003002F000FA90
:107ED8000028F3D1024A9DF9043023705371EFE76B
:107EE800C40600202DE9F0412F4D304F00232B70A0
:107EF80043786B703B689B6A8AB004460BB128468E
:107F08009847DFF8AC80002658F8043B1BB11B6A81
:107F18000BB1204698470136F3B2052B76B2F3D160
:107F28002378052B2FD00B2B35D0012B25D1214CB5
:107F3800062368468DF8003002F0CAF90199E07905
:107F480005F038FE10B91C4B019A5A611B48FFF71F
:107F58000BFE1B48FFF7AEFF6B788BB9A371194B6B
:107F68005878FFF75BFD3B685B6A0BB1114898478F
:107F78006B7813B9E07905F0AFFE0AB0BDE8F0817F
:107F8800FF23A371EFE7104B01225A74227A9A74E7
:107F9800627ADA74F1E76378002BEED00AB0BDE8B4
:107FA800F041FFF7CFBB00BFD4000020C00600207F
:107FB800DC060020F000002000070020F40000206C
:107FC800F5000020C4060020C000002030B58BB0AA
:107FD800FFF767FF0446F0B903F0FCFE831C1DD0D1
:107FE800F8B9134D2B685B69DBB1272368468DF818
:107FF800003002F06DF92B6801985B694FF4B961A4
:10800800984703F0F9FE78B92CB9094B1B68DB696E
:108018000BB10120984720460BB030BD6FF0070424
:10802800EFE74FF0FF34ECE74FF0FF34F3E700BF22
:10803800C0060020014B1878704700BF34070020A5
:10804800014B5878704700BF340700207047000084
:10805800044B9A7A0AB101225A70034B5B6903B147
:108068001847704734070020FC00002073B5224CE5
:108078006378002B33D008F03BF966680546FFF7B4
:10808800D3FB0644AE4214D2A37A93B1E0228DF812
:1080980000208DF80130217AE368019301226846B7
:1080A800FFF7F2FB08B1073010D100236370A37209
:1080B800656094F83430EBB1002384F834300F4B0A
:1080C8005B6BBBB102B0BDE87040184740F2DC51B1
:1080D8000B4808F0D9F90A4808F09CF9E8E794F841
:1080E8003520002AE5D094F8360084F83530FFF7BB
:1080F80095FCDEE702B070BD34070020FC000020CC
:108108001807002037B5104D104CC8B1C1B16272C4
:10811800012300222860E16023700D480D4B009276
:108128004FF0FF3108F0CAF800250B4825822022BD
:10813800294605F01DFE6570A574A58603B030BDFF
:1081480000232B602370EFE730070020340700205E
:108158001807002059800008480700202DE9F0473B
:108168008E4C23788CB0002B56D0C2780AB9837B0A
:1081780013B1238A01332382437B002B4CD0E02A9E
:108188004AD10023A372876897F80080B8F1220FBC
:1081980027D8B8F1220F30D8DFE818F04100FB00EB
:1081A80052005A0061006E0075008E009D00B400F8
:1081B800C7002F002F002F002F002F002F002F00A7
:1081C8002F002F002F002F002F002F002F002F002F
:1081D8002F002F002F002F002F002F00C900D000E4
:1081E800D400B8F17E0F00F0CC80B8F17F0F00F01A
:1081F800DF80B8F17D0F00F0AB80A57A002D00F08C
:108208005B81674C637A3BB94FF47A71204608F07A
:108218003BF9204608F0FEF80CB0BDE8F087E368AB
:1082280001220021A2721970A37AE1689818A0723D
:108238000620C854A37AE1689818A072CA54DCE7EB
:10824800584B9B6A002BD8D0012102209847D4E7CD
:108258007B7884F83630012384F83530CDE7042361
:108268008DF804307B78003B18BF012301A88DF8F6
:10827800083002F053F9C0E77878003818BF0120B9
:1082880002F098FEB9E7484E0FCE01AD0FC50FCEEC
:108298000FC596E8070085E807007B780A2BACD85D
:1082A800424A12685268002AA7D00CA901EB83033E
:1082B80053F82C0C9047A0E77878431E012B9CD8E4
:1082C8003A4B01381B6818BF012020729B68002BAD
:1082D80093D0984791E7E26801230821A3721170AF
:1082E800627A057BA17AAA4228BF2A46934284D2A1
:1082F80085685A1CEB5CE56801334E1CA6726B540A
:10830800D3B2EDE7E3680122A27209221A70A37AB8
:10831800E268218A581CA072D154A27A238AE168A3
:108328001B0A501CA0728B5467E7238265E705235C
:108338008DF8043001A802F077FB5EE7194BDB6A81
:1083480098475AE7194B78781B686075DB68BEE771
:10835800037B072B7FF451AF06238DF80430B7F861
:108368000130ADF808307B793A791B0443EA0223DF
:10837800FA781343642253430393BB798DF8103082
:10838800D8E73B2201A88DF804208DF8083002F0C8
:10839800C5F8012384F834302FE700BF34070020E4
:1083A80018070020FC0000205C09010830070020A5
:1083B8002A2301A88DF8043001F08AFF94F80A9066
:1083C800E6689DF808009DF809509DF80A709DF828
:1083D8000BC09DF80D309DF80E209DF80F109DF8EC
:1083E8000CE009F1010A84F80AA006F80980354E64
:1083F80094F80A903668D4F80C8009F1010A84F8D8
:108408000AA096F803A008F809A094F80A90D4F8EE
:108418000C8009F1010A84F80AA096F802A008F86D
:1084280009A094F80A90D4F80C8009F1010A84F89C
:108438000AA096F801A008F809A094F80A9009F192
:10844800010A84F80AA096F80080E66806F8098010
:1084580094F80A80E66808F1010984F80A9006F899
:1084680008C094F80AC0E6680CF1010884F80A808C
:1084780006F80C70A77AE66807F1010C84F80AC0C0
:10848800F555A57AE6686F1CA7727055A07AE5685D
:10849800461CA6722954A17AE0684D1CA572425464
:1084A800A27AE168501CA0728B54A37AE268591C26
:1084B800A17202F803E0A0E6034807F05DFF6570CB
:1084C800AAE600BF30070020180700207047000008
:1084D80000487047FC000020002070474FF0FF3034
:1084E80070470000044B054A93F81831022B18BF57
:1084F800062382F890347047D80D00209C13002082
:10850800034BD3F8483313B15B6903B1184770477D
:108518009C130020034A137843F004031370FFF7F9
:10852800EFBF00BF800700201FB50A4B8DF8090078
:1085380093F87C208DF80A2093F88C2093F8480053
:108548000D3202A98DF8082003F064FCC0B205B012
:108558005DF804FBD80D002008B5074807F00CFFAC
:10856800064B93F81A2412B1012283F81924BDE8A6
:108578000840FFF7C5BF00BF9C1700209C130020D0
:1085880010B50C4CD4F8403343F08003C4F84033A2
:1085980094F81A3413B10020FFF7DEFF94F89134F1
:1085A80023F0120343F0120384F89134BDE810401D
:1085B800FFF798BF9C1300202DE9F041DFF8AC804D
:1085C80098F81831022B06460D4602D0284BDB6A74
:1085D800984702F0A6FD044628B1022002F097FD54
:1085E800002002F099FD98F81831012B17D102F0FC
:1085F8009AFD074630B1002002F08AFD002002F003
:108608008CFD3C4602F091FD48B1002002F081FD4E
:10861800002002F083FDBDE8F041FFF763BF002CA6
:10862800F9D1144C94F8902494F81A34BAB90BB1CF
:1086380084F84164304602F017FFD8F82C0007F0A0
:1086480061FED4F8B4339842E5D30B4807F094FEA2
:1086580094F8913443F0100384F89134DBE70BB1BC
:1086680084F84154284602F0FFFEF1E7D80D0020B7
:10867800C41201089C13002034170020074A10B5C3
:10868800137843F002031370FFF73AFFBDE8104078
:10869800034B01220021022007F042BB8007002083
:1086A800910B0108074A10B5137843F008031370BB
:1086B800FFF726FFBDE81040034B012200210220EE
:1086C80007F02EBB80070020A10B01082DE9F0411F
:1086D8000F4616461D46804607F00AFE0B4A0C4C0C
:1086E8001378278123F0110343F01103C4E900082C
:1086F800137066812573FFF703FFBDE8F041054B52
:1087080001220021022007F00BBB00BF80070020D8
:108718006C070020B10B010813B507F0E9FD0D4BFC
:108728006C461860204607F037FD94E803000A4AB3
:108738000A4B83E80300137843F020031370FFF714
:10874800DFFE074B01220021022002B0BDE81040E5
:1087580007F0E6BA7C07002080070020D416002026
:10876800BE0B01082DE9F04192B0064602F0D9FC93
:10877800002840F05881AD4D95F81831012B09D0EB
:108788002B6BAB4C93B194F80431BBB1042B6FD075
:10879800032003E002F0C7FC18B10F2012B0BDE8B7
:1087A800F08102F0C2FC0028EAD0F6E7B5F82031E3
:1087B800D4F81C24013B53432B63E4E79D4803F0A2
:1087C80060FA002840F0128194F80C3123802B6B5A
:1087D8000C930DF1180895F839308DF8383040466B
:1087E80095F81C318DF83A3007F0FCFCD5F82831A3
:1087F800009302AF98E80600D5F82431384607F010
:1088080088FC97E803000FAB83E80300EB6A0D933D
:1088180000238DF844302388ADF8463095F8303180
:1088280001228DF839201BB98DF844208DF8393094
:10883800814B0093814B95F84800A3F179020CA96C
:1088480003F05DFBC0B10B28A8D1D4F8941499B1FA
:10885800002EA3D0D4F84033794843F02003C4F85D
:10886800403307F011FE764807F0D4FD002095E765
:10887800704803F03AFAA4E795F8487095F969301A
:1088880095F9392095F87D106E4E384603F044FB73
:10889800009641B2EB6C95F850203846183603F034
:1088A800DFFA0096EB6C95F8502095F9701095F862
:1088B800480003F0D5FAD4F8C413AB6DD4F8DC2320
:1088C8000B44C4F8B033EB6D1344C4F8B43394F8D4
:1088D8000431042B07D02B6E0B44C4F8B0336B6EF5
:1088E8001344C4F8B4330023089395F83031002BAF
:1088F80040D100238DF8133095F839308DF82130A8
:1089080095F838308DF82230D5F880300993D5F8AD
:1089180084300A932388ADF82C3095F8303194F8D8
:108928001B648DF82E3095F84800474B8DF8206071
:108938000DF1130208A903F0A7FA012384F84134C2
:1089480095F8393084F842349DF8133084F843346C
:10895800D4F81C34C4F85064C4F84834C4F8583403
:1089680002F0E5FBC8B1D4F81C0402F0F2FBA0B198
:10897800102013E708A802F0A7FC60B995F93900A0
:1089880094F837629DF82070FFF7CEFD3E44B04260
:10899800AFD2082002E7132000E795F81831012B21
:1089A80001D102F0D8FB02F0C5FB0023059394F82F
:1089B800043195F9395094F81B649BB1042B7FF46A
:1089C800E7AE05A802F0B4FE58BB94F8183413B10A
:1089D800059B013B0593174B05983246E9B202F017
:1089E8000DFF02E0134802F0DDFE08B11120D5E6C4
:1089F800D4F8403394F80C11218043F00203C4F8F2
:108A0800403394F8183411480133DBB284F8183431
:108A180084F845340E4B00259B6AC4F8985498474F
:108A280024E71220BAE60E20B8E600BFD80D0020D1
:108A38009C130020A4140020080E002030180020E9
:108A48000417002054170020B81700209E13002098
:108A5800C412010873B5134D134E0096EB6C95F8CC
:108A6800502095F9781095F8480003F0F9F995F831
:108A78003031337595F8480040F2012306F13C0285
:108A88003146738203F0F8F950B196F83C3086F815
:108A98008230064B00205B6B9847F37C86F8A83041
:108AA80002B070BDD80D002084170020C412010840
:108AB800F8B5324C94F81831012B05460ED0022B2C
:108AC8004ED0002B57D138B9D4E91B0104F17403F7
:108AD80083E803000020F8BD012806D102F02CFB32
:108AE8000028F8D184F81851F5E7022843D1244E1C
:108AF80084F8180106F5747CBCE80F0006F57A774F
:108B08000FC79CE8030094F8E92094F8003187E83F
:108B1800030086F8FB53D2B1022B18D1D4F80431E4
:108B28006367C6F8EC3394F87D3094F8082186F82A
:108B3800F83394F88C3084F8782086F8F93396F86E
:108B48001B2486F8E82340F20133A6F8FA33002301
:108B580086F81A340B4BDB6A9847FFF77BFFB9E7B7
:108B680048B9074B84F81801062283F89024054B6E
:108B7800DB6A9847AEE70320ADE700BFD80D0020B9
:108B88009C130020C4120108F0B5504C504EB4F8A4
:108B9800DC202287D4E92D0194F8B12084F86920DB
:108BA80004F16C0282E80300D4E92F0104F1740295
:108BB80082E80300B4F8C420A4F87C2091B0D4F86B
:108BC800CC20D4F8C810C4F884200025D4F8D020CC
:108BD800C4F888200123A4F82031C4F8801084F850
:108BE8003051A56284F81B5184F83A5084F81D511D
:108BF80084F81E51C4F83451C6F89854A6F818548D
:108C080086F81A54A4F838518DF8183004F5097309
:108C1800039304F50A7394F84800049303A92D4BB1
:108C280084F84551C4E94F55A4F84651059303F01B
:108C3800FFF8E36EC6F8D43394F87D3086F8E03355
:108C480094F88C3086F8E1334FF48073A6F8E23359
:108C580086F8D05394F8303186F8E43306F5747703
:108C68000FCF06F57A740FC497E8030040F201238A
:108C780084E80300A6F8FA33D6F8483386F81B547C
:108C8800CDE901551BB15A685B6901920293124BF9
:108C98000793A3F148020892A3F1140209920F4A1C
:108CA8000B9229330A93A2F19C030C93A2F1980327
:108CB8000D93131D0E9301A902F14C0307A802F5A9
:108CC80099620F9302F022FA11B0F0BDD80D00207E
:108CD8009C1300208407002004180020BC0E0020EC
:108CE800F8B50D4F0D4E0C4607F046FB3B6B984709
:108CF8000B4A96F84800214603F0BEF850B1094DDA
:108D0800706D95F8243485F86A347B6B9847E37C5A
:108D180085F89034F8BD00BFC4120108D80D0020B2
:108D2800C01700209C1300200F4890F81B3480F8CF
:108D3800B8330E4B93F8692080F8BB2393F87D2055
:108D480080F8C82393F88C2080F8C92393F8303131
:108D580080F8CC330022A0F8CA2300F56E7100F524
:108D68006070FFF7BDBF00BF9C130020D80D002026
:108D7800114890F89034EBB190F81B3480F8D03358
:108D88000E4BDA6EC0F8D42393F87D2080F8E023E8
:108D980093F88C2080F8E12393F8303180F8E4339D
:108DA8004FF48072A0F8E22300F5747100F5667044
:108DB800FFF796BF704700BF9C130020D80D002016
:108DC80070B5344C2421204604F0D4FF636A9842DD
:108DD80018BF60624FF01C012F4814BF0125002501
:108DE80004F0C8FF636C984218BF60644FF4807148
:108DF8002A4818BF45F0020504F0BCFFD4F84831F2
:108E0800984218BFC4F848014FF0D401244818BF4D
:108E180045F0040504F0AEFFD4F82032984218BF9C
:108E2800C4F820024FF000011E4818BF45F008059D
:108E380004F0A0FFD4F82432984218BFC4F82402E2
:108E48004FF46071184818BF45F0100504F092FF00
:108E5800D4F8A835984218BFC4F8A8054FF01401F3
:108E6800124818BF45F0200504F084FFD4F8C03537
:108E780098420F4B18BFC4F8C005D3F8483318BF41
:108E880045F040052BB11B691BB12846BDE8704071
:108E9800184770BDD80D0020000E0020200E0020BD
:108EA800240F0020FC0F0020001000208413002055
:108EB8009C1300202DE9F04F8FB04FF00009012BD3
:108EC80006460F4690468DF80D90ADF8109002D8E2
:108ED8004C46BC4202D30FB0BDE8F08F305D02F0C3
:108EE80033FA2044B842F6DC335D651C023BEDB230
:108EF800112BF0D801A252F823F000BF4D8F0008C3
:108F0800778F0008759000089D9000081B91000855
:108F180041910008A7910008CF91000855920008D8
:108F2800DF8E0008DF8E0008A9920008DF8E000897
:108F3800DF8E00085193000879930008B193000868
:108F4800E5930008052002F0A7FA70B1052100207A
:108F580002F068FA725DBA4BE51C0234E4B283F899
:108F68005C24325D83F85D24EDB22C46B1E7002322
:108F78008DF80E308DF80F308DF814308DF81830CC
:108F8800B9F1000F6DD1AF4C4FF0050994F87C2072
:108F98008DF831206B1E94F839208DF83320334436
:108FA80094F838200B938DF8342094F81A3194F8FB
:108FB80068208DF83520D4F82C218DF832300A92AB
:108FC80073B37B1C5B1BDBB28DF8303006AB0193AF
:108FD80005AB009394F848000DF10F030DF10E0254
:108FE8000AA902F05DFF8DF80D0000F007000728C0
:108FF80013D194F939209DF90E3084F839309A420A
:109008009DF80F3084F83830B8BF01229DF814302D
:10901800B8BF84F81D2184F868304FF0000A09E0D1
:109028000523D1E701220DF10D01032002F0A4F878
:109038000AF1010A5FFA8AF29DF81830B3FBF9F1D8
:109048009142EFD82B44DDB26B1EDBB29F420BD9A5
:10905800F25C032A9AD0AF4288BF1D464FF001093F
:1090680083E70534E5B2F9E71D46F7E7735D75490F
:1090780003F00F03012281F81B31023402FA03F3D3
:10908800A1F82031E4B2002204A9042002F074F807
:1090980025466AE707238DF80D30735DC3F3021286
:1090A80003F00F038DF82830E31CDBB28DF829207C
:1090B800F25C231DDBB2651DF35C0234E4B21B04D1
:1090C80043EA0223325D5F4C13436422534394F80E
:1090D80048000B930AA902F0F2FE00F00703072BE1
:1090E800EDB28DF80D000CD19DF8283084F8703061
:1090F80084F878300B9BE36663679DF8293084F821
:1091080069308DF81000012204A9052002F034F816
:109118002BE74B4BD3F8483363B11B6853B19847DF
:1091280008F03F038DF810008DF81130022204A9D1
:109138000620EBE7FF20F3E703238DF80D30735D7E
:109148008DF81C300AAB0693E31CDBB2A51DF25C5C
:10915800231DDBB206A9F35C1B0443EA0223A21C0D
:10916800D2B20534B25C134364225343E4B20A9387
:1091780000230B93335D8DF83030324B93F8480061
:1091880002F0A3FEC3B20028EDB28DF80D30FFF651
:10919800ECAE8DF81030012204A90720B6E7735D04
:1091A80003F00F03012B4FF47A7238BF01235343A6
:1091B800244A0234936503F57A73D365E4B2002236
:1091C80004A9082062E7735D1E4DC3F340128DF8B1
:1091D800152095F84800C3F3001205A903F00F0302
:1091E8008DF814208DF8163002F075FE0234013027
:1091F800E4B23FF44DAFBDF81430134AA5F87C3003
:109208009DF816309DF814A0D05CF8F7FFFB0223F8
:10921800C5F880000AA995F848008DF828308DF81F
:109228002AA002F0F7FD95F93930069040B298422D
:10923800B8BF184685F83900002204A9092025E797
:109248009C130020D80D0020CB0B010803238DF8B8
:109258000D30735D8DF82830E31CDBB2651DF25CC0
:10926800231DDBB20234F35CE4B21B0443EA02239D
:10927800325D1343642253430B93644B0AA993F85A
:10928800480002F02EFEC3B20028EDB28DF80D3072
:10929800FFF66BAE8DF81030012204A90A2035E7DD
:1092A800092002F0F9F8DFF868B1002849D009214F
:1092B800002002F0B7F80023ADF81E30A31CDBB283
:1092C800F25CE31CDBB216F803A0735D4FEA0A4AAE
:1092D8004AEA022A4AEA030A231DDBB2A51D05341D
:1092E800F35CE4B24AEA036A335D4FF47A7253439B
:1092F8000AAC1B122046ADF81C3006F04DFF454B5A
:1093080053440693DBF83C3300930DF1180A9AE8AE
:109318000600DBF8383308A806F0FBFE099B00932B
:1093280094E80600089B504606F0D8FE9AE8030029
:1093380006F00AFF01F00AFF0123EDB28BF838347A
:1093480013E68BF8380410E60C2002F0A5F8002884
:109358003FF40BAE0C21002002F064F82C4B93F87C
:109368009034043B012B7FF600AE01F0EBFEFCE5E8
:10937800A31CDBB2725DF15CE31CDBB2651DF35C20
:109388000434E4B21B04305D43EA0123134364212F
:10939800594300F00F0001F0D6FEEDB28DF8100031
:1093A800012204A91120B1E60D2002F075F8002869
:1093B8003FF4DBAD0D21002002F034F8A31CDBB232
:1093C800154AF05C735D1268251D0334E4B243EA64
:1093D8000020315DEDB201F0B8FEC6E5725DA31C58
:1093E800251D0334DBB2E4B2F15C335D1B0443EAB0
:1093F800012313436420584301F0A9FEEDB28DF810
:109408001000012204A9132080E600BFD80D002017
:109418009C130020803DD5126C0700200E4B93F85A
:109428009124920703D593F88F24012A08D90B4970
:1094380091F81A2122B18A6A501C18BF01328A6237
:109448000022A3F8182483F81A24D3F8402322F022
:109458000202C3F8402370479C130020D80D002057
:1094680070B5184C1848194D06F086FFD4F84033EB
:10947800D4F89804D5F8906023F02003C4F840335A
:1094880038B106F03FFF864203D2002385F83A3010
:1094980070BD0120FFF766F90028F9D00B28F7D036
:1094A80095F8393084F84234092094F8183484F84F
:1094B800453484F8410401F0D7FFBDE87040FFF758
:1094C800ADBF00BF9C13002004170020D80D00205A
:1094D800094BD3F84023012A0AD008490978C9075B
:1094E80008D43AB993F89204013818BF012070479C
:1094F80000207047012070479C130020800700203F
:10950800034BD3F84003431E58425841704700BFED
:109518009C1300202DE9F04FA9B0EFF3108272B62A
:10952800DFF8F0B20021DBF80030CBF8001082F34E
:109538001088B94C002B00F0E180DAB29B06039248
:1095480064D5B64D95F81831022B02D0B44BDB6ABE
:109558009847EFF3108872B6B24F06F0C9FE3E681E
:10956800D4F8B013361A3144AF4806F08DFFAE4830
:1095780006F050FFD4F8B413AC48314406F084FF29
:10958800AA4806F047FF88F3108894F81A34002B8D
:1095980000F06B81152312A995F848008DF8483022
:1095A80002F038FCD4F8B4130F900144A04806F038
:1095B8006BFF9F4806F02EFF3B6894F81B24EB6274
:1095C8000DAF38468DF870201D9306F00BFED5F8C8
:1095D8002831009306AE97E80600D5F824313046C6
:1095E80006F097FD96E803001FAB83E80300D4F864
:1095F8001C341E9395F8303195F84800003B18BF8D
:1096080001231CA98DF8713002F00DFC039BDF06C5
:1096180048D5824DDFF81CA2D5F8E42004929BF8C7
:109628000020BAF90A809AF90C90A4F88C840023D7
:1096380063F300020A9384F84434A4F8223484F8CB
:109648002534C4F82834A4F82C3484F82E34C4F80B
:10965800303484F82034C4F8343484F83834C4F806
:109668003C346F4B8BF8002094F89024DB6A84F824
:109678008E9484F88F24DAF80470BAF80860984752
:1096880094F88F3413B9694806F076FE31463846A7
:1096980001F045FD8346002800F0EA80A4F87E84A6
:1096A80084F88094039B19071AD55C4B93F81831FA
:1096B800022B02D05A4BDB6A98470220FEF712FFB2
:1096C80084F8410401F0D0FE94F81A3413B1012350
:1096D80084F8193494F8913443F0100384F89134E1
:1096E800039B5A0703D506210520FEF765FF039B58
:1096F8009B0703D504210320FEF75EFF01F02DFD33
:1097080094F89124D7065FD5002384F89234D4F8CE
:1097180040331E0644BF23F08203C4F8403312F0DE
:10972800050F00F0FB820B2001F0B6FE002800F0C8
:10973800F58294F89134DD0700F1F082580740F182
:109748000783D4F8403323F00203C4F84033D4F835
:10975800402382BB94F8915415F001011EBF2B469B
:1097680062F3000384F8913494F891345E0744BF9F
:109778006FF3820384F89134012384F8923421B181
:10978800D4F844332C481B6898476D070BD52B48F1
:1097980001F08EFE01F0BCFE28B194F8913443F03C
:1097A800040384F8913401F0C6FC94F891346FF303
:1097B800041384F89134012384F8923494F8913492
:1097C80043F0200384F8913494F8913418070AD5AB
:1097D8006FF3C3031A4984F89134D4F84433A1F1E0
:1097E8002400DB68984794F8913499070AD56FF3F9
:1097F8004103134984F89134D4F84433A1F16C003F
:109808005B68984794F89034022B1BD1FFF722F934
:1098180018E000BF800700209C130020D80D00200E
:10982800C41201087C0700201C17002034170020F0
:109838009C1700206C070020DC170020F017002080
:109848002818002094F891349A0640F1C4826FF3E6
:10985800451384F89134D4F84033002B40F0BB8290
:1098680029B0BDE8F04FFFF7ABBA84F84134A3E65E
:1098780095F81831012B0CD101F055FC804668B1E0
:10988800584601F045FC584601F047FC042384F88B
:109898008F347EB9012384F821344FE101F045FC6F
:1098A8000028F6D0404601F034FC404601F036FC72
:1098B8000523ECE73B7805935B09013B062B00F297
:1098C8001782DFE813F007001502950015029200D1
:1098D80015020602102EDDD995F830311297F6B22E
:1098E8008DF84C60002BD5D11CA804F055F912AAAC
:1098F8001CA9FF2002F09EF89DF85830C3F303031B
:1099080007468DF82C3095F8480095F87D308DF88D
:109918002D3007220BA902F090FA002F5DD1002804
:109928005BD09DF853309DF852201599C5F8E41086
:109938001B0443EA02239DF8512002201343C5F873
:10994800E03004F037F99DF8583095F8480085F86C
:109958002E71C3F30212C3F3030385F8703085F840
:1099680078309DF8593085F86920012B38BF0123DC
:109978004FF47A725343AB651344EB650DF15A0308
:109988004FF001081093113E94F81B348DF83C30C9
:109998000FA985F868808DF8446002F056FA022312
:1099A800404685F8303101F077FD18B14146384618
:1099B80001F038FD94F88F34012B00F2A78194F858
:1099C8001A34002B40F09A8194F8913443F0100334
:1099D80084F89134FEF786FD64E6012001F05CFD11
:1099E8000028E7D001210720E2E7012384F820348A
:1099F80095F87D308DF82E3094F824348DF82D307C
:109A080095F88C3095F848000D330BA98DF82C305B
:109A180002F000FAA6F10D031BB2099023EAE373E2
:109A280000B283423FF736AF0B2E7FF633AFBA4B07
:109A380025931CA8FF231C978DF874608DF8983027
:109A480002F0C4F8074600287FF424AF95F81831CF
:109A5800012B13D101F067FB002872D0384601F0C2
:109A680057FB384601F059FB04239DF87C101E98DB
:109A780084F88F34C1F3001101F06EFB9DF87C303F
:109A88001E99C4F8341413F00F0203D09DF8900007
:109A9800002862D19DF89800002861D0002A7FF440
:109AA800F9AE9DF89020002A14BF4FF003084FF03C
:109AB800020800220A92D5F8EC2095F8E9009142B4
:109AC80051D100284FD0D5F80C1195F8EAB00968A3
:109AD8000A9195F81811022902D1032184F88F14EC
:109AE800B8F1030F7FF4D6AE13F0600F7FF4D2AE57
:109AF8000492012795F82E31BBF1000F36D0BBF147
:109B0800010F13D1012B33D16FF0090646FA08F67D
:109B180006F00106C6F10206F6B2BDF87E100AAAE2
:109B2800304601F011FE38B3072823D0012384F80A
:109B380021340A9BC4F83034C4F86C34FEF720FD95
:109B4800B0E501F0F2FA002898D0384601F0E1FAC1
:109B5800384601F0E3FA052387E74FF00008A8E745
:109B68004FF00108A5E74FF0010BC3E70426D4E73F
:109B78000326D2E70823DAE71CAB009304990A9B73
:109B88003246584601F0A2FE20B1022814BF0B232A
:109B98000A2380E60A9BC4F83034C4F86C349DF874
:109BA8007C3084F82104C3F3401384F82E3484F8FD
:109BB800443494F88F3484F82274012B9EBF012218
:109BC800A86285F81E21012FC4F8280484F82C0403
:109BD80084F8410438D1022284F8202495F83A20E8
:109BE800002A4AD19DF87C20D60646D4012B94F849
:109BF80040149DF87C2005D8012901D1900601D593
:109C080001F04CFBB8F1020F94F88F3443D0B8F14F
:109C1800030F0AD09DF87C10B8F1010F4A4601F0F5
:109C28000F0120A83BD0FFF745F99DF8903084F844
:109C38002334259BC4F828349DF8983084F82C34B4
:109C4800012384F82D3430E0059A02F0E002A02ABE
:109C58001BD195F82E11012285F83A2009B92799C8
:109C68006963012B84F8202407D9D5F89020C4F81B
:109C78003C24DAF80020C4F8982495F81821002A22
:109C8800B4D1012284F82524B0E7002285F83A20CF
:109C980084F82024A6E79DF8981025984A46FFF7EF
:109CA80009F99DF8903084F823349DF89020E02A33
:109CB80008D195F81F312BB984F82324C4F8283427
:109CC800A4F82C3494F8913443F0020384F89134C6
:109CD80070E6114D013EB2B2791C284604F034F802
:109CE8000323A4F82034C4F8285484F82C64E9E742
:109CF800012384F82134FEF743FC5BE694F84434EE
:109D0800002B3FF461AE0020FEF726FC94F88F3458
:109D1800022B3FF45FAE57E6D415002094F8913437
:109D2800590715D5012001F0B7FB60B1012001F0FA
:109D38008BFB08B984F81804D4F8403323F00203E5
:109D4800C4F8403304E0062001F0A6FB0028F3D154
:109D580094F89134DA077FF5FAAC94F840240AB104
:109D6800032A18D11D4A94F8181492F868209142D1
:109D780005D29B0723D594F88F34012B1FD8184898
:109D880006F0FAFAD4F8403323F02003C4F840333D
:109D9800FFF744FBDBE4012A11D194F81924002AC7
:109DA8003FF4D5AC0D4A94F8181492F86820914203
:109DB800E5D29F0703D594F84434002BDFD194F8FB
:109DC800913400206FF3041384F8913484F8190453
:109DD800FFF746FBBBE429B0BDE8F08FD80D0020A3
:109DE800041700202DE9F04F89468DB090460746AC
:109DF800002800F08F81002900F08C810368002B77
:109E080000F088814368002B00F084818368002B70
:109E180000F08081C368002B00F07C81104601F0BF
:109E2800F5FF002800F07881BD4CBE4D384601F0A2
:109E3800AFFA40F2C4520021204603F099FF40F2E5
:109E48001C520021284603F093FFB74BC4F82C316D
:109E580004F50973089304F50A730026404609932C
:109E680008A9B24B84F848800A9384F8186184F8EA
:109E78008C608DF82C6001F0DBFF0F2306A994F8A5
:109E880048008DF8183001F0C5FF801B18BF01206D
:109E98004FF00A0B84F81C0106A994F848008DF8C5
:109EA80018B001F0B7FF4FF0060A84F8DC0006A9E5
:109EB80094F848008DF818A001F0ACFF102384F83E
:109EC800DD0006A994F848008DF8183001F0A2FFCB
:109ED8001123C4F89C0006A994F848008DF818309E
:109EE80001F098FF1223C4F8A00006A994F84800CE
:109EF8008DF8183001F08EFF1323C4F8A40006A9CA
:109F080094F848008DF8183001F084FF1423C4F841
:109F1800A80006A994F848008DF8183001F07AFFD7
:109F28001623C4F8AC0006A994F848008DF8183038
:109F380001F070FF172384F8B10006A994F84800CF
:109F48008DF8183001F066FF18230DEB0301C4F8F3
:109F5800B400C4F8BC0094F848008DF8183001F03B
:109F680059FFC0B21D2384F8B80084F8C00006A9C0
:109F780094F848008DF8183001F04CFF1E2384F83F
:109F8800C40006A994F848008DF8183001F042FF83
:109F98001F2384F8C50006A994F848008DF81830E6
:109FA80001F038FF2023C4F8C80006A994F8480037
:109FB8008DF8183001F02EFF0B23C4F8CC0006A949
:109FC80094F848008DF8183001F024FF0C2306A9F6
:109FD800A4F8D00094F848008DF8183001F01AFF62
:109FE800D4F89C306365D4F8A030A365D4F8A430C5
:109FF800E365D4F8A83023664FF00108D4F8AC30F4
:10A008000590A4F8D200636684F8B080C4F894B0D0
:10A0180084F898A0C4F84CB084F850A084F86880FC
:10A0280084F81F81C5F84893FEF7AEFDC5F8447360
:10A03800C4E90B663E4B84F8198185F89164C5F82C
:10A04800408332464FF0FF31009605F55A7006F00E
:10A0580035F9384B009632464FF0FF3105F5607000
:10A0680006F02CF9344B009632464FF0FF3105F5D7
:10A07800667006F023F902AF304B009632464FF077
:10A08800FF3105F5806006F019F9384606F0AAF8A0
:10A0980097E8030004F5927383E80300284B294FDF
:10A0A8001E60294BC5F84C33284BC5F85433284B50
:10A0B800C5F85C33274BC5F85033274BC5F85833E0
:10A0C80005F553703B68984704F5A67003F080FBCC
:10A0D80020B1112630460DB0BDE8F08F204601F0C2
:10A0E80003FB0028F5D101F039F8B8B91B4801F095
:10A0F8004DFB06460028ECD17B69984703F002FE29
:10A10800BB6D94F819019847FB6A9847012385F8B5
:10A118009234DFE70326DDE70926DBE71326D9E7D4
:10A12800D80D00209C1300200004000184070020A3
:10A1380069940008318D0008798D00086185000850
:10A1480080070020C412010821870008D58600086E
:10A158001D850008AD86000885860008C00E002011
:10A1680008B5034B0020C3F84003FEF7BBF908BD50
:10A178009C13002010B5FFF7ABF90A4C60B90A4BE5
:10A1880093F81831022B02D1084BDB6A9847012358
:10A19800C4F84033002010BDD4F84003013818BF7C
:10A1A8000120F8E79C130020D80D0020C4120108F4
:10A1B80038B5124C204606F0DFF804F1180006F016
:10A1C800DBF804F1300006F0D7F804F1980006F047
:10A1D800D3F800F0AFFF0A4B0025DB6A984744F834
:10A1E800285CFEF7EDFD0749074840F2C45203F02A
:10A1F800ABFD012344F8283C284638BD041700204D
:10A20800C4120108D80D00201408002070B52E4B88
:10A218008AB0054693F8DD008DF8090093F8DC0054
:10A228008DF80A0029489A6A90F8180403920026C3
:10A238008DF80B0004960C46002940D00692D3F8FE
:10A24800882007921A8F93F81A118DF8151052BAB0
:10A25800ADF8202093F87C2093F848308DF824300E
:10A2680003AB8DF822008DF8232000930DF10A022C
:10A278000DF10B030DF1090105A88DF8146000F02C
:10A28800D7FE9DF90900FEF74FF9607004A801F0A8
:10A298001BF8B0B9049A0F2A0DD863789A420AD8E5
:10A2A8001544AB42A3EB02012CBF00200120217012
:10A2B800C0000AB070BD002323700820F9E703200E
:10A2C800F7E71320F5E700BFD80D00209C13002006
:10A2D8001FB50446002800F010810378412B00F2D6
:10A2E8000781DFE813F0420049004D005100550096
:10A2F80059005E000501050105010501050105017B
:10A3080005010501650069006D0078007F00820085
:10A3180085008A0088008C009000930096009900C0
:10A328009C009F00AE00B200BA00B600BE00C1009B
:10A33800C500CE00CA00CC000501D2000501050108
:10A3480005010501050105010501050105010501D5
:10A3580005010501050105010501DA00DE00E2003D
:10A36800E700EB00EF00F300FC00664B93F81831B0
:10A378002371002004B010BD624B93F83031F7E729
:10A38800406803F0C3FBF4E7406803F005FCF0E71E
:10A398005C4B93F81A31EBE75A4BD3F8E030636023
:10A3A800E7E7584B011D93F8300103F00DFCE0E797
:10A3B800544B93F81931DBE7524B93F88C30D7E7BD
:10A3C8001C238DF808304F4B02A993F8480001F080
:10A3D80021FD6060CDE74C4B043493E8030084E82A
:10A3E8000300C6E7494B0434F7E7494B0434F4E764
:10A3F800484B0434F1E71A23E3E71923E1E7414B1B
:10A4080093F86830B4E73F4B5B6DC8E73D4B9B6DF5
:10A41800C5E73C4BDB6DC2E73A4B1B6EBFE7394BD8
:10A428005B6EBCE702238DF80830364B02A993F81F
:10A438007C2093F848008DF80A2001F0EBFC20718D
:10A4480097E7304B93F8DD3092E72E4B93F839308D
:10A458008EE72C4B93F8DC308AE72A4B93F8383098
:10A4680086E7284BDB6C9AE7264B93F850307FE75A
:10A47800244BD3F8843063607BE7224B8FE7264B6D
:10A488008DE7204BD3F8CC30F5E71E4BD3F82C31B1
:10A49800436001F04DFDA0606BE71A4BD3F8903094
:10A4A8007DE7184B93F81F3162E7164BB3F88830F5
:10A4B800A3805EE7134BB3F88A30F9E7114BB3F882
:10A4C800D030F5E70F4BB3F8D230F1E70D4B93F8E6
:10A4D80048200AB1062A12D1B3F8A035E8E7094B9B
:10A4E80093F848200AB1062A09D1D3F8A43556E7CB
:10A4F80004B0BDE8104000F021BE03203AE7182060
:10A5080038E700BFD80D0020440E00208C0E002034
:10A518004C0E0020940E0020140800207FB504463D
:10A5280010B9032004B070BDA34DD5F840339A0785
:10A5380000F16F820278412A00F26882DFE812F0A7
:10A548004200470055005B005F0064006900760028
:10A55800810087008D00930099009F00A500AB0043
:10A56800B5006602BA00DC00EF00160138012901C7
:10A5780042014B014F01530157015B0166025F0124
:10A58800710199018701AB01B101B801BD01C20197
:10A5980066022802660266026602660266026602B1
:10A5A8006602660266026602660266026602660263
:10A5B80066026602340239023E02430248024D0234
:10A5C80052025C020079FEF773FA30B1AAE7037908
:10A5D800022BA6D0794A82F8303195F8913443F0AD
:10A5E800200385F8913400209CE7406803F080FA46
:10A5F8000028F2D095E7406803F0BEFAF8E76F4B01
:10A60800027983F81A21E8E76C4B4268C3F8E02026
:10A61800E3E76A4E416896F8300103F0CBFA002868
:10A628007FF47FAF6368C6F8E430D6E74168002955
:10A638003FF477AF002001F0DDF90028CDD01120DC
:10A6480070E7416800293FF46CAF0120F3E74168E7
:10A6580000293FF466AF0820EDE7416800293FF480
:10A6680060AF0920E7E7416800293FF45AAF0C20A2
:10A67800E1E7416800293FF454AF0D20DBE741686A
:10A6880000293FF44EAF0E20D5E7416800293FF47A
:10A6980048AF0F20CFE74A4C484B007983F819019F
:10A6A800A36D9847E36A984797E7444B027983F884
:10A6B8008C2092E7414E037A8DF8043096F84800D2
:10A6C80096F87D308DF80530072201A901F0B5FB19
:10A6D80000283FF426AF636896F8480001930022EB
:10A6E80001A901F0AAFB00283FF41BAF6C36D4E99E
:10A6F800010186E8030070E7304E037A8DF80430D4
:10A7080096F8480096F87D308DF80530072201A9A3
:10A7180001F093FB00283FF404AFB436E7E7274E77
:10A72800037A8DF8043096F8480096F87D308DF855
:10A738000530072201A901F080FB00283FF4F1AEA3
:10A74800D4E9010106F1740383E8030096F818318F
:10A75800022B7FF442AF96F83031002B3FF43DAF27
:10A76800174BDB6A9847FEF775F936E7134E037AFD
:10A778008DF8043096F8480096F87D308DF805304D
:10A78800072201A901F059FB00283FF4CAAEBC36E4
:10A79800ADE74368029301238DF80C30074B02A9FB
:10A7A80093F8480001F056FB00287FF416AFB8E68E
:10A7B800436802930023EFE79C130020D80D002084
:10A7C800C412010803795A1E0E2A3FF6AAAE934A0C
:10A7D80082F8683001E7914B42685A65FDE68F4B75
:10A7E80042689A65F9E68D4B4268DA65F5E68B4B67
:10A7F80042681A66F1E6894B42685A66EDE6874C6C
:10A80800037994F848008DF80430062201A901F074
:10A8180014FB00283FF485AE9DF8043084F8DD3041
:10A82800DBE67E4C03798DF8043094F8480094F800
:10A838007C308DF80630052201A901F0FEFA0028C7
:10A848003FF46FAE9DF8043084F83930C5E6734C98
:10A85800037994F848008DF804300A2201A901F020
:10A86800ECFA00283FF45DAE9DF8043084F8DC3043
:10A87800B3E66A4C037994F848008DF8043009224D
:10A8880001A901F0DAFA00283FF44BAE9DF8043034
:10A8980084F83830A1E6614B4268C3F89420DA6442
:10A8A8009BE65E4B027983F8982083F8502094E663
:10A8B8005A4B4268C3F884208FE6584B4268C3F865
:10A8C800CC208AE6012B40F0A480554C2421204658
:10A8D80003F050FA636A984201D0172022E61C213F
:10A8E80004F1280003F046FA636C9842F5D14FF45E
:10A8F800807104F1480003F03DFAD4F848319842D9
:10A90800EBD1D42104F5A67003F034FAD4F8203240
:10A918009842E2D1002104F5097003F02BFAD4F82B
:10A9280024329842D9D14FF4607104F50A7003F0CB
:10A9380021FAD4F8A8359842CFD1142104F2AC50AA
:10A9480003F018FAD4F8C0359842C6D1334E2146E0
:10A95800304640F2C45203F0F7F9204640F2C452A0
:10A96800002103F005FA95F81B3485F8E833736F76
:10A97800C5F8EC3396F87D3085F8F83340F20123BA
:10A98800A5F8FA33274B96F819019B6D984724E6EA
:10A998008379012B3FF6C5AD204B42684068C3F868
:10A9A8002C2100F0BDFE48E61C4B4268C3F89020FD
:10A9B80013E61A4B027983F81F210EE6174B82889B
:10A9C800A3F8882009E6154B8288A3F88A2004E6B4
:10A9D800124B8288A3F8D020FFE5104B8288A3F899
:10A9E800D220FAE50D4B93F848200AB1062A12D175
:10A9F800A288A3F8A025F0E5084B93F848200AB1EF
:10AA0800062A08D16268C3F8A425E6E500F098FB99
:10AA1800DBE5012086E5182084E500BFD80D00207D
:10AA280014080020C41201082DE9F04387B0002360
:10AA3800ADF800300646002800F0EE800361FEF70E
:10AA480047FD20B10124204607B0BDE8F08300F09F
:10AA580065FD0028F6D100F05BFD014618B96F4886
:10AA6800142203F085F96E4D95F89134012243F0D4
:10AA7800040385F8552485F8913433788DF804302B
:10AA88000021013B8DF80520ADF806100C2B00F2D3
:10AA9800BB80DFE803F007B9B9B97982B9B990B9D1
:10AAA800AD9AA900D5F8407317F02007CAD196F8D7
:10AAB8000480B8F1020F46D1DFF868815A4CFEF7DE
:10AAC80063F896F9051098F848003A4601F00FFA2D
:10AAD80088F83900B37988F83830384607238DF874
:10AAE8000530FDF7E5FFFF2304F58670A5F80C3166
:10AAF800C5F8084185F8047103F04EF804F58A702A
:10AB080003F004F83846FDF72DFE0446002839D036
:10AB180096F9051098F84800012201F0E8F988F83C
:10AB28003900D5F894343361002C71D000F0F0FC72
:10AB3800002888D195F8913485F81A0460F38203C7
:10AB480085F891347FE7B8F1010F4FF00204E8D19E
:10AB5800DFF8D0908DF8144099F8480089F81D71F5
:10AB680002A901F065F9337989F830318DF805705B
:10AB78008DF80680FDF7C4FC95F8913443F0100376
:10AB880085F891340024CCE700226946022000F0C1
:10AB9800F3FA0028F6D01324C3E7244BB288DB6B02
:10ABA80096F90C10B0689847D5F8403343F0020383
:10ABB800C5F84033E6E702A90D2000F053FB002852
:10ABC800E0D0002269460D20E1E7164B93F81831D2
:10ABD800D3B9347904F0070000F0ABFA8DF80040DF
:10ABE800012269461020D2E7002269461220CEE7EA
:10ABF8008DF8072000F08EFA044638B900F087FA7D
:10AC0800204600F089FABDE702248AE7012488E794
:10AC180001A800F0D1FB16E7032414E7F017002081
:10AC28009C130020D80D00209E130020C412010898
:10AC38002DE9F04F99B08046059118B9032019B055
:10AC4800BDE8F08F00230361FEF742FC04460028AC
:10AC580040F0A58046460FCE0EAD0FC514225248CF
:10AC680098F800A0B8F80C7098F90EB04F4E21462D
:10AC780003F07EF84E4B012283F8412496F83021E8
:10AC8800022A25460BD196F81821022A07D196F8F0
:10AC98001E2122B9BAF1010F38BF4FF0010ABAF1EB
:10ACA800010F2BD0BAF1030F2AD0BAF1000F33D11C
:10ACB80002229DF83C30DDF84090029362F347157C
:10ACC800012496F87C108DF8321002220CA996F80F
:10ACD80048008DF8302001F09DF896F81A3196F862
:10ACE80030C196F81D1140B2002B63D0BCF1010FA2
:10ACF80057D1002955D1002C61D153E00422D8E75F
:10AD08000023DDF83C90BDF840709DF942B00293F5
:10AD180065F01F050124D4E74FF0000BD946CDF8A4
:10AD280008B0CEE74FF0010084F81A04D2E005F22B
:10AD38009A420BA900F0D4FA002800F015811320DC
:10AD4800049B33871A4B002283F81A2423E105F267
:10AD58009A452A460BA900F0C3FA0028EFD10B9BAD
:10AD680084F82801C4F82C5184F83031FCE0B9F19A
:10AD7800000F00F0F980002A00F0F6804946E01C38
:10AD880002F0E2FF94F8373201332380ECE012201E
:10AD9800D6E70220D4E70720D4E71320D2E7012022
:10ADA8004DE7FCB90220F6E0DC170020D80D0020A2
:10ADB8009C130020002CF5D05845B8BF584696F88B
:10ADC8007C308DF82000052296F848008DF8223056
:10ADD80008A901F032F800283FF430AF9DF8203080
:10ADE80086F839306F4A704BD2F89804D3F89040FF
:10ADF80038B105F087FA6C4B84423CBF002283F8D7
:10AE08003A20198F1A8F93F830010491996A0991A1
:10AE180052BA0028BFD093F81B0100B9186393F801
:10AE28001801ADF85820013893F87C2093F81A419E
:10AE38001491D0F1000BD3F888108DF85B204BEB00
:10AE4800000B93F8482093F83A0093F868308DF88F
:10AE58005A3009AB0093554B03904FF001008DF821
:10AE68004C0015918DF85C20A3F12F01A3F130025D
:10AE780013A88DF84D4000F0DBF8039B4FEA0B1B3D
:10AE88004BEA431B00264BEA801B4BEAC413B1452F
:10AE9800444C039308BF37463A46494604F59C702C
:10AEA800CDE90A669B46268084F81A6402F04CFFB6
:10AEB800E9B2A570C5F34215FAB2042D3A4E039BC8
:10AEC80084F837223FF42EAF072D3FF450AF022D00
:10AED8007FF45FAF364D84F80D110420029984F891
:10AEE8000401FF2084F80C0184F8281184F8143137
:10AEF800D6F8E410C4F8085105F59B730AA8C4F8FD
:10AF0800101184F83021C4F82C3100F011FC00280D
:10AF18007FF43DAF0A9BA4F844040BA8A4F81631AB
:10AF2800C4F84C3400F0D0F900287FF408AF0B9B2C
:10AF3800D3B196F93900FDF7F7FA94F83732002BB8
:10AF48003FF405AF0B9B0F2B3FF6F1AE05F58B7267
:10AF58000BA90F2000F0C4F900287FF4F0AE0B9B7A
:10AF680063F3030B84F814B10598FDF7FBFB002885
:10AF78007FF4E6AE099B86F83A00B36200F080F9E8
:10AF880000287FF40AAF94F8913484F840A443F081
:10AF9800010384F89134034BD3F89434C8F8103083
:10AFA8004DE600BF9C130020D80D0020400E002065
:10AFB8009E13002037B50B4D8DF8040004460F2270
:10AFC80095F8480001A900F038FF40B1064A85F815
:10AFD8001C4192F8913443F0200382F8913403B075
:10AFE80030BD00BFD80D00209C13002010B5FFF71E
:10AFF800C1F8044688B90A4805F0BEF9094805F0C1
:10B00800BBF9094805F0B8F900F094F8FDF7BCFD64
:10B01800064BDB6A9847204610BD0124FBE700BFBA
:10B02800041700201C17002034170020C412010840
:10B038002DE9F04F8BB047780093149B90F90C8062
:10B0480090F90D6090F80EB08A4641681960044680
:10B058009146002F58D002238DF8103004A9C37BE5
:10B06800007C8DF8123000F0D5FEB4F808C0618974
:10B0780043B26068984545466144B8BF1D4660457F
:10B0880034BF00270127884209D30A218DF8101000
:10B09800207C019304A900F0BDFE019B46B2B4F8E0
:10B0A80008C0608961680CEB400E714519D3A1EBAB
:10B0B8000C01B1FBF0FC00FB1C1191B9984503DCB5
:10B0C8002378CBB94FF0010B21238DF81030207C69
:10B0D800E37B8DF8115004A98DF8123000F09AFE28
:10B0E80045B2009B8AF80050384689F8006083F81A
:10B0F80000B00BB0BDE8F08F0223207C8DF824301F
:10B1080006A900F095FEDDE74546EAE77047704777
:10B11800704770470020704770477047704700209D
:10B1280070470020704700207047002070470020BB
:10B138007047704770477047022070470220704779
:10B148000220704770470020704770477047002002
:10B1580070470020704770477047704710B5054C1E
:10B168004FF403722046002102F002FE0020C4E9D9
:10B17800000010BDB81800202DE9F843814690461C
:10B1880000293CD01F4C2023224604F1100012F85D
:10B19800017F6FBB8242FAD11B4E3368013403B979
:10B1A8003460736803B11C6000252560C4F808800A
:10B1B80074601FFA88F284F80490601D02F0C4FDE0
:10B1C800B9F1110F4FF0000398BF104D6373D6F813
:10B1D800083298BF25FA09F503F1010398BF05F075
:10B1E800010543442573C6F808323846BDE8F8839C
:10B1F800013B13F0FF030446C6D10227F5E70127F8
:10B20800F3E700BFBF180020B8180020200702008D
:10B2180010B518B3124A1368984204D10368136032
:10B22800002305E00B46002BFAD019688842F9D1B3
:10B238005168884208BF53600BB101681960D2F8A1
:10B2480008328168013B00245B1A04602146C2F879
:10B258000832102202F08CFD204610BD0120FCE7C8
:10B26800B8180020054B1B6813B11A798242FAD12D
:10B27800002B0B600CBF032000207047B81800207B
:10B2880010B5054B186800B910BD037B04680BB9ED
:10B29800FFF7BEFF2046F6E7B818002038B5084B80
:10B2A800084C186800B938BD03790568112B05D812
:10B2B80024FA03F3DB0701D5FFF7AAFF2846F1E7D5
:10B2C800B81800202007020028B1044BD3F8083230
:10B2D8000360002070470120704700BFB8180020A5
:10B2E8002DE9F04107460E46154642B339B3154BD2
:10B2F8001C6800232CB93046FFF7E6FF0020BDE8A4
:10B30800F081A268F91A0132914215D32279EA54E0
:10B31800581C22895FFA80F8611D55FA80F002F006
:10B3280013FDA368246898445FFA88F3E2E720468F
:10B338002568FFF76DFF2C46002CF8D1DBE70120CC
:10B34800DDE700BFB81800200238C0B211289ABF44
:10B35800014B185C00207047DB0B010830B50B4B24
:10B3680093F820200446084672B100211C33057862
:10B37800A54208D001319842CDB214BF043010382C
:10B38800AA42F4D8002030BD1046FCE7C41A0020B9
:10B3980010B5084C00232060142204F10C00FF2192
:10B3A80084F82030C4E9010002F0E2FC012384F8AB
:10B3B800213010BDC41A002010B50E4A92F8201092
:10B3C800042915D8936804781C7044785C70C47894
:10B3D800807898700131DC7082F8201002F11C012D
:10B3E8008B4214BF043302F10C039360012010BD9B
:10B3F8000020FCE7C41A0020094B93F8200068B12C
:10B408005A6803F11C018A4200F1FF3014BF04326C
:10B4180003F10C0283F820005A600120704700BF36
:10B42800C41A002010B5074B93F82020044608469C
:10B4380032B15968FFF792FF10B10123447083704D
:10B4480010BD00BFC41A002008B5064B93F8202091
:10B458002AB15968FFF782FF08B1407808BD01207A
:10B46800FCE700BFC41A002030B50A4A92F8201041
:10B47800536882F8210061B1916801241C32DD789B
:10B48800587005B99C70934214BF0433103B99421D
:10B49800F5D130BDC41A002008B5044B5968FFF730
:10B4A8005DFF003818BF012008BD00BFC41A002086
:10B4B800F7B50422154E044600210DEB020096F85C
:10B4C800207002F055FC0025EBB29F4201D803B072
:10B4D800F0BD7368197821705A786270987838B11D
:10B4E800336820469B689847FFF786FF0135EBE7EE
:10B4F800DB788DF804108DF805208DF80730FFF7FC
:10B508007BFF01A8FFF758FFF0E700BFC41A00202F
:10B51800014B93F820007047C41A0020034B93F89E
:10B528002000042894BF002001207047C41A00207E
:10B538001FB50024CDE90244C41F8DF800408DF8E2
:10B5480001100C0AADF80420090C120C8DF8031038
:10B558008DF806208DF8073002461B0A012168463F
:10B568008DF802408DF8083002F05DFA002818BF07
:10B578000E2004B010BD2DE9F04188B090460D466C
:10B588000F9A0746002847D000240121CDE904443A
:10B598008DF810109DF838108DF81510ADF816308C
:10B5A800190CCDE900441B0ECDE902448DF8193081
:10B5B800ADF81A20130C120E07948DF818108DF898
:10B5C8001C308DF81D20E3B21E01002DF6B203DCFD
:10B5D800002008B0BDE8F081013310218DF81F303C
:10B5E80042466B460DEB010002F0B3F90346A8B9D9
:10B5F800102D28463E44A8BF10206946327811F81D
:10B6080001CB013382EA0C02984206F8012BF5DCE3
:10B61800103D2DB20134D6E70920DAE70E20D8E72D
:10B628000138032815D8DFE800F002080C100A4B8F
:10B638001B681B690B6000207047074B1B685B6920
:10B64800F8E7054B1B689B69F4E7034B1B68DB694C
:10B65800F0E70520704700BFE81A00202DE9F04107
:10B66800C4B00C464A9E17461D468046B8B3B1F58D
:10B67800807F36D84FF488720021684602F078FB44
:10B68800492300934FF48073ADF804302B0C8DF8E8
:10B698000830330CADF80650ADF80A608DF80C3060
:10B6A80022460023414604A82D0E360E8DF80E3092
:10B6B8008DF809508DF80D608DF80F4002F044FBAD
:10B6C80004F110014B9A3B4689B2684602F02BF907
:10B6D80010B1012818BF0E2044B0BDE8F081092040
:10B6E800FAE70D20F8E7000010B590B10A4C2822BF
:10B6F8000021206002F03CFB2368084A1A60002001
:10B708004FF0FF32C3E90302C3E90522C3E9072268
:10B7180010BD0820FCE700BFE81A00200001010165
:10B72800024B1B6818600020704700BFE81A002011
:10B7380030B1044B1B68DB6801330360002070479D
:10B7480009207047E81A002013B500230C4601931E
:10B75800CAB101A9FFF764FF18B9019B591C02D1AE
:10B76800146002B010BD99B2611A002901DD5C189D
:10B77800F6E702D113600720F3E71B0C1B0403F55F
:10B7880080331C44ECE70920EBE7000028B1044BA8
:10B798001B681C334362002070470920704700BFB4
:10B7A800E81A00201FB5044600B3002303A803933A
:10B7B80002F090F9104ABDF80C30126820469380C8
:10B7C800E38200F05EFA98B904F118030093216847
:10B7D8000123132202F09CF860B9204600F051FAC8
:10B7E800003818BF0120000104B010BD0920FBE794
:10B7F8001020F9E70E20F7E7E81A0020F0B5054613
:10B8080087B01C4613B9092007B0F0BD2E4E336827
:10B81800DB68834255D894F82020002A0CBF082200
:10B828000922834205D3204600F05FFA68B1102050
:10B83800EAE7002301900093A36894F82810606A4F
:10B84800FFF799FE0028EED0DEE723792168B4F8E7
:10B8580008C0A768043B9AB20029D4D0B2F5807F0B
:10B868002DD8ADF80EC08DF817304FEA174C04F1FB
:10B878002C033F0E8DF8117000932F0C08234FF006
:10B88800490EADF80C008DF814708DF816002F0EC7
:10B898000DEB0300CDF808E08DF810C0ADF812509C
:10B8A8008DF8157002F034F808B10E20ACE7204688
:10B8B80000F01BFA0028BAD13368DD60A4E70D2038
:10B8C800A2E70620A0E700BFE81A00202DE9FF4103
:10B8D8000A9D80460F4616461C46002D5AD0002366
:10B8E80003A910460393FFF79BFE18B1062004B086
:10B8F800BDE8F081039B9C4201D80133F6D128466C
:10B9080000F064F9002847D1264B1A78424503D045
:10B918001A79424542D10120AA68BA4240D103EBC4
:10B928008002EB6A92F801802979CDE90043043955
:10B93800927828683B4689B2FFF790FE0028D6D156
:10B9480095F820300194002B4FF00103009314BFA9
:10B958004246082295F82810686A3B46FFF70BFE16
:10B968000028C4D1013E032EC1D8DFE806F0020743
:10B978000B0F0D4B1B681C611C62B8E70A4B1B6858
:10B988005C61F9E7084B1B689C61F5E7064B1B688F
:10B99800DC61ACE70920AAE70F20A8E70B20A6E79F
:10B9A8000220A4E734010020E81A00201FB50B2963
:10B9B8004FF00003CDE90033CDE902330A4607D042
:10B9C8000C2914D00A2910D00A2005B05DF804FB10
:10B9D800012802D120238DF800300021684602F0AA
:10B9E80022F8002818BF0E20EFE73023F3E70B21D9
:10B9F800F4E7000038B5054602F010F8044610B127
:10BA08000E24204638BD002DFBD1094B1B680B21A5
:10BA18009878FFF7CBFF0028F2D10C21FFF7C6FF7B
:10BA28000028EDD10A21FFF7C1FF0028E9D0E7E798
:10BA3800E81A00202DE9F04380468FB00C461746DF
:10BA4800002A6BD0002969D0002529461D2206A8A6
:10BA5800059504F0A7FE8DF81350344D2B680DF1B1
:10BA680014099E88CDF804900DF1130302933B79D5
:10BA780000933B6832462146404601F0F0FF00281B
:10BA88004ED138683A79494602F05EF9384600F0F6
:10BA98004FF8002846D13C7AFA79BB79240444EA65
:10BAA80002241C432B689A6894423DD99C609DF8F7
:10BAB80013000B21FFF77AFF034658BB0C21FFF751
:10BAC80075FF034630BB0A21FFF770FF034608BB2A
:10BAD8007B7ABA7AFF7A3F0447EA02271F433A463D
:10BAE800334621460920FFF723FD034690B9334624
:10BAF8003A4621460820FFF71BFD034650B92A683D
:10BB08009DF8131091700021D1604FF0FF31C2E908
:10BB18000411916118460FB0BDE8F0830923F9E7D5
:10BB28000E23F7E70F23F5E70323F3E7E81A0020CE
:10BB380010B50446002845D00168002942D011F804
:10BB4800013B43710322063002F0FEF8204603222F
:10BB580050F8091B043102F0F7F82168CB79E3604B
:10BB68000A7A43EA0223E3604A7A43EA0243E3603B
:10BB78008A7A43EA0263E360CB7A23740B7B6374AB
:10BB88002379212B1AD110220D3104F1120002F071
:10BB9800DBF81D222168501C8B5C6362085C43EA59
:10BBA8000023901C6362085C033243EA004363622B
:10BBB8008A5C43EA02636362002010BD112B03DC38
:10BBC8000D22E7E70220F8E70120F6E710B5044662
:10BBD800002854D00168002951D00B7843714B7864
:10BBE80083608A7843EA02238360CA7843EA02437F
:10BBF80083600A7943EA026383604B7903738B7924
:10BC0800C381CA7943EA0223027BC38102F00F028F
:10BC18000831103002F098F8237B002203F00F035C
:10BC280084F8202084F82820227903F10800111ACA
:10BC380004290DDD21680933043AD21A085C84F816
:10BC48002000D2B2606A84F82820194402F07CF8F7
:10BC5800237922681A44002012F8043CE36212F89F
:10BC6800031C43EA0123E36212F8021C43EA01437E
:10BC7800E36212F8012C43EA0263E36210BD02207A
:10BC8800FCE710B5044660B3036853B30279162A7B
:10BC980029D942791A700146082251F8060B013059
:10BCA80002F05CF82146082251F80E0B093002F028
:10BCB80055F82368E28A5A74E38A22681B0A937447
:10BCC8002368A269DA74A36922681B0A13752368BA
:10BCD800628B5A752368E27E9A75172323710020B8
:10BCE80010BD0120FCE70220FAE738B50446002819
:10BCF80063D00168002960D0037B90F8282003F006
:10BD08000F03002A57D1083320790432134498428C
:10BD180055D363790B702368A2685A70A3682268A8
:10BD28001B0A937023686289DA702368E27A1A71B1
:10BD38002368227B5A712368E2899A71E389226811
:10BD48001B0A2146D371227B51F8100B02F00F0217
:10BD5800083001F0F9FF237B94F8282003F00F0343
:10BD680003F108052AB1226894F82010515503F10F
:10BD78000905206894F82820616A284401F0E4FF46
:10BD880094F828302268E16A2B44D1545A1CE16A9D
:10BD9800206892B2090A81549A1C2168E08D92B2F7
:10BDA8008854DA1C216894F82F0092B2043388541E
:10BDB8002371002038BD0933A6E70120FAE70220E5
:10BDC800F8E70000024B1A8810431880704700BF3C
:10BDD800EC1A002008B5074B1B883BB1FEF7CAF9DF
:10BDE800002814BF6FF00200002008BD6FF00100AA
:10BDF800FBE700BFEC1A002010B5034B00241C80A1
:10BE0800FEF7AEF9204610BDEC1A0020B0FA80F01B
:10BE18004009704782B018B9084602B000F0CAB8A5
:10BE2800002002B0704710B9084600F077B9704793
:10BE380010B9084600F08EB9704703460846114607
:10BE48000BB900F0E5B90020704710B9084600F0BA
:10BE58006DBD704710B9084600F006BA002070475B
:10BE680010B40446084611461A46019B14B910BC82
:10BE780000F014BA10BC70470346084611460BB9C7
:10BE880000F03EBA0020704710B404460846114638
:10BE98001A4614B910BC00F0ABBA002010BC7047A9
:10BEA80030B40546084611461A46DDE902341DB984
:10BEB800029430BC00F02ABB002030BC704710B997
:10BEC800084600F0DBBB0020704710B9084600F0B8
:10BED8006BBD0020704710B9084600F0EABB00208F
:10BEE800704710B9084600F0E7BB002070470346CA
:10BEF800084611460BB900F001BC0020704710B489
:10BF08000446084611461A46019B14B910BC00F0B5
:10BF1800F7BB092010BC704710B404460846114608
:10BF28001A4614B910BC00F061BDC8B210BC704705
:10BF38000048704701000102064B10B51B6A044611
:10BF4800984730B10448054B204498428CBF0020E4
:10BF5800012010BDC412010840C220C980B92A00BE
:10BF6800F0B5114B85B00C4610491F56054601F037
:10BF78004BF80F4BE4B25E6A072D4FF00103CDE991
:10BF8800024301460AD105220023CDE900234FF4DC
:10BF98007A727A431846B04705B0F0BD08220020EF
:10BFA800CDE900203A46F5E7A80C0108880C0108FD
:10BFB800C41201081FB5002300930378013B372BF7
:10BFC80021D8DFE803F01C242020201E2020202078
:10BFD8004143454E2055585B5E6164206C1E6E736C
:10BFE800787A20207D8126202020202020202020D3
:10BFF8002020202083858A2020838A208C90C37863
:10C008000BB102230093009805B05DF804FB837818
:10C01800F6E743788DF8043005238DF805308378EA
:10C02800003B18BF01235B008DF8063010238DF804
:10C038000730304B1B6801A803F55872CDE902237D
:10C0480000F0C2FF0090DEE74023DBE72023D9E7BA
:10C05800827890F9013012B9274AD35CD2E7274A8F
:10C06800FBE7827890F90130002AF8D1244AF4E7F6
:10C0780040F6B833C6E74FF47A73C3E74FF4FA6370
:10C08800C0E741F28833BDE741F27073BAE71D4853
:10C098004FF47A7101F03CFE00F5FA60D2E71A4BD2
:10C0A800B0E7144B1B6803F55873ABE7114B1B68DB
:10C0B80003F55B73A6E71023A4E70E4B1B68A1E703
:10C0C8004FF0834300939EE7104BFBE7104B99E733
:10C0D80040F21113ADF8003095E7032392E790F989
:10C0E80001300C4AB9E70C4990F9010000F08CFFC7
:10C0F800A8E700BFF41A00207D0C01086D0C0108A8
:10C10800750C010818FCFFFF00EA06379A990940E8
:10C1180040F70937A80C0108880C010837B50B4B04
:10C1280002781B680C2101FB02335B7A03EB4304A2
:10C13800074B1D6803690093C3684278816805EB63
:10C14800C40000F0DDFC03B030BD00BFF41A0020CD
:10C15800F01A002070B586B0027B6423ADF8003079
:10C16800012A4FF00003CDE90133CDE903338DF8FF
:10C1780002308DF8143030D0022A39D05ABB036807
:10C188004BB343683BB31F4D80682B601E4B18228E
:10C198006946186001F0D8FD1C4B2C6893E807002D
:10C1A8000C3384E8070093E8070004F10C06032326
:10C1B80086E80700A4F86C33012204F55B7104F5E6
:10C1C800587000F08EFC2B684FF6B072A3F87823F5
:10C1D8000522C3F87C2306B070BD0A49086843608D
:10C1E800036100F55B7100F5587000F07AFCF2E726
:10C1F800044B1B68B3F86023B3F86C130A43A3F825
:10C208006023E8E7F41A0020F01A002088090108E2
:10C2180008B503460A2924D8DFE801F006232323BA
:10C22800230B161B23212100BDE808400068FFF7F7
:10C2380083BE90F900009978052271B900F011FCCD
:10C24800003818BF012008BD052293F9000000211D
:10C25800F4E790F900005978EEE70221EEE70722AB
:10C26800F3E70020EFE7000008B502791AB1012AC8
:10C278000BD0002008BD084B01681B68012203F59C
:10C28800587000F02EFC0120F4E7034B01681B688E
:10C2980003F55B70F5E700BFF41A0020F7B5052831
:10C2A800144D1C46A8BF052058700E46294617464F
:10C2B80000F0AAFE94F90130A070072B13D13220A8
:10C2C80000F0A2FD0C4BDB6D0546984704F10C020B
:10C2D80008340346019200943A463146284600F055
:10C2E80098FD03B0F0BD054A55F82310D05C00F066
:10C2F80083FDE7E7880C0108C4120108A80C0108AF
:10C308002DE9F04F344F90F901607B68D0F8049024
:10C318008BB00446884698470546002859D1E37CE7
:10C3280073B92E4A2378126803EB4303990002EB92
:10C338008303D3F80490B9F1000F01D152F80190AA
:10C34800274B484613F906B0FB689847A37C228917
:10C35800D7F818A00993072E28D100230121CDE989
:10C368000223204A0693CDE90431CDE9073305219C
:10C37800CDE900214FF47A7202FB0BF24CF25031F6
:10C388001846D047637C13B3174B995D7B6D0D310D
:10C39800C9B228469847E07C3246494600F046FE36
:10C3A80088F8006001200BB0BDE8F08F002101255E
:10C3B8000823CDE90013CDE90715CDE90511CDE92D
:10C3C80003110292A1782B465A462846D9E7074B13
:10C3D800DBE70020E7E700BFC4120108F41A0020D9
:10C3E800A80C010885450100750C01087D0C0108A1
:10C3F8002DE9F04F8DB090F90130DFF8FCA0DFF89F
:10C40800FC90CDE90A123E4A12F903B00278DAF834
:10C4180000300C2505FB02333A4A5B7A126803EBBD
:10C42800430302EBC303044693F9021090F9020098
:10C4380000F0E5FD3449064694F9010000F0E4FDFA
:10C44800A26861688046304600F00BFD2178DAF872
:10C458000020D9F80C306943074650589847D9F856
:10C468001C309C4694F901300025072B4FF47A6361
:10C47800CDE90753CDE905552DD10123CDE9035366
:10C488000523CDE901534FF47A7303FB0BF30093B3
:10C498003946434646F2A81228466746B8472378E5
:10C4A800DAF800200C214B4394F90110D05800F021
:10C4B800DFFDA18994F90100FFF752FD0B9B217B59
:10C4C8001860D9F85430284698470A9B01201E70F6
:10C4D8000DB0BDE8F08F01200823CDE90350CDE968
:10C4E80001032A46CDF800B0654643463946A847B9
:10C4F80001200546D3E700BFF41A0020C412010842
:10C50800A80C0108F01A0020880C01082DE9F04F4A
:10C518008FB0002405468A46914698460494ADF8A3
:10C528001440ADF8024007264FF0010B2B7AA342C6
:10C5380006D9686804A9204400F0F6FB00285ED1FB
:10C5480002238DF8083002A86B7A8DF80A30FFF7BD
:10C5580031FDAB7A8DF81D309DF811308DF81E3005
:10C568009DF812308DF81F309DF810308DF820306E
:10C57800EB7A8DF821302B7B8DF822306B7B8DF890
:10C58800233010238DF81C608DF824303A4E8DF836
:10C598002C000DF102030A9305238DF82D30336822
:10C5A8000C930723ADF834302B6806930DF1120273
:10C5B80004AB0DF1110106A800F0D0FB07280546D1
:10C5C8000BD130680C22002100F5587001F0D0FB27
:10C5D8003368BDF80220A3F860239DF811308AF86B
:10C5E80000309DF8123089F800309DF8103088F836
:10C5F8000030189B28461C700FB0BDE8F08F9DF8DE
:10C608001330BDF81470ADF802702044C4B2F3B909
:10C6180017B3194A00201168072602464FF00C0C80
:10C62800062B1BD10CFB00FE51F80EE0BEF1000FEB
:10C6380004D00BFA00F23A4397B2012201301028D5
:10C64800EED1002A3FF472AFADF802706EE75A1EC1
:10C65800042A01D9062BDCD0062667E747FA00FE34
:10C668001EF0010FEAD00CFB00FE51F80EE0BEF1FF
:10C67800000F08BF0626E1E7F41A002038B5054682
:10C688004068FFF759FC0522841D002195F9000038
:10C69800E4B200F0E6F908B904F0FD0495F90100E8
:10C6A8000722002100F0DDF908B904F0FB04204658
:10C6B80038BD00207047000010B503780F2B0446E2
:10C6C80018D84068FFF738FC22780B4902EB420281
:10C6D8000968831C01EB820051F82220DBB21AB9E9
:10C6E80003F0FD0358B210BD032B06BF6268426019
:10C6F8000223F7E70020F6E7F41A0020022070472B
:10C708002DE9F04FDFF838810446D8F8000099B0D9
:10C718008946174600211E460122032300F558705A
:10C72800CDE90611CDE908118DF814108DF8151012
:10C73800ADF8163000F0B7F938B9D8F80020B2F8DB
:10C74800603343F00303A2F86033D8F80020637A1B
:10C758008DF8283002F55871CDE90B12394A94F951
:10C76800083012680D920DF116020F92226810928D
:10C7780062681192D4E90301A27A8DF84820012257
:10C788008DF8492013AA82E803001025227DE18A4A
:10C798008DF8293018468DF85420ADF83850FFF739
:10C7A800DFFB0AAB17930DF1150316900093314682
:10C7B800019705AB06AA10A800F0C2FB064698BB75
:10C7C8009DF81410204F013901F0A2FA1F4B1B6984
:10C7D8000393C4B24FF00C0B04F160036B44D8F818
:10C7E800000013F848AC9DF814300BFB0AFC013428
:10C7F8003946B4FBF3F203FB1244D0F87C33B0F9AA
:10C80800782350F80C00DDF80CC0E4B2E04728B1FA
:10C8180089F800A0304619B0BDE8F08F013D15F049
:10C82800FF05D9D10D26F5E70C2801BFD8F800205F
:10C83800B2F8603343F00303A2F86033EAE700BFBD
:10C84800F41A0020F01A0020400D0300C412010859
:10C85800F8B50679012E054648D90F2E48D8036841
:10C86800187A40F303000522002140B200F0F9F8DD
:10C878002B680446187A40F303100522002140B2C1
:10C8880000F0EFF8B8B1B4FA84F4640929680B7AB7
:10C89800086843F3030243F303135BB252B29A42AC
:10C8A800C8BF0124FFF748FB80F00103DBB224B1C5
:10C8B8000533D8B2F8BD0124E8E7DBB90E4F296883
:10C8C8003B6806EB460003EB80000C2201F03CFAC3
:10C8D8003A680C2303FB062320465C72B2F8601307
:10C8E8000123B3400B43A2F86033E3E70620E1E7F6
:10C8F8000320DFE70420DDE7F41A002010B40178F4
:10C9080001290ED9084B18680C234B43C418002280
:10C91800C250C4E9012200F5587010BC102200F082
:10C92800A9B8002010BC7047F41A00202DE9F04186
:10C9380086B050238DF81430037A102B074630D177
:10C948004368DD7B6DBB0224A8466426062C14D8F8
:10C958007A68535D03932A44517843EA0123039389
:10C96800927843EA02437343CDE9033863B96846D2
:10C978008DF80040FFF7C2FF0DE0CDF80C808DF870
:10C988001480CDF81080F2E703AB01A801938DF86D
:10C998000840FFF75DFF0134E4B2102C05F10305F0
:10C9A800D4D106B0BDE8F0811FB5026803791168DB
:10C9B80049B901A88DF80430FFF7A0FF78B103202A
:10C9C80005B05DF804FB02A802928DF80C30FFF761
:10C9D8003FFF042805D0052805D00028EFD0002007
:10C9E800EEE70220ECE70120EAE70000C90020B9E1
:10C9F800034B0B449856C0B27047024BF9E700BF8F
:10CA08002D0C0108ED0B0108F0B59A42069D03DBD9
:10CA18009DF914309A4220DD0020F0BD03EB43035A
:10CA280031F814C005EB830300264CFA06F7FF071C
:10CA380007D51F7A07F00F0E964502DCB2EB171FD9
:10CA48000DDD0136102E03F10C03EED10134E4B2F2
:10CA58002301DBB29842E1D8DEE70024F8E70120A1
:10CA6800DBE7884204DB9042CCBF002001207047FE
:10CA78000020704710B51409B4EB111F03464FEAA4
:10CA880011100ED391420CD202B201F00F0133F80B
:10CA98001240012000FA01F124EA010123F81210E2
:10CAA80010BD0020FCE7F0B528B100EB41050127D7
:10CAB8000020914200D3F0BD002435F802CB234674
:10CAC80007FA04F636EA0C0608BF013304F101043C
:10CAD80008BFDBB2102CF3D118440131C0B2C9B27F
:10CAE800E7E710B500B149B910BD31F8134020F897
:10CAF80013400133DCB2A242F7D8F5E70023F9E787
:10CB080082B030B504880493D2B9B3F5616F15D3F8
:10CB180049F6AF2542F21072AB4298BF4FF47A72D1
:10CB2800944238BF14466143BDE83040C3688B4225
:10CB38008CBF5B1A0023C36002B070476422EFE722
:10CB4800012C38BF0124EEE72DE9F04F8FB01546D0
:10CB5800199F03939DF8603007930C46804603F0B5
:10CB6800C7FB6A4A0590A7F5F633303BB3FBF2F3EF
:10CB7800534303F5F63B0493182313FB05430BF1CA
:10CB8800300B069300254FF0FF3A069B9C4207D1D5
:10CB9800002D14BF50464FF0FF300FB0BDE8F08FA6
:10CBA800BDF96830ADF824300999199738460897C7
:10CBB80003F02EFB2688B8F1000F5FD1B7F5616F3F
:10CBC8005AD349F6AF2242F21073974298BF4FF4F6
:10CBD8007A739E4238BF1E46642E59D1DFF83091D1
:10CBE800A060A1680CA803F035FB0D9B0093DDE95C
:10CBF80008120C9B0AA803F08CFA039A0A9B0AB93C
:10CC0800079A2AB122694A4502D1424A93420ED96B
:10CC1800414BC4F80C909F4209D90023ADF82C3041
:10CC28000B99CDF828B0584603F0F2FAA060606876
:10CC380008B9C4F80C90C4F81090B8F1000F04D0EB
:10CC480003F060FBE3680344E360D4E903329342F2
:10CC5800059B88BFE26063601B9BE1687343994250
:10CC680004D20398E8B9B8F1000F1AD001231D4483
:10CC78002375EDB2183488E76423AAE7039B0BB940
:10CC8800234BE360012EDFF8889038BF0126CEE7FA
:10CC9800B6F57A7F0ABFDFF88490DFF88490A06049
:10CCA8009FE700209342207506D85B1A9A4505F144
:10CCB800010528BF9A46EDB2B8F1000FDAD1642E0B
:10CCC800184AADF82C801DD049F6B023B6F57A7F06
:10CCD80018BF1346974281BF049A02F5A83202F59D
:10CCE800C0729B180A931A9B00930AAE96E8060036
:10CCF800199B304603F00DFA96E8030003F088FA12
:10CD08008246B7E74FF46163E4E700BF8051010052
:10CD180040771B007F5101002FEC010080A8120111
:10CD2800002E930230EC01000378032B14D14378D2
:10CD380003F00F021B098A704B7083788B80C278CE
:10CD480043EA02238B800379C3F3021203F00F0333
:10CD5800CA700B7005207047002070472DE9F34713
:10CD68009A464379057990F907609146044690F907
:10CD780006208846D3B190F90870002D37D00F2AC5
:10CD88001BD194F909200F2E27D194F90A00072DF9
:10CD980002D1002F08BF012788F8002089F8000079
:10CDA80028468AF8007002B0BDE8F08790F90B7049
:10CDB80090F9092090F90A60DFE7A369019394F9D3
:10CDC8001530009394F914302169207BFFF71CFE7D
:10CDD8000028D8D105F0FD05D5E794F91D00B0422B
:10CDE800D5DC94F91C30B34203DA05F0FB05304674
:10CDF800D2E73046CBE70000024B03FA00F0B0FB65
:10CE0800F1F0704740420F004FF4FA53B3FBF0F0D3
:10CE1800704730B54FF47A750C1F6A4300FB042243
:10CE280052001EBF00F1FF341219B2FBF0F291421A
:10CE380038BF1146039A1160820048431CBF013075
:10CE480040084FF47A71121A01FB1323002BCABF52
:10CE580003F2E73393FBF1F1B3FBF1F1049B1960A3
:10CE680030BD38B5400014460D46F4F7CFFD0146F5
:10CE78002846F4F719FD2146F4F716FDF4F708FCE7
:10CE880003F0D6FCF4F7E4FC40B238BD2DE9F74FC7
:10CE9800019300239C469E46048A1E01F6B2B442C2
:10CEA80046D906EB46054FEA4309AD00002447681A
:10CEB80037F809702741FF0729D5876807EB050A66
:10CEC8007F5927B3077837B9476927B137F8097009
:10CED8002741FF071BD59AF8087090F901B047F36E
:10CEE80003084FFA88F8D84511DC47F303177FB2D7
:10CEF8005F450CDB9AF8097007EB4708C76807EB32
:10CF0800C8073F7D5FB90CF1010C5FFA8CFC013456
:10CF1800102C05F10C05CAD10133DBB2BCE70EF1C8
:10CF2800010706EB040801F80E805FFA87FEEEE7BA
:10CF3800019B82F800E083F800C003B0BDE8F08FE1
:10CF48002DE9FF4704464068DDE90C671D468A461F
:10CF5800914603F0D7F923681B1A3B604FF000088D
:10CF68000123337085F80080636813B12368834216
:10CF780024D8D4F81CC0CAF80080A3699CF800E043
:10CF88000393D4E9030101AB83E80300237D0093F5
:10CF9800DCF80C10237A627A7046FFF7D5FD334629
:10CFA80038602A46E0694946FFF770FF2B782BB1B5
:10CFB800C7F80080002004B0BDE8F0873378002B64
:10CFC8000CBF0C200B20F6E737B590F9002090F93C
:10CFD8000250954204460FD0013A52B295420BD006
:10CFE800A368019394F9013000936168E0782B46B7
:10CFF800FFF70AFD0028EFD0104603B030BD884285
:10D00800B8BF08467047000051F82000054B984209
:10D0180005D0054BC31A58425841400070470120BB
:10D02800704700BF90D0030020A1070005281FB556
:10D038000ED80C4B53F820300093CDE901120A4B5F
:10D0480001220021022002F06BFE05B05DF804FB0E
:10D05800CDE90012054B01220021022002F060FEFA
:10D06800F3E700BF1C0D0108B00C0108CF0C010844
:10D0780007B5054BCDE9000101220021022002F08D
:10D088004FFE03B05DF804FBEB0C010810B510224D
:10D0980004460021F13000F06BFE0021C4F81411A1
:10D0A8002046F022BDE8104000F062BE0246084665
:10D0B800102100F0A5B92DE9F0430446D0F8140179
:10D0C80085B00E46154604F2011988B3C0F1100860
:10D0D8009045474628BF1746BAB2484400F034FE88
:10D0E800D4F814313B440F2BC4F814312DD9A8457A
:10D0F8002BD204F1F00304F5807113F8012F187C8A
:10D108008B4282EA00021A70F7D104F1F10810226A
:10D118004146684600F018FE22466946684600F017
:10D12800F1F910226946404600F00EFE3E44ED1B20
:10D1380004F5807804F1F107102D09D8AAB2314618
:10D14800484600F001FEC4F8145105B0BDE8F0836C
:10D1580004F1F003711E13F8012F11F8010F434574
:10D1680082EA00021A70F6D110223946684600F0A9
:10D17800EBFD22466946684600F0C4F9102269466C
:10D18800384600F0E1FD1036103DD5E7F0B589B01E
:10D198000C46102200210546684600F0E9FD2246AB
:10D1A8006946684600F0AEF99DF90030002B6A46E2
:10D1B8004FF0000143DA137812F8010F01315B00D8
:10D1C80043EAD0130F2902F8013CF4D19DF80F303F
:10D1D8005B0083F08703D4F81401DBB210288DF8C4
:10D1E8000F303BD104F58073694604F5887013F855
:10D1F800016F11F8012B984282EA06021A70F6D1E3
:10D2080004F1F00304F5807113F8012F187C8B42A8
:10D2180082EA00021A70F7D110220DEB020004F125
:10D22800F10100F091FD2246294604A800F06AF9B0
:10D2380010220021684600F09BFD09B0F0BD13786C
:10D2480012F8010F01315B0043EAD0130F2902F8ED
:10D25800013CF4D19DF80F305B00BCE79DF900302C
:10D26800002B6A464FF0000137DA137812F8016F85
:10D2780001315B0043EAD6130F2902F8013CF4D1CF
:10D288009DF80F305B0083F08703471CDBB28DF8F5
:10D298000F30102F04EB0003C0F10F064FF080028F
:10D2A80088BF002600F5817083F8012100213246ED
:10D2B80020443E4403F076FAC4F8146104F5807300
:10D2C800694604F5887013F8016F11F8012B98422C
:10D2D80082EA06021A70F6D192E7137812F8016F03
:10D2E80001315B0043EAD6130F2902F8013CF4D15F
:10D2F8009DF80F305B00C8E70A7803785340037045
:10D308004A784378534043708A78837853408370CF
:10D31800CA78C3785340C3700A79037953400371BC
:10D328004A794379534043718A79837953408371A9
:10D33800CA79C3795340C3710A7A037A5340037296
:10D348004A7A437A534043728A7A837A5340837283
:10D35800CA7AC37A5340C3720A7B037B5340037370
:10D368004A7B437B534043738A7B837B534083735D
:10D37800CA7BC37B5340C373704710B50B781478CE
:10D388006340037054784B786340437094788B788B
:10D3980063408370D478CB786340C37014790B7979
:10D3A8006340037154794B796340437194798B7965
:10D3B80063408371D479CB796340C371147A0B7A53
:10D3C80063400372547A4B7A634043728B7A947A3F
:10D3D80063408372D47ACB7A6340C372147B0B7B2D
:10D3E80063400373547B4B7B63404373947B8B7B19
:10D3F80063408373CB7BD27B5340C37310BD000063
:10D40800A1F11003DBB2102B2DE9F047044604D834
:10D418003A4820FA03F3DB0705D4002382F8F030FA
:10D42800FF20BDE8F087561E254615F8013B06F893
:10D43800013F631B0B4413F0FF00F6D101F11C03FD
:10D448009B005FFA83FCC3F30313013BDFF8B09042
:10D4580082F8F030884653184FF0010EB8FBF1FA05
:10D4680001FB1A8A1AF0FF0A13F8047C13F8036CFC
:10D4780013F8025C13F8014C30D119F806A019F81A
:10D48800056019F8045019F807404FEADE1707EB52
:10D4980047078EEA0A0A07EBC7074FEA4E0EFFB2A4
:10D4A8005FFA8EFE87EA0E0E574692F800A087EACA
:10D4B8000A071F7057787E405E70967875409D7099
:10D4C800D57808F104085FFA88F86C40C445DC7028
:10D4D80002F1040203F10403C0D8A2E71829E4D931
:10D4E800BAF1100FE1D1DFF818A01AF807701AF88E
:10D4F80006601AF805501AF80440D6E70101010041
:10D50800340F01082DE9F04FA3B092F8F0301D91C7
:10D518001B920193002B00F0538101461EA8FFF7D0
:10D528002CFF1B9BA74CA84DA84E10330293002339
:10D5380003939DF87C0004909DF886000590205C7C
:10D5480006909DF87B000790205C089004989DF851
:10D5580081C0205C099014F80C000A909DF88000A6
:10D568000B909DF885009DF878809DF87DE09DF8EA
:10D5780082A09DF887900C909DF87A00029B1C93DE
:10D5880014F80A2014F8093014F8081014F80E706A
:10D598000D90205C0E909DF87F000F90205C1090FD
:10D5A8000B98205C11900C98205C12909DF88400D8
:10D5B80013909DF8790014909DF87E001590205CDA
:10D5C80016909DF883001790205C18901398205CA3
:10D5D80019901498205C1A900398013003900298CF
:10D5E800DDF804B0103002909DF80C00834536D861
:10D5F8008DF878108DF87A2009990E9A8DF87C109C
:10D608008DF882201199069A8DF880108DF87E2069
:10D618001999169A8DF884108DF886200A99189A07
:10D628008DF87D108DF887201299109A8DF87B302F
:10D638001B9B8DF881108DF883201A99089A1D98E4
:10D648008DF885108DF87F201EA903EB0B128DF83D
:10D658007970FFF792FE002023B0BDE8F08F15F82F
:10D6680008B082EA03008BEA000016F80EB080EAE0
:10D678000B008DF8780015F80E004B40434016F863
:10D688000A0043408DF8793081EA070315F80A103B
:10D69800594016F80930594016F808308DF87A10B4
:10D6A8007A40534015F8092053408DF87B30089A8A
:10D6B800069B5340049AAA5C534016F80C2053402A
:10D6C8008DF87C30DDE908325A4015F80C305340AB
:10D6D800059AB25C53408DF87D30DDE909325A4035
:10D6E800059BEB5C5340079AB25C53408DF87E3043
:10D6F800069B0A9A5340049AB25C5A40079BEB5C1B
:10D708005A408DF87F200E9B109A53400B9AAA5CC2
:10D7180053400C9AB25C53408DF88030DDE91032EA
:10D728005A400C9BEB5C53400D9AB25C53408DF809
:10D738008130DDE911325A400D9BEB5C53400F9A62
:10D74800B25C53408DF88230129A0E9B53400B9A6C
:10D75800B25C5A400F9BEB5C1C995A408DF88320B1
:10D76800169B189A5340139AAA5C5340149AB25CB9
:10D7780053408DF88430DDE918325A40149BEB5C35
:10D788005340159AB25C53408DF88530DDE9193263
:10D798005A40159BEB5C5340179AB25C53408DF886
:10D7A80086301A9A169B5340139AB25C5340179AC4
:10D7B800AA5C1EA853408DF88730FFF79DFDB8E698
:10D7C800FF2049E7340F0108340E0108340D010821
:10D7D80008B538B1044A05491060D82200F0B4FAF7
:10D7E800002008BD0220FCE7F81A00206414010894
:10D7F8000A4B1A6870B5002302F1180503EB0314ED
:10D808002E5D864204D1183422440A60002070BD7F
:10D8180001330B2BF2D10320F9E700BFF81A0020DF
:10D828002DE9F041CCB00646DDF8488117461C4684
:10D838000D4631B3B8F1000F23D006A8FFF726FC38
:10D84800204601A9FFF7D4FF0446B0B9019906A8FC
:10D858000131FFF72BFC26B11022314606A8FFF74D
:10D868002AFC3A46294606A8FFF725FC06A902A87D
:10D87800FFF78CFC029BC8F8003020464CB0BDE88E
:10D88800F0810224F9E7000030B595B013A90446E9
:10D89800FFF7AEFF002830D11B4B0C2101FB00F233
:10D8A800D5189A5CA2422AD1139B1A7C1092DA7B73
:10D8B8000F929A7B0E925A7B0D921A7B0C92DA7A0F
:10D8C8000B929A7A0A925A7A09921A7A0892DA7913
:10D8D80007929A7906925A7905921A790492DA7817
:10D8E80003929A7802925B7801930022AB680093C6
:10D8F8001146064B022002F013FA15B030BD013074
:10D908000B28CBD1F9E700BFAC110108341001088E
:10D9180010B40B2B019C03D8019410BCFFF780BFF7
:10D92800032010BC704730B50D4685B0144601463B
:10D9380068B103AA002000922A460390FFF770FFFF
:10D9480018B90398001B18BF012005B030BD02208C
:10D95800FBE72DE9F0430D46BFB0144699468046D3
:10D9680020B31BB311F00F0122D1F02201A800F05F
:10D97800FFF920466946FFF73BFF044648B900987F
:10D9880001AA10210130FFF73BFD2E46AF1BFFB265
:10D998001EB920463FB0BDE8F08301AA09EB070194
:10D9A80008EB0700FFF7AEFD103EEFE70224F0E7B3
:10D9B8000524EEE7F0B5184E3468024685B00846EF
:10D9C800002304F1180103EB03154F5D97421ED1A4
:10D9D8000D2A05F1190513D10023CDE90033CDE94E
:10D9E80002330C2210216B46FFF7B3FF0446306860
:10D9F80010226946284400F0A7F9204605B0F0BD7A
:10DA080001461022601900F09FF90024F5E7013360
:10DA18000B2BD8D10324F0E7F81A002009B1FFF73F
:10DA2800C9BF022070471FB51446A0B10C2A01D106
:10DA38000B2912D10023CDE90033CDE902330A4680
:10DA48006B461021FFF785FF18B969462046FFF796
:10DA5800B1FF04B010BD0220FBE70320F9E7F8B5D9
:10DA68001E46DDE907479DF818505BB354B34FB322
:10DA7800212D29D819462A46204600F065F90122A9
:10DA8800631C691EB018FFF764FFF8B9E37ADB0975
:10DA98003B70EBB96319204613F8012C13F8021CEC
:10DAA800120642EA014213F8041C0A4313F8031C45
:10DAB800012342EA0122291FFFF735FF003818BF6A
:10DAC8000120F8BD0220FCE70520FAE70720F8E767
:10DAD8000420F6E710B5044628B1044B5B69984763
:10DAE8002060002010BD0220FCE700BFC41201081E
:10DAF80008B5014630B1044B0822186800F024F933
:10DB0800002008BD0220FCE7F81A002008B530B153
:10DB1800044B0822196800F017F9002008BD0220FC
:10DB2800FCE700BFF81A00207FB5124E0023044618
:10DB380002A801930D46FFF7E9FF33685B6901937B
:10DB48006CB102AA082312F8011B41B9013B13F07A
:10DB5800FF03F8D102A8A04702A8FFF7C9FF35B113
:10DB6800019B23B901A8A8473368019A5A6100208C
:10DB780004B070BDF81A002008B5014638B1054B4D
:10DB880018680822104400F0DFF8002008BD0220C1
:10DB9800FCE700BFF81A002008B538B1044B196833
:10DBA8000822114400F0D0F8002008BD0220FCE74C
:10DBB800F81A0020034B1B6802280CBF1961596131
:10DBC80000207047F81A002049B1064B1B68D3E9BA
:10DBD8000423022808BF13460B6000207047022068
:10DBE800704700BFF81A002030B58FB000240546F2
:10DBF8000CA80994FFF78AFF9DF8373007939DF822
:10DC0800363006939DF8353005939DF834300493EB
:10DC18009DF8333003939DF8323002939DF83130EC
:10DC280001939DF830300093224621461E4B022076
:10DC380002F076F80AA8FFF7AFFF9DF82F30079398
:10DC48009DF82E3006939DF82D3005939DF82C30C5
:10DC580004939DF82B3003939DF82A3002939DF886
:10DC6800293001939DF82830009322460F4B214616
:10DC7800022002F055F809A92846FFF7A5FF9DF8EC
:10DC8800243003939DF8253002939DF826300193A4
:10DC98009DF8273000932246054B2146022002F0CA
:10DCA8003FF80FB030BD00BF90100108CE1001083A
:10DCB8000C11010808B50020FFF7E6FD0120FFF769
:10DCC800E3FD0920FFF7E0FD0820FFF7DDFD002058
:10DCD800FFF78AFF002008BD10B504460B20FFF7A8
:10DCE800D3FD0C20FFF7D0FD0920FFF7CDFD08205C
:10DCF800FFF7CAFD0A20FFF7C7FD2046FFF774FFAC
:10DD0800002010BD014B1860704700BF3C01002087
:10DD18000B4A30B514680B4D43F2390305FB043345
:10DD28001360091A6FF00042B3FBF2F2C2EBC27241
:10DD380001319B1A93FBF1F201FB1233184430BDF9
:10DD48003C0100206D4EC64101380A44914200D181
:10DD5800704711F8013B00F8013FF7E710440A4407
:10DD6800914200D1704711F8013B00F8013DF7E7F7
:10DD780002F018BD30B530B10A4D01444FF0FF3301
:10DD8800814201D1D84330BD10F8012B53400822FD
:10DD980043F30004013A2C4092B284EA5303002A68
:10DDA800F6D1EDE72083B8ED01207047054B4FF41D
:10DDB80000529A62044B1B6813B15B6803B11847A1
:10DDC800704700BF00040048881B0020054B4FF433
:10DDD80080529A62044B1B6813B1DB6803B1184781
:10DDE800704700BF00040048881B002001207047CE
:10DDF8000120704701F03EB901F02CB910B501F0CF
:10DE08000FFE0E21044640F61F1001F023F92046AC
:10DE1800012101F0EFFDBDE8104001F0CDBA00008E
:10DE280070B50C4E01EB40030D46B3654FF6FF711C
:10DE3800002304461A46084601F054FB96F856009B
:10DE4800002101F0D7FD29462046BDE8704001F0C9
:10DE58008BBA00BF2C1B002010B5044601F0A0FEB1
:10DE680001281CD101F0A4FE34B11248214602F069
:10DE78000BFB104802F0CEFA0F4C104B00214FF468
:10DE88008052A1659A6194F8560001F0B3FD637859
:10DE98006BB16FF07F40BDE8104001F049BA002334
:10DEA80040F262211A46084601F01CFBDCE7A06834
:10DEB8008001F0E7FC1A00202C1B00200004004819
:10DEC800002001F0B5B9000008B501F0BDF804382C
:10DED800C0B2032896BF024B0020185C08BD00BFE3
:10DEE8008E12010808B501F0B0FD033008BD01F03D
:10DEF8003FB901F0FFB808B501F0F6FC08BD000015
:10DF080038B50D46144601F053FB284601F088FD4C
:10DF18000E21054640F61F1001F09CF82846012105
:10DF2800074D01F067FD01F047FA4FF47A7161433C
:10DF3800284602F0A9FA2846BDE8384002F06ABA35
:10DF4800141B002001F034BB08B5084B002193F8DE
:10DF5800560001F04FFD00234FF4C0711A460846E1
:10DF680001F0C0FABDE8084001F01ABA2C1B0020E5
:10DF780010B5044601F014FE01281CD101F018FE6A
:10DF880034B11248214602F07FFA104802F042FAF2
:10DF98000F4C104B00214FF48052A1659A6194F800
:10DFA800560001F027FD63786BB16FF07F40BDE844
:10DFB800104001F073B9002340F262211A46084666
:10DFC80001F090FADCE7A0688001F0E7FC1A002075
:10DFD8002C1B00200004004808B54FF0040001F095
:10DFE8000DF9BDE808400220F4F776BC08B5002317
:10DFF8001A461946184601F075FABDE8084001F0BE
:10E0080063B900001D4B73B51D4D186000241D48F1
:10E018006C70C5E90144AC6501F08EFAAC8101F081
:10E02800F9F92146204601F041FC2146042201204D
:10E0380001F0F2FA144E154D4FF6FF7123462246B1
:10E04800084601F04FFAFFF7C7FF2246104B00942D
:10E058004FF0FF31304602F031F90E4B0094224662
:10E068004FF0FF31284602F029F9304602F084F9D2
:10E07800284602B0BDE8704002F07EB9881B002037
:10E088002C1B002041F00008141B0020FC1A002063
:10E09800B5DD0008D5DD00080128084805D1084B82
:10E0A800C17719700E3001F09DBB437D012B03D160
:10E0B800034B81751970F5E7704700BF2C1B0020D2
:10E0C800400100200D4B10B5044618735873012009
:10E0D80000F016F85CB134214FF4E86000F0BAFFA4
:10E0E8004421BDE8104040F2417000F0B3BF142154
:10E0F8004FF4E86000F0AEFF2421F2E72C1B00206B
:10E1080038B5114C0546207001F057FD052D04D88F
:10E11800DFE805F0090B03171709032001F066FA79
:10E128000023637338BD0020F8E7012001F05EFA90
:10E13800207B637B8342F5D06073BDE83840FFF7EE
:10E14800C1BF0220EAE700BF2C1B00202DE9F043E5
:10E158001E4687B000230546CDE901330C46174615
:10E1680001F01DFD032D5BD8DFE815F07A00C10032
:10E178000C010400A27C082A69D8A16801A801F052
:10E18800D5FE2168002962D042F210729142E37CE8
:10E19800874D50D80322AA7385F83820E96385F89B
:10E1A80044304FF002086368A17DDB002B82042312
:10E1B800AB74A37CDB00EB7402294FF000032B75D2
:10E1C800637D02D0227D022A46D103F10F02D2B22A
:10E1D800012A01D9012B3AD1764B774A1968039461
:10E1E8004FF0010903A88DF8149001F0D5FC70BB1D
:10E1F800287685F817906875FFF762FE4046FFF7A6
:10E208007FFF6E4801F082FA6D4801F0EBFA01A831
:10E2180000F080FF208A00F051FFA08900F096FFEF
:10E22800384601F0FDFB624C84F8560001F0BCFC56
:10E23800666000200DE04FF00008E963890885F862
:10E248000E8085F8388085F844302964ABE74FF0B4
:10E25800FF3007B0BDE8F083EB7529766A75CBE728
:10E268002368002BF3D0A27C082AF0D8504DA1686F
:10E2780001A801F05BFE002385F838302268EA63C4
:10E28800E27C85F84420A269AB732A646268D200F4
:10E298002A820422AA74A27C2B75D200EA74A27D79
:10E2A800022A02D0237D022B1CD1627D02F10F03CA
:10E2B800DBB2012B01D9012AC9D13E4B3E4A19686C
:10E2C80003944FF0010803A88DF8148001F064FC52
:10E2D8000028BCD1287685F817806875FFF7F0FD0F
:10E2E80000208CE7617DE9752A766B75F6E7304D7D
:10E2F800012185F83810227885F85020637885F850
:10E308005130A37885F85230E3788B4202D0022B43
:10E3180003D03BB985F8533004E00B3A012A29D8D9
:10E3280085F853104FF0010885F80E80A388AB8359
:10E33800A379AB77E37985F82030237A85F8213003
:10E34800FFF7BEFD4046FFF7DBFE1C4801F0DEF993
:10E358001B4801F047FA95F85130062B40F6890022
:10E368000AD100F087FE00F0FB0140F6890000F0BA
:10E3780071FE55E70023CDE700F07CFE40F0040174
:10E38800C9B2F2E72368013BB3F57A7FBFF45FAF08
:10E398000320FFF7B5FE0648022380F838302368CB
:10E3A8008364162380F84C30383001F0AFF937E732
:10E3B8002C1B0020881B0020141B0020641B00203D
:10E3C8003A1B0020F0B51E4687B00023CDE9013383
:10E3D800144607460D4601F0E2FB002C724C16BFAE
:10E3E800012300230026637027B1012F7AD0002073
:10E3F80007B0F0BDAB68002B00F0D280EB68002BB3
:10E4080000F0CE80AA7F082A00F2CA80296901A8F4
:10E4180001F08CFD2868003818BF012000F0D6FFF5
:10E4280084F83870AB68E36395F8203084F844309A
:10E43800686801F057FBA77384F84500EB68DB00B8
:10E448002382EB7FA374AB7FDB00E37495F8213064
:10E45800237595F82230002B3ED12A7D95F824109B
:10E46800A275022995F8232001D0022B36D102F19A
:10E478000F03DBB2012B02D9012A40F0918000235F
:10E488008DF81430494B4A4A1968049503A801F0DD
:10E4980083FB002840F0848001232076E3756075B3
:10E4A800FFF70EFD0020FFF72BFE424801F02EF982
:10E4B800414801F097F901A800F02CFEA88B00F064
:10E4C800FDFD288B00F042FE4FF4FA53AA6873430F
:10E4D800B3FBF2F3A3608AE7FF22BFE7E275217678
:10E4E8006375DDE72B8E002B5AD095F83230A86A79
:10E4F800012B0CBF2F7DFF27003818BF012000F02B
:10E5080065FFF0B200F06EFF012184F8381095F82D
:10E518002C2084F8502095F82D3084F8513095F847
:10E528002E3084F8523095F82F308B4202D0022BCF
:10E5380003D03BB984F8533004E00B3A012A27D8BA
:10E5480084F853102B8EA38395F83230A3770126D5
:10E55800AB8E2384A673E777FFF7B2FC3046FFF74C
:10E56800CFFD144801F0D2F8134801F03BF994F8B4
:10E578002130B34240F236700CD100F07BFD00F040
:10E58800FB0140F2367000F065FD4FF6FF73A1E71E
:10E598000023CFE700F06EFD40F00401C9B2F0E7B8
:10E5A8004FF0FF3024E700BF2C1B0020881B002001
:10E5B800FC1A0020641B00203A1B00202DE9F04FB4
:10E5C80085B082460E9DBDF840809DF844709DF848
:10E5D8004890019193461E4601F0E1FABAF1010F05
:10E5E800524C54D0BAF1040F00F09180BAF1000FE8
:10E5F8003AD10B22304684F8442084F838A0E563E9
:10E6080001F070FA4FEAC803B9F1000F238241F60E
:10E61800040363820CBF0123F223E37587F001072B
:10E628000123237684F84500C4F840B084F80EA08E
:10E6380084F814A06775FFF743FC5046FFF760FDA8
:10E6480004F1380001F062F804F10E0001F0CAF894
:10E65800374A1068516802AB03C302A800F05AFD9C
:10E6680040F2FF1000F02AFD019801F0D9F90E21BF
:10E6780084F8560040F61F1000F0ECFC94F85600A1
:10E6880001F092FA169B636005B0BDE8F08F294946
:10E6980084F838A0EAB2895D84F8502076BB0B3D37
:10E6A800012D8CBF00250125053A012A04D8B8F1AF
:10E6B8000C0F38BF4FF00C081F4B9DF83C201B78FF
:10E6C80084F85350E37701259DF8543084F85110AD
:10E6D80084F8522084F82130A573A4F81C80A77709
:10E6E80084F82090FFF7ECFB2846FFF709FD134854
:10E6F80001F00CF8124801F075F8B5E7012E04D1C5
:10E70800A5F10C035D425D41CEE70025CCE75046FC
:10E71800FFF7F6FC022384F8383004F1380016239A
:10E72800A56484F84C3000F0F1FF9DE72C1B002015
:10E73800A0090108C012010840010020641B002044
:10E748003A1B00202DE9F04F87B0DFF8B4B29DF8EE
:10E7580064A09DF84C90029314469DF854309DF89F
:10E768005020BDF84880039205468BF801A0BDF8FB
:10E77800446001930F4601F012FABAF1000F18BF76
:10E788004FF00008DFF87CA2039AB9F1000F08BF28
:10E79800FF22012D8AF8002000F0C880052D48D0FE
:10E7A800002D40F0C080284600F010FE0B223846AD
:10E7B8008BF844208BF83850CBF83C4001F092F9A4
:10E7C800019B8BF8450041F60402002BABF81220A0
:10E7D8009AF800208BF816200CBF0122F2228BF841
:10E7E8001720F600012289F001098BF818208BF810
:10E7F8000E50ABF810608BF814508BF81590FFF79B
:10E808005FFB2846FFF77CFC0BF1380000F07EFF29
:10E818000BF10E0000F0E6FF7B490868496804AA7E
:10E8280003C204A800F076FC40F2FF1000F046FC9A
:10E8380071E0012000F0CAFD09224FF000098BF8B1
:10E84800442038464FF44872CBF840208BF8389073
:10E85800CBF83C4001F046F94FF48052ABF8122057
:10E868009AF800208BF845008BF8162028460122DC
:10E87800F6008BF817208BF80E90ABF81060ABF809
:10E8880014908BF81890FFF73BFC0BF1380000F060
:10E898003DFF0BF10E0000F0A5FF5B498868C968D1
:10E8A80004AA03C204A800F035FC40F2FF1000F0EF
:10E8B80005FC40F6B80000F0DDFB00F0EF0140F683
:10E8C800B80000F0C7FB042140F6B90000F0C2FB15
:10E8D80040F69B0000F0CEFB00F0E30141F0080198
:10E8E80040F69B0000F0B6FB40F2D16000F0C2FB9E
:10E8F80040F01801C9B240F2D16000F0ABFB40F221
:10E90800AC6000F0B7FB00F08F0141F0500140F21D
:10E91800AC6000F09FFB4FF4FA5202FB08F2B2FB26
:10E92800F4F2CBF8082007B0BDE8F08F002000F023
:10E938004DFD36498BF83850E2B2C95D8BF850204E
:10E94800002F4DD10B3C012C8CBF00240124053A2B
:10E95800012A02D80C2E38BF0C26029B9AF80020F8
:10E968008BF852308BF85340019B8BF81F20012401
:10E978009DF860208BF821208BF851108BF82030FF
:10E988008BF80E40ABF81C608BF81E90FFF798FAD6
:10E998002046FFF7B5FB1E4800F0B8FE1D4800F002
:10E9A80021FF5FFA88F000F01DFD40F6A30000F09B
:10E9B80061FB00EA040140F6A30000F04BFB9BF862
:10E9C8002120A24240F2367013D100F053FB00F030
:10E9D800FB0140F2367000F03DFB4FF6FF72A0E7F6
:10E9E800012F04D1A4F10C035C425C41AFE7002481
:10E9F800ADE700F03FFB40F00401C9B2E9E700BF12
:10EA08002C1B002040010020A0090108C0120108A9
:10EA1800641B00203A1B0020F0B58BB00D4604465D
:10EA280017461E46FFF74CFA0020FFF769FB204601
:10EA380000F0BEFD00240123CDE9084303234FF471
:10EA4800167229462046CDE90644CDE90444CDE9AD
:10EA58000244CDE900532346FFF774FE2046FFF732
:10EA680087FAFFF73FFAF3F737FF01F041FC044656
:10EA7800204601F047FCB04205D30124FFF720FAF5
:10EA880020460BB0F0BD00F02FFF8742F0DA0024DB
:10EA9800F4E70000F7B500230C4640F201211A46BE
:10EAA8000646084600F01EFD644B654D4FF40052C3
:10EAB8009A6195F85600012100F09CFF2B78012BF4
:10EAC80040F6890013D195F85130062B0FD100F08C
:10EAD800D1FA00F0FB0140F6890000F0BBFA2B7870
:10EAE800042B6CD8DFE803F0524B527F090000F08A
:10EAF800C1FA40F00401C9B2EDE7524A731E10464C
:10EB0800C6F101074FF0000CF9188C426FDC0022A7
:10EB1800E7001346BA4271D19A0142EAC3125B0177
:10EB280083F020031343661C0355F6B202234648BC
:10EB3800AB73AE7600F056FE0021F12000F08AFAA1
:10EB48000021F02000F086FAAB6C642B70D17021A4
:10EB5800F32000F07FFA1D21F22000F07BFAE1009B
:10EB68008C1CF420090A00F075FA04F0FE01F52067
:10EB780000F070FA33486FF07F4231461DE0EC77C1
:10EB8800314800F02FFE0022214615E001F008F878
:10EB98000128074625D121460DF10702304601F02C
:10EBA80004F80446A0B99DF807302748AB7500F073
:10EBB80019FE9DF807102246304600F065FB69688B
:10EBC800224801F061FC214801F024FC002006E005
:10EBD8001F4B3A460021022001F0A2F8032003B09F
:10EBE800F0BDAC75CCE70223AB73AC76C8E713F87D
:10EBF800011FC943197002F801CB85E7D1106FEAEC
:10EC0800020C715C0CF0070C013241FA0CF101F0B6
:10EC180001014FEAE20C4B40D14310F80CE001F03F
:10EC2800070103FA01F141EA0E0100F80C1071E73F
:10EC3800E121F32000F00EFA04218DE700040048DA
:10EC48002C1B00208C1B00203A1B0020141B0020CA
:10EC580030120108F0B5BDF814409DF818709DF801
:10EC68001CE09DF8205040B1012814D00122002357
:10EC780098180138B0FBF2F0F0BD87F00107E30007
:10EC880003EBC70318330EEB450503EBC5034FF43D
:10EC98007A714B43ECE7501F012803F1040302D8B3
:10ECA8000C2C38BF0C24D1B9A2F10B0CBCF1010F0C
:10ECB8008CBF4FF0000C4FF0010C2801002F00EB27
:10ECC800CE000CBF14250025A0EB8200062A4FEACF
:10ECD80082062844A2F102070DD8354610E0012922
:10ECE80006D1A2F10C00D0F1000C4CEB000CE4E7CB
:10ECF8004FF0000CE1E70830BCF1000FEDD0BD008B
:10ED08000028ACBF2E182E1C701E90FBF5F003FBDC
:10ED18000044094B062A5A5C8CBF0C340E340A2A6C
:10ED280009D8A30001334FF47A71BB404B43034920
:10ED380051F822209CE7FFDEC01201089412010856
:10ED480008B5094B012193F8560000F053FE4FF423
:10ED5800D7602D2100F07EF900F033FBBDE80840B4
:10ED6800024800F07BBA00BF2C1B0020FFFF0F00F9
:10ED780073B5A44CB4F854300025202B8DF80350FB
:10ED8800019500F01B8114D8082B0DD87BB1013BED
:10ED9800072B0CD8DFE813F042005B000B00CD0016
:10EDA8000B000B000B00FD00102B00F0008102B0DF
:10EDB80070BDB3F5807F00F0988011D8402B00F02B
:10EDC8001081802BF3D1284600F032FA8E4B1B6855
:10EDD800002BECD09B69002BE9D028469847E6E742
:10EDE800B3F5007FE3D1894B01222946022000F0C8
:10EDF80097FF00F029F9042840F08580844B854866
:10EE08004FF400529A6201F0B7FA284600F010FA5F
:10EE18007D4B1B68002BCAD05B6814E07C4B7D4897
:10EE28004FF400529A6201F0A7FA002000F000FAAD
:10EE380000F0B8FE012801D100F0BDFE724B1B683E
:10EE4800002BB4D01B68002BB1D09847AFE7704BAC
:10EE580071484FF480529A6201F08EFA657895B93C
:10EE6800284600F0E5F9294640F6021000F0F2F8CD
:10EE780040F6441000F0FEF840F00201C9B240F636
:10EE8800441000F0E7F8FF220DF1030163485E4DDE
:10EE980000F05AFD624800F071FD2B68002B86D007
:10EEA8009E68002E83D094F82430012B08D194F961
:10EEB800313094F930209DF803105848B04776E770
:10EEC800E06B01A900F022FE019B9DF80310534856
:10EED8004FF47A7203F5FA7393FBF2F32A685BB284
:10EEE800956894F92920A84761E7284600F0A0F919
:10EEF800454B1B68002B3FF45AAF9B69002B3FF42E
:10EF080056AF01206AE700F09FF805287FF44FAF5D
:10EF18003F4B41484FF480529A6201F02DFA28463F
:10EF280000F086F9384B1B68002B3FF440AFDB68D4
:10EF380089E700213B4B0122022000F0F1FEA16D80
:10EF480000293FF434AFC1F3074140F6031000F045
:10EF580081F894F8591040F6041000F07BF894F802
:10EF6800581040F6051000F075F840F6021000F051
:10EF780081F840F00101C9B240F6021000F06AF8C9
:10EF8800002340F262211A460846A36500F0AAFA57
:10EF98000DE7254B01220021022000F0C1FE00F000
:10EFA800FFFD01287FF403AF00F006FEFFE61F4BCC
:10EFB80001220021022000F0B3FEF8E6164801F015
:10EFC800DBF9607808B900F033F90F4B1B68002BA8
:10EFD8003FF4EDAEDB68002B3FF4E9AE9847144BE5
:10EFE800E6E7144B01222946022000F099FE6078DA
:10EFF80008B900F01DF9044B1B68002B3FF4D7AE8D
:10F008001B6920E72C1B0020881B002045120108E3
:10F0180000040048141B0020FC1A00208C1B002050
:10F02800501B002059120108621201086C120108D5
:10F03800751201087E120108024BA3F85400FFF76D
:10F0480097BE00BF2C1B0020014B1878704700BFEB
:10F058009A1C002007B501238DF807100DF107024F
:10F0680001460348F7F7BEF803B05DF804FB00BF9C
:10F078003802002007B5012301460DF107020448B4
:10F08800F7F7E9F89DF8070003B05DF804FB00BF47
:10F098003802002010B50446F4F724FE01280CD1EC
:10F0A80040F62310FFF7E6FF00F0F901214340F690
:10F0B8002310BDE81040FFF7CDBF10BD10B50C4BB5
:10F0C8001B7804469BB94FF4D760FFF7D3FFC4F30E
:10F0D800002100F0FE0001434FF4D760FFF7BAFFAC
:10F0E800E1B240F2B960BDE81040FFF7B3BF10BD10
:10F0F800991C002010B51346EFF3108472B60A4627
:10F1080001460348F7F76EF884F3108810BD00BF76
:10F118003802002008B5014608224FF4D860FFF7EE
:10F12800E9FF002008BD000007B5074B1B7840BA6F
:10F13800ADF804002BB9022201A940F2BC60FFF728
:10F14800D9FF03B05DF804FB991C002007B5074BF5
:10F158001B7840BAADF804002BB9022201A940F28D
:10F16800BE60FFF7C7FF03B05DF804FB991C0020E1
:10F1780010B51346EFF3108472B60A4601460348E9
:10F18800F7F769F884F3108810BD00BF3802002033
:10F1980010B51346EFF3108472B60A4601460348C9
:10F1A800F7F74BF984F3108810BD00BF3802002030
:10F1B8000A4601460020FFF7EBBF000010B51346D2
:10F1C800EFF3108472B60A4601460348F7F768F968
:10F1D80084F3108810BD00BF3802002010B5134614
:10F1E800EFF3108472B60A4601460348F7F76EF843
:10F1F80084F3108810BD00BF3802002013B5044600
:10F208000020F4F749FD0220FFF744FF04F007044B
:10F2180001220DF1070184208DF80740FFF7DEFF7A
:10F22800024B00221A7002B010BD00BF9A1C0020C9
:10F2380007B501228DF807000DF107018020FFF7BF
:10F24800CDFF9DF80730002B034B14BF022201228B
:10F258001A7003B05DF804FB9A1C002007B5094B2F
:10F268008DF8060004221A70030C8DF8043003226E
:10F27800030A01A983208DF80530FFF7AFFF03B01B
:10F288005DF804FB9A1C002010B51446FFF790FFA8
:10F298002046BDE81040FFF7E1BF000007B5094B65
:10F2A8008DF8060005221A70030C8DF8043003222D
:10F2B800030A01A982208DF80530FFF78FFF03B0FC
:10F2C8005DF804FB9A1C002073B5002640F6E200A6
:10F2D8000196FFF7CFFE00F0FE01054640F6E2007A
:10F2E800FFF7B8FE40F6E500FFF7C4FE00F07F0127
:10F2F800044640F6E500FFF7ADFE6FF07F40FFF7EC
:10F30800CDFF04220DEB020140F61900FFF730FF94
:10F318003046FFF78DFF294640F6E200FFF79AFED8
:10F32800214640F6E500FFF795FE019802B070BD52
:10F3380013B50C4B04460522972140F6AC001A7011
:10F34800FFF788FE230C8DF804300322230A01A955
:10F3580082208DF805308DF80640FFF73FFF02B098
:10F3680010BD00BF9A1C002007B5030C8DF80030B3
:10F37800030A8DF801300B0C49BA8DF80200ADF87C
:10F3880004100622694694208DF80330FFF726FF03
:10F39800024B06221A7003B05DF804FB9A1C002089
:10F3A800002208B51146C520FFF718FF014B0722B8
:10F3B8001A7008BD9A1C002000221146D120FFF7C0
:10F3C8000DBF00221146D220FFF708BF07B5012262
:10F3D8008DF807000DF107019F20FFF7FFFE03B02E
:10F3E8005DF804FB07B501228DF807000DF1070150
:10F3F800A020FFF7F3FE9DF807103F2907D901F079
:10F40800F8010131C9B240F20670FFF723FE03B0DC
:10F418005DF804FB07B5F4F765FC431E58425841F4
:10F428008DF8070001220DF107019620FFF7D6FE9F
:10F4380003B05DF804FB07B500F07F008DF8070006
:10F4480001220DF107018920FFF7C8FE03B05DF81E
:10F4580004FB0000154B984207B51BD8144B984283
:10F468001BD8144B98421BD8134B98421BD8134BEC
:10F4780098428BBF6B2229226F232B238DF80420FF
:10F4880001A9022298208DF80530FFF7A7FE03B0E6
:10F498005DF804FBE122E923F0E7D722DB23EDE75F
:10F4A800C122C523EAE775228123E7E700E9A435ED
:10F4B80080F8A9328044E52D000B6B1B40FC5419E1
:10F4C80007B58DF8062004228DF804008DF8051084
:10F4D80095200DEB02018DF80730FFF77FFE03B092
:10F4E8005DF804FB07B552BAADF8042040BA08220B
:10F4F80049BAADF80000ADF802105BBA694610468B
:10F50800ADF80630FFF76AFE03B05DF804FB07B5F7
:10F518000B0C042200F0070049BA8DF80400ADF87E
:10F52800061097200DEB02018DF80530FFF756FE07
:10F5380003B05DF804FB000010B508B1194B186062
:10F54800F3F7CEF80220FFF7A5FD0024164B20465E
:10F558001C70FFF76DFEF4F7C3FB012817D14FF4B9
:10F568002071FFF7D4FF40F611102146FFF772FD16
:10F578004FF07F00FFF75FFF0E2140F61F10FFF7E7
:10F5880069FDF4F755FB094B01221A7010BD1021D3
:10F5980040F61110FFF75EFD102140F61210FFF73C
:10F5A80059FDE9E78C1C0020901C00209A1C0020C3
:10F5B80037B50C4D2B7804461BB9FFF74BFF0123D9
:10F5C8002B700023084A6006E109F2F79DFA04222D
:10F5D80000BA01900DEB02018620FFF7FFFD03B092
:10F5E80030BD00BF901C00200048E80107B5094B5A
:10F5F8008DF807000146187018B940F2AC60FFF7A3
:10F6080029FD01220DF107018A20FFF7E7FD03B06C
:10F618005DF804FB991C0020012873B50C461646BA
:10F6280037D10020F4F760FBA042B8BF44B20E28DF
:10F6380005461AD101231A4600210420FFF740FF8E
:10F648006FF010039C42B8BF1C46182140F6E70033
:10F65800FFF700FD022201A98E208DF804408DF8E5
:10F668000560FFF7BBFD02B070BD01230A28E4B2B4
:10F678001A464FF0000105D11846FFF721FF033461
:10F6880064B2DDE70720C5F10E05FFF719FF2C442A
:10F69800F6E740F6D800FFF7EDFC40F01E01C9B2CE
:10F6A80040F6D800FFF7D6FC0120F4F71DFBA04276
:10F6B800B8BF44B2142805464FF001034FF00002CA
:10F6C8000CD105210320FFF7FBFE023464B26FF072
:10F6D80008039C42B8BF1C463821B7E7112805D15A
:10F6E80003210220FFF7ECFE0534EFE70E2804D1D2
:10F6F80002210846FFF7E4FEE9E7C5F116050721F0
:10F7080004202544FFF7DCFE6CB2E0E713B5314A6C
:10F718000446516810686B4603C32F4B20781B784A
:10F72800834201D0FFF762FF2378032B27D8DFE855
:10F7380003F00239283C6268284BB3FBF2F31A0C39
:10F74800A1688DF800208DF802301A0A237B8DF805
:10F758000330637B8DF801208DF80430204A0023A4
:10F768004806C909F2F7D0F9030C40BA8DF80530FC
:10F77800ADF80600082269468B20FFF72FFD02B07E
:10F7880010BD2269154BB3FBF2F31A0C8DF800205B
:10F798008DF802301A0A237D8DF801208DF8033088
:10F7A8000422E8E7A3690093FAE762680B4BB3FB0E
:10F7B800F2F31A0C8DF800208DF802301A0A237B18
:10F7C8008DF80330637B8DF801208DF80430052215
:10F7D800D1E700BFB0090108991C00200000093DCD
:10F7E8000048E8011FB52E4A0446D1689068127C8B
:10F7F80001AB03C31A702B4B20781B78834201D0CE
:10F80800FFF7F4FE2378032B26D8DFE803F002384D
:10F818003302637AF12B21D14FF6FF70FFF784FC96
:10F8280048F20500FFF792FC02236288A188ADF830
:10F83800061052BAE188ADF804208DF80B30227A10
:10F84800A37A8DF80A20ADF808108DF80C3009223B
:10F8580001A98C20FFF7C2FC04B010BDF22BE4D143
:10F8680041F60F50FFF760FC41F22100FFF76EFCF4
:10F878000623DAE7237B8DF804300122E8E7E389E1
:10F88800094A5BBAADF80430237C13708DF8063052
:10F89800637C8DF80730638AADF808300622D7E715
:10F8A800B0090108991C0020981C002007B5022205
:10F8B8008DF804008DF805108F2001A9FFF78EFC44
:10F8C80003B05DF804FB000010B51346EFF3108495
:10F8D80072B60A4601460348F6F730FD84F31088ED
:10F8E80010BD00BF3802002007B5012201A915206C
:10F8F800FFF7EAFF9DF804004042401003B05DF8AE
:10F9080004FB000037B505460C46022201A9132066
:10F91800FFF7DAFF0A4B1B78012B0DD1094B1B7837
:10F92800012B09D140F20270FFF7A4FB9DF80530C6
:10F938002870237003B030BD9DF80400F6E700BFBF
:10F94800991C0020981C0020F7B50D460646002497
:10F958000DF10701284617468DF80740FFF7D2FF3B
:10F968002A78BA4207D89DF807003146FFF726FCE7
:10F97800204603B0F0BD0120FBE7000013B50322C9
:10F98800044601A91420FFF79FFF184B1A7822702C
:10F998004AB1012A17D014220021204600F0D0FADB
:10F9A8000F2323700DE09DF8043023719DF8053076
:10F9B800A2605B425B10A3719DF806305B425B104E
:10F9C800637102B010BD9DF804305B425B10237375
:10F9D8009DF9053002339B1063739DF806305B4236
:10F9E8005B10A373024B1B682361EAE7991C002094
:10F9F800941C0020012908B5034608460ED1012BA6
:10FA080007D10420FFF746FB0220BDE80840F4F7C1
:10FA180043B9022B14BF08460320F6E70120F4E798
:10FA280038B50446F4F75AF950B102280CBF02253C
:10FA38000125284602222146FFF7EEFD284638BD5B
:10FA4800102CB4BF01250225F3E70A2070470000F7
:10FA5800014B01201B6818478C1C0020014B022019
:10FA68001B6818478C1C0020014B40201B68184756
:10FA78008C1C002011B1012904D07047044B1B686D
:10FA880080201847024B4FF480701B68F9E700BFCD
:10FA98008C1C0020024B4FF400701B68184700BFF5
:10FAA8008C1C0020014B20201B6818478C1C002050
:10FAB800014B04201B6818478C1C0020014B0820B0
:10FAC8001B6818478C1C0020014B10201B68184726
:10FAD8008C1C0020024B4FF480401B68184700BF65
:10FAE8008C1C002010B568B1074A002352F8334037
:10FAF800844202EBC30101D9087910BD0133162BEA
:10FB0800F4D1FEE71F20F8E75013010873B51D4B29
:10FB18000193044640F607000D46FFF7ABFAC0F321
:10FB2800C10308336B4413F8042C00F007030133B6
:10FB380002FA03F3144AB2FBF3F2B2FBF4F007281B
:10FB48001ED84000042834BF042302234FF4D66093
:10FB580002FB03F4FFF78EFA060240F2B160FFF7EA
:10FB680089FA06F470663043030544BF6FEA005013
:10FB78006FEA105063094343DB112B6002B070BD7C
:10FB88000123E3E704080A0C0048E8014FF0FF30BE
:10FB980070474FF0FF3070474FF0FF3070477047A5
:10FBA800002070470020704770474FF0FF307047C3
:10FBB8004FF0FF30704770477047704770B5EFF3EC
:10FBC800108672B6144B5C8A1A8A944213D1C4F513
:10FBD800806292B2904206D3844218D901229A7068
:10FBE80000221C805A825A8A0A800244C2F30902FF
:10FBF8005A8200200DE006D9C4F58065ADB2854271
:10FC0800F1D88242E9E7121B92B28242EBD84FF058
:10FC1800FF3086F3108870BD9C220020EFF310811E
:10FC280072B6034AD38A0133D38281F310887047AE
:10FC38009C220020EFF3108172B6034AD38A013B5D
:10FC4800D38281F3108870479C22002010B50848A1
:10FC58001822002100F074F906484FF48062002150
:10FC680000F06EF9044B05481B68BDE810401847C2
:10FC78009C2200209B1E0020500A0108F1FD00086C
:10FC8800014B5860704700BF9C220020014B18723E
:10FC9800704700BF9C22002073B5EFF3108572B641
:10FCA8001C4CE08A00282FD1FFF7B8FF218A628A0E
:10FCB800914227D0A378012B12D1238820805B1A88
:10FCC8009BB20221A382A17063B9A3702382238A05
:10FCD8009A428BBFD21AC3F58063A282A38201E045
:10FCE800002BF4D0268A0C4B1E4485F31088F2F7BB
:10FCF800E1FD0A4BA18ADB680193304602B0BDE8FA
:10FD080070401847FFF796FF85F31088002002B06F
:10FD180070BD00BF9C2200209B1E0020500A0108D5
:10FD280008B4F0B586B00023ADF800302B4B0B9C1F
:10FD38001D7A85424CD3D86881434CD15B681BB18E
:10FD480012B1694602A898470CAB22464FF40071DD
:10FD58002348019300F0F4FBFFF760FFBDF8003083
:10FD680018440DF1020180B2FFF728FF01302AD0B4
:10FD78000023BDF80020BDF802601A480DF1080CF8
:10FD88001F4699B216FA83F58A42ADB215D817B153
:10FD98003244ADF80220BDF80250019B22464FF4D0
:10FDA8000071284400F0CCFBFFF744FFFFF774FF15
:10FDB80006B0BDE8F04001B070471CF8011B415582
:10FDC80001330127DDE7FFF735FF6FF00200EFE7AA
:10FDD8006FF00400ECE76FF00500E9E79C220020D3
:10FDE8009B1C00209B1E002013B5EFF3108472B6F5
:10FDF800204B9A78588A022A1DBF1A8A998A521863
:10FE0800002214BFC2F309029A7090421A8228D0C5
:10FE1800D98A012925D19978012913D119888A1AF3
:10FE2800022192B2997000219A82198062B99A705F
:10FE38001A821A8A90428BBF801AC2F58062988211
:10FE48009A8201E00029F4D0188A0B4A104484F3FE
:10FE580010880A4A998AD368019302B0BDE8104015
:10FE6800184784F31088F2F729FD02B0BDE8104066
:10FE7800FFF7E0BE9C2200209B1E0020500A0108CC
:10FE8800024A00231360024A13607047B822002018
:10FE9800B422002010B5EFF3108472B641B10129E5
:10FEA80003D1064A13680343136084F3108810BD16
:10FEB800024A136823EA0003F6E700BFB8220020CD
:10FEC80010B5EFF3108472B641B1012903D1064A87
:10FED80013680343136084F3108810BD024A136843
:10FEE80023EA0003F6E700BFB422002038B5EFF399
:10FEF800108572B60A4B0B4C1B6833B123689847C0
:10FF08006368984785F3108838BD074B1B681BB199
:10FF1800A3689847E368F4E7236998476369F0E7BB
:10FF2800B8220020DC090108B422002001380A4464
:10FF3800914200D1704711F8013B00F8013FF7E703
:10FF480000F030BC10B5EFF3108472B6064A13689F
:10FF580003431360054A52F83130034342F8313005
:10FF680084F3108810BD00BF08230020BC220020A5
:10FF780070477047B0F5803F3ABF00041023002354
:10FF8800B0F1807F3EBF08330002DBB2B0F1805F82
:10FF980038BF00014FEA1070054A38BF0433125CBD
:10FFA80038BFDBB2C3F11F03981AC0B2704700BF55
:10FFB800001401082DE9F84F384D394ED5F8008066
:10FFC800DFF8E0B0DFF8E0A0DFF8E090D6F800C096
:10FFD800374FDBF80010374CDAF80020D9F800303A
:10FFE80008EA00002860286800EA020E1EEA0C0FE2
:08FFF80001D019421ED04FF0A8
:020000040801F1
:10000000FF333B60FFF7B8FFEFF3108472B633683D
:10001000DBF80020DAF800100B4029680B4205D10C
:10002000D9F80030134201D1F2F7D6FB84F31088DF
:10003000FFF7A3FFC5F80080BDE8F88F23682368A9
:100040000340134062681A4204BF4FF0FF326260FF
:1000500060681840FFF792FF62683860012303FA76
:1000600000F022EA00026260EFF3108172B63A6893
:100070009340326822EA03023260226822EA0303D4
:10008000236081F310880E4A3B6852F8233098476A
:10009000D6F800C0DBF80010DAF80020D9F80030FC
:1000A000A5E700BF4401002008230020042300200E
:1000B0004801002000230020FC220020BC22002058
:1000C000C422002010B51146EFF3108472B6FFF77A
:1000D00055FF034B43F8201084F3108810BD00BF78
:1000E000C422002082B082B00DF1080C0CE9060099
:1000F000BDF8042003930B44BDF810100A4491B2DC
:1001000012B2B2F57A7FA2BFA1F57A72013312B2B0
:100110000360828002B002B0704782B082B00DF1FD
:10012000080C0CE90600BDF804200393CB1ABDF8B7
:100130001010521A91B212B2002ABEBF01F57A72A3
:1001400003F1FF3312B20360828002B002B0704745
:1001500030B585B0114D6B4683E803000023029350
:10016000ADF80C3003A82B699847009BBDF80440FC
:100170000290181ABDF80C30E41AA3B224B2002C75
:10018000BEBF03F57A731CB200F1FF302B689847AD
:10019000AB682046984705B030BD00BF100A010883
:1001A00073B5114E002305460093ADF8043001A845
:1001B00033699847F36800909847736804469847F6
:1001C000009B1844BDF8043023449AB21BB2B3F527
:1001D0007A7FA2BF0130A2F57A731BB2286028464D
:1001E000AB8002B070BD00BF100A010837B5002314
:1001F0000093ADF80430074B04461B6901A89847EB
:100200006D46009095E8030084E80300204603B0A3
:1002100030BD00BF100A010837B50F4D02AB03E92E
:100220000300EB6898476B6804469847BDF80430B4
:10023000009A1B1B99B21BB2002BA2EB0002BEBF9F
:1002400001F57A7102F1FF320BB24FF47A7000FBC4
:10025000023003B030BD00BF100A01082DE9F041A3
:100260004FF47A75B1FBF5F5C5EB4513DFF83C802B
:1002700005EB8303A1EBC3039CB2D8F80C30064610
:100280009847D8F8043007469847E31999B21BB24B
:10029000B3F57A7F2844A2BFA1F57A7301301BB26F
:1002A0003060B3803046BDE8F08100BF100A01081D
:1002B000024B00221A60024B1B6818470C230020D7
:1002C000240A0108F8B50446174608461E467CB1C4
:1002D00073B1084B00255B6A25609847069B6060F8
:1002E0002581A572E6602361E77265612846F8BD45
:1002F0000120FCE7240A010810B5034CE369984784
:10030000A36ABDE810401847240A010870B5064DDD
:10031000EB69064698476B6A044630469847AB6AD5
:10032000201ABDE870401847240A0108054B1B68D5
:100330000BB918467047834201D05B69F8E701208A
:10034000704700BF0C2300202DE9F3410B4E336AA8
:10035000044698470123B7692372D4F80080054604
:10036000B8472844804502D2B84728442060B36883
:100370002068019302B0BDE8F0411847240A010843
:1003800070B520B3EFF3108672B6124D2B680122C0
:10039000827253B10022427298425C690ED102729D
:1003A0003CB120462C60FFF7CFFF86F31088002079
:1003B00070BD094BDB6898472C60F6E71A465B690D
:1003C000002BF2D09842F9D143695361EDE7012047
:1003D000EEE700BF0C230020240A0108084B10B5EB
:1003E0001A685369516911B95061416110BD0468BF
:1003F00019688C4202D91A465B69F3E71946F3E79C
:100400000C230020044A13680BB1002119724361C8
:100410001060FFF799BF00BF0C2300202DE9F041C9
:10042000044600282DD0FFF781FF50BB657A45BBFD
:10043000EFF3108872B6144E6768336A98478742A4
:100440002CBF27602060114FA5724FF48073238169
:100450003B684BB9336998472046FFF7D3FF88F3D1
:1004600010882846BDE8F081B3699847236818448E
:100470003B6820601B6898422046EED3FFF7AEFF32
:10048000EDE70125EDE700BF240A01080C23002059
:1004900010B5044608467CB1084B5B6A984760601B
:1004A0002046FFF743FF40B12046FFF769FF204693
:1004B000BDE81040FFF7B2BF012010BD240A0108BB
:1004C0002DE9F041EFF3108772B61D4E1D4D736993
:1004D00098473369044698472B684BB94FF000089A
:1004E0002B688BB9286828BB87F31088BDE8F0819A
:1004F000011B241A1A688A428CBF121900221A6042
:100500005B69002BF6D1E9E71C681CB1B369984719
:100510008442E7D22C6863692B60A4F80880D4E990
:10052000033098476389B3F5807FD9D12046FFF720
:1005300075FFD5E7037A002BD6D1FFF705FFD3E788
:10054000240A01080C2300202DE9F04F002997B060
:1005500081461E4640F3118104464F1E1378A4EBDA
:10056000090023B90023237017B0BDE8F08FB8420B
:10057000F8DA252B05D004F8013B904608F101027A
:10058000ECE792F801E0AEF1300102F10108AEF1C2
:1005900030034A424A41092B2BD8414600250A2004
:1005A000884611F8013BA3F1300CBCF1090F1BD9AF
:1005B00098F80030692B00F09E801DD8632B29D05D
:1005C000642B00F09880582B5AD0252B1AD198F81C
:1005D0000030002B00F0938004F8013BA4EB0903EA
:1005E000BB4280F28A80C9E700FB0533A3F13005E6
:1005F000D6E74FF0FF35DBE7752B7ED0782B41D067
:10060000732B1CD0252304F8013BA4EB0903BB4248
:1006100073DADCE7002D05F1FF3AD8BF4FF0000A8E
:1006200052462046202100F0C1F8A244002D56F881
:10063000043B8AF80030D8BF01252C449EE7504B7C
:1006400056F804BBBBF1000F08BF9B465846F0F7B5
:10065000B7FE2A1A8542B8BF0022824620212046D2
:10066000019200F0A3F8019A00232244534502DBD3
:1006700002EB0A0482E71BF80310D1540133F5E7BB
:1006800042F040021021DFF8FCB0DFF8FCA056F881
:1006900004CB12F0400F18BFDA46BEF1300FCDF890
:1006A00008A0A4EB09030CBF4FF0300A4FF0200A5A
:1006B0009207A7EB03036046CDF80CA022D50028D3
:1006C00020DA4042013D4FF02D0C05AA0192002294
:1006D0008246B0FBF1F001FB10AB029810F80BB0B2
:1006E000019800F801BB5145019002F10102BAFBEB
:1006F000F1F0EDD910E042F002020A21C3E708F15F
:10070000FF386BE7BCF1000F02D04FF0000CDCE7C4
:1007100030228DF814200122BEF1300FA5EB020526
:1007200004D02020002D05F1FF350ADCBCF1000FBC
:1007300005D02D21013B04F8011B3FF41FAF2544D8
:100740000AE0013B04F8010BECD117E7039904F828
:10075000011B013B3FF412AF291B0029F6DC05A960
:10076000114423442244A2423FF408AF11F8010D82
:1007700004F8010B9C42F6D100E70020F4E600BF2C
:10078000101401083C1401081714010810B50139B0
:100790000244904201D1002005E0037811F8014F96
:1007A000A34201D0181B10BD0130F2E702440346FA
:1007B000934200D1704703F8011BF9E770B50D4D66
:1007C0000D4C641BA4100026A64209D10B4D0C4C05
:1007D00000F0B2F8641BA4100026A64205D170BD3B
:1007E00055F8043B98470136EEE755F8043B984727
:1007F0000136F2E7441501084415010844150108C3
:100800004815010800F003B8002200F00EB80A44B1
:10081000914200F1FF3300D1704710B511F8014B40
:1008200003F8014F9142F9D110BD13460A4619460B
:10083000FFF7BCBF000000002DE9F041C1F30A57EB
:10084000A7F2FF36132E02460B460C46054680469D
:1008500035DC002E17DA34A3D3E90023F0F7BEFD10
:1008600000220023F0F7EEFF50B1002C57DA24F0FD
:1008700000442C430025AC422D4C08BF4FF00044EF
:1008800023462A4624E02B4F374101EA070C5CEA55
:10089000000C1DD024A3D3E90023F0F79FFD002214
:1008A0000023F0F7CFFF0028EAD0002CBEBF4FF4A2
:1008B00080133341E41824EA07040025E0E7332ECF
:1008C0000ADDB6F5806F03D1F0F788FD02460B46CE
:1008D00010461946BDE8F081A7F213474FF0FF3CE0
:1008E0002CFA07F70742F3D00FA3D3E90023F0F760
:1008F00075FD00220023F0F7A5FF0028C0D0002CD2
:100900000ADA142E01D1013406E0C6F134060123BF
:10091000B3401D444545F6D325EA0705B0E7002559
:100920002C46ADE7AFF300809C7500883CE4377E31
:100930000000F0BFFFFF0F00F8B500BFF8BC08BC17
:100940009E467047F8B500BFF8BC08BC9E4670478D
:100950000000000001000000020000000000000094
:100960008813000010270000204E000030750000A2
:10097000409C000050C3000060EA0000C0D40100A9
:1009800080A903000053070000EA063700000000BA
:100990005000000040F70937000000005000000040
:1009A000C194C10000000000B22700000000000058
:1009B0000000000000000000000000000000000037
:1009C00000000000B5010008F1010008C409010899
:1009D000FC7F003F00350113C4120008B325000856
:1009E00099250008612500089D2500085D2500085F
:1009F000C52500085975336E3148344F3152354E94
:100A0000395332543653256473253033643A000029
:100A1000CD2900086D2A0008DD290008792A000880
:100A20003D2A0008852A000800000000ED29000882
:100A3000A529000871290008292900088129000832
:100A40009529000835290008392900084D29000892
:100A5000012D0008292D0008AD2C0008992C000854
:100A600052464143005056585858002159756E4817
:100A70006F726E205354532052657669766521005B
:100A8000A0860100400D0300801A060000350C000E
:100A900040420F0080841E0000093D0000127A00D1
:100AA0000024F40000366E010048E801006CDC020E
:100AB0000000000000000000000000000000000036
:100AC0000000000000000000000000000000000026
:100AD000010000000200000003000000040000000C
:100AE00001000000030000000500000001000000FC
:100AF00001000000060000000A00000020000000C5
:100B000002000000040000000800000010000000C7
:100B10004000000080000000000100000002000012
:100B2000010002000400060008000A000C0010008A
:100B300020004000800000010804020408010101B7
:100B400001010103070100006572726F723A2052C1
:100B50006567696F6E206973206E6F7420646566C7
:100B6000696E656420696E20746865204D573A206F
:100B7000736574206C6F726177616E5F636F6E6610
:100B80002E68206163636F7264696E676C790D0A09
:100B9000004D414320727854696D654F75740D0A9C
:100BA000004D414320747854696D654F75740D0A8A
:100BB000004D4143207278446F6E650D0A004D412F
:100BC00043207478446F6E650D0A00080A0C0D0E00
:100BD00010121415181A1B1D1E21240305020501ED
:100BE00006020205000006000001050404020202DC
:100BF00002020202020202020202020203020202D4
:100C000002020203040302020202020405040302B8
:100C10000202020506050403020202060706050495
:100C20000302020707070605040302070700000086
:100C300000000001020100000000000203020100A8
:100C40000000000304030201000000040504030285
:100C5000010000050605040302010006070605045D
:100C60000302010707070605040302070700000B3C
:100C7000357DF2F2F233337373DEDEDEDE3333734F
:100C800073F2F2F2F200000048E8010048E80100C7
:100C900048E8010048E8010048E8010048E8010090
:100CA00090D00300000000000C0B0A09080707326F
:100CB00052585F2573206F6E20667265712025641F
:100CC00020487A2061742044522025640D0A005285
:100CD00058206F6E206672657120256420487A2046
:100CE00061742044522025640D0A005458206F6E10
:100CF000206672657120256420487A206174204442
:100D0000522025640D0A00310032004D756C746963
:100D10005F43004D756C74695F500000070D01085A
:100D2000090D0108630A01080B0D0108190D0108DE
:100D3000130D0108A584998D0DBDB1545003A97DF3
:100D40001962E69A459D408715EBC90BEC67FDEAF1
:100D5000BFF7965BC21CAE6A5A41024F5CF434087E
:100D60009373533F0C52655E28A10FB509369B3D26
:100D70002669CD9F1B9E742E2DB2EEFBF64D61CEE3
:100D80007B3E7197F568002C601FC8EDBE46D94BBD
:100D9000DED4E84A6B2AE516C5D75594CF100681F4
:100DA000F044BAE3F3FEC08AADBC4804DFC175630A
:100DB000301A0E6D4C14352FE1A2CC3957F2824710
:100DC000ACE72B95A098D17F667EAB83CA29D33C34
:100DD00079E21D763B564E1EDB0A6CE45D6EEFA693
:100DE000A8A4378B324359B78C64D2E0B4FA0725F4
:100DF000AF8EE918D5886F7224F1C751237C9C21EE
:100E0000DDDC86859042C4AAD8050112A35FF9D023
:100E1000915827B93813B333BB7089A7B6229220F3
:100E200049FF787A8FF88017DA31C6B8C3B07711E6
:100E3000CBFCD63AC6F8EEF6FFD6DE916002CE566F
:100E4000E7B54DEC8F1F89FAEFB28EFB41B35F45DA
:100E50002353E49B75E13D4C6C7EF5836851D1F9D9
:100E6000E2AB622A0895469D30370A2F0E241BDF1D
:100E7000CD4E7FEA121D583436DCB45BA476B77DC4
:100E800052DD5E13A6B900C140E379B6D48D677216
:100E90009498B085BBC54FED869A66118AE904FE29
:100EA000A078254BA25D80053F2170F16377AF42AA
:100EB00020E5FDBF811826C3BE35882E9355FC7AE8
:100EC000C8BA32E6C0199EA344543B0B8CC76B28AA
:100ED000A7BC16ADDB647414920C48B89FBD43C424
:100EE0003931D3F2D58B6EDA01B19C49D8ACF3CF4E
:100EF000CAF447106FF04A5C38577397CBA1E83EAD
:100F000096610D0FE07C71CC9006F71CC26AAE6949
:100F100017993A27D9EB2B22D2A907332D3C15C9B3
:100F200087AA50A50359091A65D784D082295A1E69
:100F30007BA86D2C637C777BF26B6FC53001672BD0
:100F4000FED7AB76CA82C97DFA5947F0ADD4A2AFBD
:100F50009CA472C0B7FD9326363FF7CC34A5E5F1CB
:100F600071D8311504C723C31896059A071280E279
:100F7000EB27B27509832C1A1B6E5AA0523BD6B3CD
:100F800029E32F8453D100ED20FCB15B6ACBBE393D
:100F90004A4C58CFD0EFAAFB434D338545F9027F29
:100FA000503C9FA851A3408F929D38F5BCB6DA21E2
:100FB00010FFF3D2CD0C13EC5F974417C4A77E3D0E
:100FC000645D197360814FDC222A908846EEB81464
:100FD000DE5E0BDBE0323A0A4906245CC2D3AC6227
:100FE0009195E479E7C8376D8DD54EA96C56F4EA32
:100FF000657AAE08BA78252E1CA6B4C6E8DD741F43
:101000004BBD8B8A703EB5664803F60E613557B905
:1010100086C11D9EE1F8981169D98E949B1E87E9BF
:10102000CE5528DF8CA1890DBFE6426841992D0F6E
:10103000B054BB16232323232323202573202530DC
:1010400032583A253032583A253032583A25303223
:10105000583A253032583A253032583A25303258ED
:101060003A253032583A253032583A253032583AFB
:10107000253032583A253032583A253032583A2500
:101080003032583A253032583A253032580D0A005D
:10109000232323232323204465764555493A2020E2
:1010A00020202020253032583A253032583A253039
:1010B00032583A253032583A253032583A253032B3
:1010C000583A253032583A253032580D0A00232339
:1010D00023232323204170704555493A20202020A6
:1010E0002020253032583A253032583A25303258AF
:1010F0003A253032583A253032583A253032583A6B
:10110000253032583A253032580D0A002323232344
:10111000232320446576416464723A2020202020F5
:10112000253032583A253032583A253032583A254F
:101130003032580D0A004170704B65793A202020FA
:101140002020004E776B4B65793A2020202020002C
:101150004E776B534B65793A202020200041707008
:10116000534B65793A20202020004442496E744B4D
:1011700065793A202020004D43526F6F744B65799A
:101180003A2020004D434B454B65793A20202020E2
:10119000004D43417070534B65795F303A004D43C9
:1011A0004E776B534B65795F303A000000000000CA
:1011B0004150505F36110108010000004E574B5F4F
:1011C00043110108080000004E574B53501101080D
:1011D00009000000415050535D1101080A00000051
:1011E0004442495F6A1101080B0000004D4352540C
:1011F000771101080C0000004D434B458411010894
:101200000D0000004D434B30911101080E0000000D
:101210004D415330911101080F0000004D4E5330E5
:101220009E110108100000005A45524F6B12010830
:10123000526164696F53656E64204F76657273699D
:101240007A650D0A004952515F52585F54585F54F5
:10125000494D454F55540D0A00505245204F4B0DF6
:101260000A0053594E43204F4B0D0A004844522068
:101270004F4B0D0A00484452204B4F0D0A00495273
:10128000515F4352435F4552524F520D0A000201D3
:1012900000030000841E0000093D0000127A0000D7
:1012A00024F4000048E8010090D0030020A10700CA
:1012B00000000000B128000061510000C3A200003E
:1012C000040506000DE00008D1DE000809E1000871
:1012D0004DDF000821EA0008F5DF00084DE70008AF
:1012E000C5E50008B1DD00085DEC00089DEA0008D6
:1012F000E1DF0008C9DE000879DF000851DF0008DF
:1013000009DF0008FFDE000801DE0008FDDD00083F
:10131000FBDE0008F7DE0008A1E00008CDE00008D1
:10132000EDDE000879ED000861DE000829DE000826
:1013300049ED000805DE0008CDE3000855E100088E
:1013400095FB00089BFB0008F5DD0008F9DD0008AF
:10135000C01200001F000000A816000017000000C7
:10136000841C00000F000000E42500001E000000A7
:10137000B42D000016000000083900000E00000027
:101380002C4C00001D000000685B000015000000F0
:10139000747200000D000000589800001C0000004E
:1013A00034B7000014000000E8E400000C00000066
:1013B000783101001B000000686E0100130000007E
:1013C00034CA01000B000000286202001A0000006D
:1013D00040DB0200120000003C9303000A00000002
:1013E000C0C204001900000060B305001100000035
:1013F000382007000900000020A1070000000000BD
:1014000004030202010101010000000000000000CD
:101410003C4E554C4C3E0030313233343536373843
:10142000396162636465666768696A6B6C6D6E6F6B
:10143000707172737475767778797A0030313233DF
:101440003435363738394142434445464748494A9E
:101450004B4C4D4E4F505152535455565758595A64
:041460000000000088
:101464000000000000000000000000000000000078
:101474000000000000000000002B7E151628AED2EC
:10148400A6ABF7158809CF4F3C012B7E151628AE65
:10149400D2A6ABF7158809CF4F3C082B7E1516282A
:1014A400AED2A6ABF7158809CF4F3C092B7E151693
:1014B40028AED2A6ABF7158809CF4F3C0A0000002E
:1014C400000000000000000000000000000B00000D
:1014D40000000000000000000000000000000C00FC
:1014E4000000000000000000000000000000000DEB
:1014F40000000000000000000000000000000000E8
:101504000E000000000000000000000000000000C9
:10151400000F0000000000000000000000000000B8
:1015240000001000000000000000000000000000A7
:081534000000000000000000AF
:08153C0084FEFE7F01000000A7
:041544005D0100083D
:04154800390100085D
:10154C0000000000B903002010270000000001007B
:10155C00000000000000000000000000040000007B
:10156C00401F0000DD2700080D2800082528000872
:10157C0091280008992F00088D310008F52E0008DD
:10158C00B731000800000000FD2E0008D53000081F
:10159C00653B0008D92E0008D72E0008BD31000885
:1015AC00352F0008DD2E0008E92E000859310008FF
:1015BC000200180101054D3C4D0400002008190FD4
:1015CC0028040A413F00050A010000050203FFFF41
:1015DC00FFFFFFFFFFFFFFFF0F01030002000000F2
:1015EC0000000000000000000000000000000000EF
:1015FC0000000000C0D4010000093D0010000000F4
:10160C0000000000000700200000000000000000A7
:10161C00FF00000000000000000700200000000098
:10162C0000000000000000000000000000000000AE
:10163C00000700200000FF0000000000E000000098
:10164C000D8100083D800008498000087580000865
:10165C0000000000000000006581000855800008B3
:10166C00D58400080000000000000000000000000D
:10167C0000000000000E0F0D010908110100000010
:0C168C00FF000000FFFFFFFFFFFFFFFF5B
:0400000508003CFDB6
:00000001FF
